:020000040000fa
:080000000014040000000000e0
:020000040000fa
:100008004015000040150000401500004015000094
:100018004015000040150000401500004015000084
:100028004015000040150000401500004c8b0000f2
:10003800401500004015000040150000647d0000d8
:10004800401500004015000040150000000f00009a
:10005800e00e0000401500004015000040150000ab
:100068004015000040150000401500004015000034
:100078004015000040150000401500004015000024
:100088004015000040150000401500004015000014
:100098004015000040150000726800005a68000012
:1000a80040150000401500004015000040150000f4
:1000b80040150000401500004015000040150000e4
:1000c80040150000401500004015000040150000d4
:1000d80040150000401500004015000040150000c4
:1000e80040150000401500004015000040150000b4
:1000f80040150000401500004015000040150000a4
:100108004015000040150000401500004015000093
:100118004015000040150000401500004015000083
:100128004015000040150000401500004015000073
:100138004015000040150000401500004015000063
:100148004015000040150000401500004015000053
:100158004015000040150000401500004015000043
:100168004015000040150000ca680000b268000091
:100178004015000040150000401500004015000023
:100188004015000040150000401500004015000013
:100198004015000040150000401500004015000003
:1001a80040150000401500004015000040150000f3
:1001b80040150000401500004015000040150000e3
:1001c80040150000401500004015000040150000d3
:1001d80040150000401500004015000040150000c3
:1001e80040150000401500004015000040150000b3
:0801f800401500004015000055
:020000040000fa
:100208004015000040150000401500004015000092
:100218004015000040150000401500004015000082
:100228004015000040150000401500004c8b0000f0
:10023800401500004015000040150000647d0000d6
:10024800401500004015000040150000000f000098
:10025800e00e0000401500004015000040150000a9
:100268004015000040150000401500004015000032
:100278004015000040150000401500004015000022
:100288004015000040150000401500004015000012
:100298004015000040150000726800005a68000010
:1002a80040150000401500004015000040150000f2
:1002b80040150000401500004015000040150000e2
:1002c80040150000401500004015000040150000d2
:1002d80040150000401500004015000040150000c2
:1002e80040150000401500004015000040150000b2
:1002f80040150000401500004015000040150000a2
:100308004015000040150000401500004015000091
:100318004015000040150000401500004015000081
:100328004015000040150000401500004015000071
:100338004015000040150000401500004015000061
:100348004015000040150000401500004015000051
:100358004015000040150000401500004015000041
:100368004015000040150000ca680000b26800008f
:100378004015000040150000401500004015000021
:100388004015000040150000401500004015000011
:100398004015000040150000401500004015000001
:1003a80040150000401500004015000040150000f1
:1003b80040150000401500004015000040150000e1
:1003c80040150000401500004015000040150000d1
:1003d80040150000401500004015000040150000c1
:1003e80040150000401500004015000040150000b1
:0803f800401500004015000053
:020000040000fa
:100400000000fa000b380700a4d32000340290004b
:100410008402e800a4d3200035029800a4d3200071
:1004200034029000e00f520017003a00a4d32000dd
:10043000240290008402e800a4d320002502980042
:10044000a4d3200024029000e00f52000e003a00d6
:10045000a4d32000140290008402e800a4d320005a
:1004600015029800a4d3200014029000e00f52005f
:1004700005003a00a4d32000140278008402e800aa
:10048000a4d32000050a78000080fa0000000600ce
:100490000400fa000002eb00040f78002e4307006e
:1004a000d93f0700433107006b3c0700a706070050
:1004b0007038070091430700e43d070060d4200036
:1004c000d940070000027800e00f52001700320008
:1004d00014002000346a880004202c00150020003d
:1004e000446a8800556a880034868000846a8800df
:1004f0006022b800646a8800756a88000002eb0018
:10050000946a88000002eb00a46a88003000200092
:1005100086030700610b2d0030002000d231070058
:1005200060d42000dc4007000200370030002000cb
:100530007e030700946a80006102620084007800f4
:10054000100020000d400700946a800062026200e3
:10055000840078002000200008400700946a800092
:10056000640262008400780010002000314007001f
:10057000946a8000680262008400780020002000f5
:100580002c400700946a80007002620084007800aa
:1005900010002000cc3f0700956a80000402200074
:1005a000048262008400780020002000c63f07001b
:1005b000a46a800004007800933d0700300020000a
:1005c00071030700300020001b04070020002000fa
:1005d00056030700200020006b03070020002000c6
:1005e00015040700846a800034868800446a80000d
:1005f000556a8000366a8000064378008001eb006f
:100600000041eb00864078000000eb0088360700d0
:100610006037070034868000e00f52000a00320085
:1006200010002000933f0700070037000000000083
:100630000500370000000000030037000000000044
:1006400001003700000000000f3c070000027800a6
:10065000140798006aff0700146a8000e00f520038
:10066000190032001e029000e00f5200010032001b
:10067000f93d070034868000e00f5200ebff3200a6
:100680001e029000e00f5200eaff32001e0fe80049
:100690001e027800f90f5200e8ff36000002eb005e
:1006a000040f78007f3f07000002780004f0a700e5
:1006b0000402ea000402e9004f22de000400780090
:1006c0006c3f0700e0ff3700300020009531070045
:1006d00000027800e00f52000300320030002000da
:1006e0007002070007003700200020008d3107004e
:1006f00000027800e00f52000200320020002000cb
:1007000068020700b4728000e00f5200cdff320093
:100710000002eb00040078000080fa0000000600f0
:100720000a00fa0020079800310798004207980055
:100730000002eb00040f780014002000146a880007
:10074000be029000743e2000848f52002c003600c0
:10075000be0290004e02900084824200c43e2000ff
:10076000848f520026003e0024868000be02900046
:1007700004825200140798001d003700a5d3200002
:100780001e0290000402420004824200140278001b
:100790004822de0004427800ae029000844a7800cd
:1007a0002e0290000402e80024079800a5d3200040
:1007b0001e029000040242000482420014027800eb
:1007c00004427800ae029000844a78002e02900025
:1007d0000402e800240798001e0290000402e800ca
:1007e000140798004e0290000402e90044079800a4
:1007f0004e029000e00f5200e0ff3a000200370086
:1008000014002000040f78001e0278000400780015
:100810000080fa00000006001000fa00400798006f
:100820005107980062079800730798000002eb00d8
:10083000040f780014002000146a88005e02900003
:10084000ef0f520006003600de0290006e029000ac
:100850008482420024032000848f5200020036006c
:1008600014002000820037007e029000e00f52004a
:100870003d003a00de0290006e0290008482420049
:1008800004022000848f520034003600de02900003
:10089000e4022000848f520030003e00ee00900001
:1008a0005e0090007d3707002c0037000002eb004f
:1008b000140798005e029000ef0f52000700360008
:1008c0005e029000ff0f520004003e005e009000a8
:1008d0008d42070000027800140798005e02900025
:1008e000ff0f520008003600de02900014032000c3
:1008f000848f520004003e005e009000d73707004e
:1009000000027800140798001e0290004822de00c2
:1009100004427800ce029000844a78004e02900093
:100920000402e800440798001e0290000442780088
:10093000ce029000844a78004e0290000402e80043
:10094000440798006e0290000402e90064079800d2
:100950005e0290000402e800540798006e029000c6
:10096000e00f5200d1ff3a007e029000e10f5200ea
:100970003e003a00de0290006e0290008482420047
:1009800004022000848f520035003600de02900001
:1009900014032000848f520031003e006e0190004d
:1009a000de0090004e009000d8370700000278006b
:1009b000040f78002a0037004e029000144278009d
:1009c0000482fb00240798004e0290000402e80015
:1009d000440798002e0290004822dd00240798006a
:1009e0004e029000144278000482fb003407980005
:1009f0004e0290000402e80044079800ae02900006
:100a000004f02f00848262003e039000f40f200067
:100a10000402630004824200140798005e02900002
:100a2000ef0f5200080036005e029000ff0f5200e8
:100a300005003e009e0090005e0090007642070098
:100a400000027800040f78006e0290000402e900b2
:100a5000640798005e0290000402e80054079800c2
:100a60006e029000e00f5200d3ff3a001e027800a1
:100a7000040078000080fa00000006000400fa007c
:100a8000000f7800110798009e0278008400200073
:100a9000110009008402d800000278008102780069
:100aa0009e02900004824200144278008482fb007f
:100ab0001e03780074002000110009000403d80010
:100ac0000003780001027800160020000432dd00e7
:100ad00004826200040078000080fa000000060032
:100ae0000600fa00000f780011079800220798000e
:100af0002e029000e00f5200170032009e02780094
:100b000084002000809fbe00110009008402d800ec
:100b100000027800810278004f00be008402780055
:100b20001e039000050343009e02900004824200d1
:100b300014427800844278009e0378006782630044
:100b400017002000043add000442780004c272005d
:100b5000044b7800150037009e02780084002000c6
:100b6000110009008402d800000278008102780098
:100b7000840278001e039000050343009e0290004b
:100b80000482420014427800844278009e03780078
:100b90006782630017002000043add0004427800f9
:100ba00004c2ea0004c26200044b78000080fa002c
:100bb000000006000e00fa00300798004107980078
:100bc000520798006307980014002000146a8800f8
:100bd0004e029000e00f520005003200ce0290005d
:100be0005e02900004824200ea0f520002003600ca
:100bf00014002000c90037006e029000e10f52007f
:100c000053003a000002eb00040f78004400370064
:100c10009e0278004e029000048242001407980061
:100c2000be0090001e00780094ff070000027800cc
:100c3000240798001e0290006123b9000082eb0097
:100c40008082eb000602420087824a008600200074
:100c500007002000860f5200878f5a002d003e00ab
:100c600004600100080037000b0037000e00370059
:100c70001100370014003700170037001a00370042
:100c80001c0037001e003700ae009000100020004e
:100c90003a3e070021003700ae00900020002000ff
:100ca000363e07001d003700ae0090001000200007
:100cb000603e070019003700ae00900020002000c1
:100cc0005c3e070015003700ae00900010002000c9
:100cd000fd3d070011003700ae009000200020000d
:100ce000f93d07000d0037002e0290003486880081
:100cf0000a0037002e029000246a8800070037009f
:100d00000002eb00146a880010002000d93d0700a3
:100d10000200370014002000800037001e0fe8009a
:100d20009e0278005e029000848f5200b8ff390066
:100d300034868000e00f520003003a00246a8000ed
:100d400004007800cb3d07000002eb007300370081
:100d50006e029000e00f52006f003a005e029000b9
:100d60004322de000402e800040178008000eb006a
:100d70003e0090003a0907000002eb00040f7800e3
:100d80005f0037009e0278004e029000048242000d
:100d9000140798001e0290006123b9000082eb0046
:100da0008082eb000602420087824a008600200013
:100db00007002000860f5200878f5a004c003e002b
:100dc00004600100080037001000370018003700e9
:100dd0002000370028003700300037003800370087
:100de0003d00370044003700641780004222de00d7
:100df000614262000482fb0004017800be009000a2
:100e00001e00780036ff07003c00370064178000a2
:100e10004322de00614262000482fb00040178008c
:100e2000be0090001e0078002dff07003300370041
:100e3000641780004422de00614262000482fb00ed
:100e400004017800be0090001e00780024ff070017
:100e50002a003700641780004522de0061426200ec
:100e60000482fb0004017800be0090001e007800a0
:100e70001bff070021003700641780000442780040
:100e8000614262000482fb0004017800be00900011
:100e90001e00780012ff070018003700641780005a
:100ea0000402d100614262000482fb000401780068
:100eb000be0090001e00780009ff07000f003700f9
:100ec0003486800004017800be0090001e00780087
:100ed00003ff070009003700246a8000040178003e
:100ee000be0090001e007800fdfe070003003700e2
:100ef0001400200009003700000000001e0fe80069
:100f00009e0278005e029000848f52009dff39009f
:100f10000002eb00010037005400200004007800bc
:100f20000080fa00000006000600fa00000f7800ba
:100f3000110798002207980014002000146a880006
:100f400014002000040078000080fa000000060071
:100f50000c00fa004007980051079800d4c0b30075
:100f6000444798000002eb00040f78006602470037
:100f7000840078004e009000f32e070000027800f5
:100f8000e00f5200430032006e429000844078002f
:100f90004e009000092f07006e42900054479800c1
:100fa0005e429000ed4f520003003a00a1c0b30032
:100fb0004e009000012f0700de4290004e4290004c
:100fc00084cf5200180032005e429000e84f520079
:100fd0000b003200c4728000ff0f520008003c007a
:100fe000c4728000a5e52000850242005e439000a7
:100ff000864a78000402e800c472880006003700c0
:10100000c4728000e00f520003003400c4728000fc
:101010000402e900c4728800de0290000042eb0086
:10102000844a78001b00370014002000040f780069
:101030000002eb00140798000b0037001e0290001e
:10104000de029000848242001e039000a4e520008e
:101050000402430014427800844a78001e02900083
:101060000402e80014079800c47280009e029000f9
:10107000848f5200f1ff3400c4728000de029000c1
:10108000848242000042eb00844a78000002eb00b8
:10109000c47288001e027800040078000080fa0004
:1010a000000006000400fa00100798001e009000df
:1010b000cb2f070000027800e00f520099003200a9
:1010c0008e0078001e0090009f2e0700000278001e
:1010d000e00f5200930032001e4278000482fb00b1
:1010e0006123b90034ff2f00f5ff2f0006024200f4
:1010f00087824a007605200007002000860f5200f4
:10110000878f5a0081003e00046001007c00370098
:101110007e0037007d0037007c0037007b00370001
:101120007a00370079003700780037007700370001
:101130007600370075003700740037007300370001
:101140007200370071003700700037006f00370001
:101150006e0037006d0037006c0037006b00370001
:101160006a00370069003700680037006700370001
:101170006600370065003700640037006300370001
:101180006200370061003700600037005f00370001
:101190005e0037005d00370034003700360037004e
:1011a000380037003a0037003c0037003e00370077
:1011b0004000370042003700440037004600370047
:1011c0005200370051003700500037004f00370001
:1011d0004e0037004a0037004c0037004b00370004
:1011e0004a003700490037003e003700470037000b
:1011f0004600370045003700440037004300370001
:101200004200370041003700400037003f00370000
:101210003e0037003d0037003c0037003b00370000
:101220003a00370039003700380037003700370000
:101230003600370035003700340037003300370000
:101240003200370031003700300037002f00370000
:101250002e0037002d0037002c0037002b00370000
:101260002a003700290037001e0037001e009000ba
:101270000e0107002b0037001e009000160107002a
:10128000280037001e0090001d01070025003700d0
:101290001e0090004a010700220037001e00900047
:1012a0009f0107001f0037001e009000cb010700c0
:1012b0001c0037001e009000f701070019003700de
:1012c0001e00900010020700160037001e0090005c
:1012d0002f020700130037001e00900032020700a3
:1012e000100037001e009000462707003000200045
:1012f000fa2e070020002000f82e07000900370012
:101300001e009000cc00070006003700410e2d00a3
:101310001e009000542e0700610f2d001e0090004b
:10132000512e07000080fa00000006000200fa00bb
:10133000000f7800a4102d00841f780034112d00b8
:10134000841f780044002000841f780014002000cf
:10135000841f7800f4112d00841f780060d52000d0
:10136000d7080700ea87570061d520001e007800e3
:101370003d2e070021152d001e0078003a2e070093
:101380000080fa00000006000200fa00000f78005a
:10139000346a8000841f780064162d00841f780052
:1013a00060d52000c6080700e487570061d52000fb
:1013b0001e0078002c2e0700446a8000556a8000c9
:1013c000849fbe0094172d00841f780060d52000f4
:1013d000bb080700e687570061d520001e00780093
:1013e000212e0700846a800004017800d1182d00a6
:1013f0001e007800372e0700946a8000841f780052
:10140000c4192d00841f780060d52000ac080700a7
:10141000e4875700946a8000610262000442780009
:10142000e04f52000a00320060d520009307070009
:10143000000278008402780064d520000482420013
:1014400082002000411b2d00040078007d0707006a
:10145000946a800062026200e00f52000a003200cb
:1014600060d520008507070000027800840278001c
:1014700064d520000482420082002000c11b2d00a0
:10148000040078006f070700946a8000640262001d
:10149000e00f52000a00320060d5200077070700f5
:1014a000000278008402780064d5200004824200a3
:1014b00082002000411c2d00040078006107070015
:1014c000946a800068026200e00f52000a00320055
:1014d00060d52000690707000002780084027800c8
:1014e00064d520000482420082002000c11c2d002f
:1014f0000400780053070700946a800070026200bd
:10150000e00f52000a00320060d520005b070700a0
:10151000000278008402780064d520000482420032
:1015200062002000411d2d000400780045070700df
:10153000956a80000402200004826200e00f5200dd
:101540000a00320060d520004c0707000002780036
:101550008402780064d520000482420062002000ea
:10156000a11d2d000400780036070700956a800051
:10157000f403200004826200e00f52000a003a00e7
:1015800060d520003d070700000278008402780043
:1015900064d520000482420062002000011e2d005c
:1015a000040078002707070060d5200033070700f4
:1015b000000278008402780064d520000482420092
:1015c00042002000611e2d00040078001d07070066
:1015d00061d520001e007800a32d0700a46a8000ba
:1015e000841f7800a41e2d00841f780060d5200081
:1015f00033080700e487570061d520001e007800fb
:10160000992d0700646a8000756a8000849fbe007f
:1016100014202d00841f780060d5200028080700c2
:10162000e687570061d520001e0078008e2d070048
:101630000080fa00000006000400fa00100798007d
:1016400051212d001e009000872d07000002eb00a5
:10165000040f7800100037001e0278008402420058
:10166000840c21000482420014027800e00f520032
:10167000080032001e02780084024200840c21001f
:101680000482420014027800840078001e0090005a
:10169000752d07001e0fe8001e027800eb0f5200a8
:1016a000edff36000080fa00000006000200fa009c
:1016b000000f78006037070060d42000763c0700f8
:1016c00014002000b47288000002eb0004007800cf
:1016d0000080fa00000006000200fa00000f780007
:1016e0001e00780011ff07001e00780026ff07008b
:1016f0000002eb00040078000080fa000000060001
:101700000400fa00100798000002eb00040f7800b4
:1017100081212d001e009000532d07000600370088
:1017200037fb0700146a8000e00f5200020032000d
:101730000002eb001f00370061d520001e00900062
:1017400003fe070000027800e00f5200f4ff3200b1
:1017500060d520005c06070000027800040f7800c6
:101760001e027800e00f5200040032000402200044
:101770009e027800848f52000b0036009e1f780076
:1017800094222d00841f780060d52000cc0707002c
:10179000e487570061d520001e009000322d07001d
:1017a0000082eb00030037001e027800346a8800d4
:1017b0000002eb00040078000080fa000000060040
:1017c0000600fa002007980011252d002e00900039
:1017d000252d07000600370009fb0700146a80006a
:1017e000e00f5200020032000002eb004900370017
:1017f00061d520002e009000d5fd07000002780082
:10180000e00f5200f4ff320060d520004d060700c3
:101810000002be00048fbe001e02be00066029004a
:1018200007002000860f5200878f5a002c003200dc
:101830000660290007002000860f5200878f5a009b
:101840000b003e000658220007002000860f5200c1
:10185000878f5a002400320006b0240007002000c1
:10186000860f5200878f5a00210032000a0037008d
:1018700006102e0007002000860f5200878f5a00a6
:101880001d00320006202c0017002000860f520099
:10189000878f5a001a0032001e02be00849fbe00cd
:1018a00034262d00841f780060d5200084070700af
:1018b000e687570061d520002e009000ea2c070033
:1018c000c1272d002e009000e72c0700e1282d00f5
:1018d0002e009000e42c07000082eb000d00370082
:1018e000000000000700370000000000050037007e
:1018f0000000000003003700000000000100370076
:10190000000000001e02be00446a8800556a88007c
:101910000002eb00040078000080fa0000000600de
:101920000400fa00100798000002eb00040f780092
:10193000112b2d001e009000cb2c07000600370055
:10194000affa0700146a8000e00f52000200320074
:101950000002eb001e00370061d520001e00900041
:101960007bfd070000027800e00f5200f4ff320018
:1019700060d52000d405070000027800040f78002d
:101980001e027800e00f52000e0032001e027800a6
:10199000e10f52000b0032009e1f7800942d2d00a5
:1019a000841f780060d5200045070700e4875700b2
:1019b00061d520001e009000ab2c07000082eb00d8
:1019c000030037001e027800846a88000002eb00e2
:1019d000040078000080fa00000006000400fa000d
:1019e000100798000002eb00040f780011302d0062
:1019f0001e0090009c2c07000600370080fa0700ac
:101a0000146a8000e00f5200020032000002eb0076
:101a10001e00370061d520001e0090004cfd07001d
:101a200000027800e00f5200f4ff320002012000b3
:101a30008000eb0060d520009d0607000002be007c
:101a4000040f780004fc2f001e026200e00f520019
:101a50000b0032009e1f780074362d00841f780022
:101a600060d5200016070700e487570061d52000e5
:101a70001e0090007c2c07000082eb000300370062
:101a80001e027800946a88000002eb0004007800cf
:101a90000080fa00000006000200fa00000f780043
:101aa000f1372d001e0078006f2c0700060037006c
:101ab00053fa0700146a8000e00f5200020032005f
:101ac0000002eb000d00370061d520001e007800f9
:101ad0001ffd070000027800e00f5200f4ff320003
:101ae00060d520007805070000027800050020007e
:101af000646a8800756a88000002eb0004007800c0
:101b00000080fa00000006000400fa0010079800a8
:101b10000002eb00040f7800b1392d001e00900088
:101b2000512c07000600370035fa0700146a8000c0
:101b3000e00f5200020032000002eb0011003700fb
:101b400061d520001e00900001fd07000002780012
:101b5000e00f5200f4ff3200020120008000eb0091
:101b600060d52000520607000002be00040f780076
:101b70009e027800f403200004826200a46a8800b8
:101b80000002eb00040078000080fa00000006006c
:101b90000200fa00000f78000082eb0004007800d9
:101ba0000080fa00000006000200fa00000f780032
:101bb0000082eb00040078000080fa0000000600bc
:020000040000fa
:101bc0000000fa000080fa00000006000000fa00a1
:101bd0000080fa00000006000400fa00000f780000
:101be00011079800be0007009560a8001e02900033
:101bf000e00f5200030032009580a8008580a80005
:101c0000010037009580a900c20007000080fa009b
:101c1000000006000c00fa002047980022079800f8
:101c200033079800014f98005407980014002000d3
:101c3000040f78002062a8002e029000be029000df
:101c40000660290007002000860f5200878f5a0087
:101c5000210032000660290007002000860f520094
:101c6000878f5a000b003e00065822000700200014
:101c7000860f5200878f5a001100320006b02400f0
:101c800007002000860f5200878f5a000f00320095
:101c90001a00370006102e0007002000860f5200a1
:101ca000878f5a000f00320006202c0017002000fa
:101cb000860f5200878f5a000d0032000f00370048
:101cc000f402200044118800100037007401200045
:101cd000441188000d003700b40020004411880032
:101ce0000a00370074002000441188000700370004
:101cf00034002000441188000400370074012000e3
:101d0000441188000002eb00040f780021e2a800d3
:101d100020a2a9002022a9002042a9002002a90097
:101d2000044020001411880023e2a90023a2a80087
:101d30008560a9008580a9004405800004c0a10039
:101d400004d0a00004e0a0004405880054058000f1
:101d50000400a1000410a0000420a1005405880084
:101d60009560a8009580a9001e0278000400780004
:101d70000080fa00000006000200fa00004f780020
:101d80001e02fb00241188001400200004007800cb
:101d90000080fa00000006000200fa00000f780040
:101da000d4878000044278009e027800844a78003c
:101db00014002000040078000080fa0000000600f3
:101dc0003600f800809fbe00829fbe00849fbe0048
:101dd000869fbe000000fa008580a900a4838000d1
:101de000040001000080fa004f03be004f02be0055
:101df0004f01be004f00be003600f9000040060053
:101e00003600f800809fbe00829fbe00849fbe0007
:101e1000869fbe000400fa000002eb001407980041
:101e20000002eb00040f78008560a9001411800007
:101e300062026200e00f52001d0032002222a9005f
:101e40000200370034118000d4878800141180000c
:101e500061026200e00f5200faff3a0019003700f9
:101e60001411800068026200e00f5200020032008c
:101e7000140020001407980014118000640262000e
:101e8000e00f52000200320014002000040f78001e
:101e900034118000d48788001e027800e00f5200c1
:101ea00004003a0094838000040001000100370020
:101eb000000000001411800061026200e00f520077
:101ec000e7ff3a000080fa004f03be004f02be0059
:101ed0004f01be004f00be003600f9000040060072
:101ee0000000fa00840f210014427800e04f5200f5
:101ef00001003a00ff3ffc00840f210014427800eb
:101f00000442e80004007800f8f0b7000080fa000e
:101f1000000006000000fa00840f2100144278003f
:101f20000442e9000002fd00f8f0b7000002fd00e5
:101f3000840f210014427800e04f520001003a0063
:0c1f40000000fc000080fa000000060019
:020000040000fa
:101f4c000000fa004382a9004362a9004342a800a2
:101f5c004322a9004302a80042e2a90042c2a90000
:101f6c0042a2a800141280000420a0000430a0009b
:101f7c000440a00014128800141280000400a10078
:101f8c000410a0001412880045e2a90045c2a90063
:101f9c0045a2a9004422a9004402a90040c2a900fc
:101fac0041e2a8000080fa00000006000200fa00de
:101fbc00000f780000000000041280006202620032
:101fcc00e00f5200fcff3a001e0278004412880019
:101fdc00000000000412800061026200e00f520059
:101fec00fcff320044128000040078000080fa00ec
:041ffc0000000600db
:020000040000fa
:1020000000000000000000000000000000000000d0
:1020100000000000000000000000000000000000c0
:1020200000000000000000000000000000000000b0
:1020300000000000000000000000000000000000a0
:020000040000fa
:102800004f4722000e7f24000e01880000000000c8
:1028100000012000200288000c000700c0032600f1
:102820000100200011000700000020000000e0006f
:102830000200320000000200000000004802020016
:10284000000000000040da000000fe004440a90043
:1028500000e720000000e00003003200000020003c
:10286000a00188004440a8000000060091018800f3
:10287000800078000000eb0015003700e280400087
:1028800032a0b4009101ba00e280400032a0b4004e
:102890009102ba00e280400032a0b4000002eb00d6
:1028a000472bde00f507b200602ce10004003a007f
:1028b0000059eb008301e900fdff3e0004003700f2
:1028c0006128e100010032000082eb0004000700f3
:1028d0001101ba000200e000e8ff3a000000060023
:1028e0003159ba008301e9000c0032002159ba00c5
:1028f0008301e900080032000400e00003003a0010
:10290000e280400032a0b400f5ff370011d9ba00d0
:102910008301e900faff3a008100e800e18040000d
:1029200032a0b4000000060084760400000000001d
:102930009a760400000000000e77040000000000fa
:10294000ac76040000000000847704000000000062
:102950000278040000000000647804000000000019
:1029600052690400000000006a69040000000000d1
:10297000da690400000000007c6904000000000027
:102980003c6a0400000000003c6b040000000000f2
:10299000186c0400000000009a8a04000000000087
:1029a000da87040000000000006e04000000000050
:1029b000546d040000000000f46c040000000000ee
:1029c000d06e040000000000c67f0400000000007c
:1029d000ac800400000000004681040000000000fc
:1029e000f686040000000000da5b0400000000002e
:1029f000045c0400000000002e5c040000000000e5
:102a0000585c040000000000825c0400000000002c
:102a1000ac5c0400000000003a5e0400000000000e
:102a2000005e040000000000c25e04000000000020
:102a3000ea5e0400000000006c5e0400000000007c
:102a4000125f040000000000a05f0400000000000e
:102a5000e25f0400000000007a5f04000000000054
:102a6000b45b0400000000005258040000000000a5
:102a7000d05b0400000000001260040000000000b1
:102a80000040da000000fe001004b100070035002d
:102a90009001b100040034007000b1000300350063
:102aa0009001b10001003c0010000500000005008d
:102ab0006900e100040035006d00e100030034000e
:102ac0000002b10001003200000005001000050006
:102ad000800078001106b100030035009101b100bb
:102ae00001003c000050a1000000060003f0a2001d
:102af000889fbe008a9fbe008c1f7800d20007000e
:102b0000d90033006450e1004f0032006420e1003e
:102b10005200320003826c0007003b000905d00020
:102b20000306d000820f54000c065d00020039003d
:102b30000200320089017800030678008582550082
:102b400004003d000003fd008103fd008502ea0052
:102b50008b854200840f720002003b006000100071
:102b6000e08018006011b8000005eb007a28e10051
:102b70000a00390006007800c75ddd00f707b200e3
:102b8000878075002d003700828171000a0178006e
:102b9000610560008180d1000080d3008502e900da
:102ba000f9ff3b00060440008784480002003b0018
:102bb00060041400e0841c000988a30007003200b0
:102bc0008a81710082817100610164008904d100f1
:102bd0000884d3008b05e800170037000978a300ac
:102be00013003a000b00e000130034008b05e900ed
:102bf0000804440089844c000a4474000978a30046
:102c00000d003a000b00e000070034008b05e900de
:102c10000804440089844c0001003a000b002000a5
:102c20000978a300f7ff32000001eb000200370033
:102c3000828171000a0178005d0007000cf0a70096
:102c400001f0a000910037006420e10002003a008a
:102c5000838f6c00910033000801be000200be00ab
:102c60008a003700889fbe008a9fbe008c1f7800b4
:102c7000750007007c00330003866c006450e1009f
:102c80002e0032006420e100330032006150e10088
:102c90002f0032006120e1003100320085855500af
:102ca000eb07b000090020000804200005003700f1
:102cb0000804440089844c000a00310006034300e4
:102cc00087834b000001530081815b00f8ff3300d4
:102cd0000203be000800a0000804440089844c00e0
:102ce000f6ff3900c639dd008301730001003200b0
:102cf000130020008904d1000884d3000998a300a0
:102d0000050032000800a7000300a0008904d100dc
:102d10000884d3008b05e8008904d1000884d3001f
:102d20000001eb000281d2002100070001f0a100a8
:102d30000cf0a70001f0a000540037006420e1006f
:102d4000560032000801be000200be00f7ff370047
:102d50006120e100510032006000b800f3ff37004d
:102d60000000200001f82700f0ff3700839f680073
:102d70000100e00002003d0060001000e08018004b
:102d80000300e00002003d0060011100e081190035
:102d9000790007004f00e00002003b0060001000d7
:102da000e0801800000006006011b80082003700c3
:102db00081002000618055000b003d000b002000c9
:102dc00061fe2f000100e1001d00340082817100ce
:102dd000610164008904d1000884d3000000e80088
:102de000faff3a00710020006100640003007000e7
:102df000020060000900320061044400e0844c00dd
:102e00000988a500050032008b05e8006808e1008c
:102e100002003a008904d1000884d300f20f200098
:102e20000258e10005003d00c75ddd00f907b20072
:102e30008980750008007800000006000bf8270064
:102e40008b007800000005000004be008900070028
:102e50000003be000405be000200be00850007009e
:102e6000844f7500000006000200be006450e100bf
:102e7000050036006420e100020036000968a30066
:102e800001003a000800be000160a0004f06780073
:102e90004f05be004f04be0000000600f0ff2f00eb
:102ea000f1ff2700f9ff3700889fbe008a9fbe0010
:102eb0008c1f7800e4ff0700ebff330003866c00f3
:102ec0006450e100240032006420e1002700320059
:102ed0006150e100220032006120e1002100320057
:102ee0008b854200eb07b1000134b800003ab8000e
:102ef0000804420089844a00013ab8000030b80052
:102f00008880400009014a000400330000004000ae
:102f100081804800020149008b05e900c909dd00f4
:102f2000830170000100320013002000c814de008d
:102f30004814dd004709de001200b200c808de00b8
:102f4000088470009aff070001f0a1000cf0a700b0
:102f500001f0a000cdff37006120e100cfff32007b
:102f60000801be000200be00f7ff37006150e1001b
:102f7000fcff3a00c9ff37006022b80006022000bb
:102f80000000d0008180d2000482d2008582d2006d
:102f90000000a0000202520083825a0003003100a8
:102fa0000202420083824a000000a1000603e900f9
:102fb000f3ff3a0000000600889fbe008a9fbe0013
:102fc0000082700004027100048271002600320049
:102fd0000004be000200be006011b8006b092000b2
:102fe000950220000182cf000a0039000541b1009e
:102ff0000082cf00070039000541b1000982cf00ef
:10300000040039000541b1000882cf0001003900f9
:103010000541b10005425200120032000a003b0097
:1030200082817100610164008100d1000080d300c1
:103030008984d3000884d3008b05e8000442e800ab
:10304000f7ff3a00070037000804440089844c0069
:1030500000004800818048008b05e9000442e90037
:10306000f9ff3a0052ff07004f05be004f04be00b3
:1030700000000600c70ade00f107b200f50fb2003b
:1030800008003200e1cf4200020032000170a000cf
:1030900024000500810f70000100320004080500c3
:1030a00044000500810f700002003a001400050082
:1030b0008502e9000000400081c04800fcff3b00a1
:1030c0000170a0002400050006c2b30000027800d1
:1030d00004007800b042780086cf5200fbff320037
:1030e000e9cf5200f9ff3200d6c2b30086cf5200ba
:1030f00003003a000002780016c0b3000500370054
:103100000043eb00b7c2b30087cf520001003a0082
:10311000000278000000eb00020037006a00b900ee
:1031200000804200b402fb000503b100e98f5200a9
:10313000faff3600e04f5300010032000000ea00c1
:1031400000000600889fbe008a9fbe0004c2b30034
:103150003044780080047800844f5400fcff320033
:10316000e94f5400faff3200d4c2b300844f540038
:1031700003003a00394478001ac0b3000500370054
:103180000045eb00b4c2b300844f540001003a0084
:10319000394478006000b8000bcdb3000900370057
:1031a000a2002000030020007c1607000b42440010
:1031b0000482fb00050020000400400085804800d8
:1031c000394478000882fb000403b100e90f520083
:1031d000f3ff3600e04f550002003200600010009f
:1031e000e08018004f05be004f04be00000006003e
:1031f000e4392100e08f510002003a00b33a210087
:1032000003027800831f7800841f7800801f7800f5
:10321000811f7800821f7800c43a2100841f780043
:103220008044210001000700080107000000fa00a7
:1032300068815700cfb897008a0807000080fa001d
:10324000000006000002780002003700315a7800c2
:103250000201e900e00f5100fcff3a000000060007
:103260000002780002003700015a78000201e900ec
:10327000e00f5100fcff3a00000006000002780059
:103280008042eb00b4cf1200fdff3a000080ea005c
:103290000000420000000600ea874700889fbe0049
:1032a0008a9fbe008c9fbe008e1f780001067800aa
:1032b000820478000002eb0044a38800840f5600cb
:1032c00001003200000e780000057800ba46780050
:1032d0000a0478000d00fb00f5fd0700e00f500028
:1032e000faff3a008d427800d4c2b30084cf520076
:1032f00003003a00b84278001ec0b3000500370052
:1033000000477800b4c2b30084cf520001003a00f5
:10331000b842780004c3b30084cf520012003a00d0
:10332000b8427800e08f540002003200f08f540061
:1033300010003a0084c7b30084cf5200030032006b
:1033400084c5b30084cf520003003a00b84278002d
:103350000901200007003700e08f540005003a0003
:103360008900200003003700e08f540001003a007c
:10337000a90020008046eb006055b800614bb90001
:10338000d6b79f00e7b79f000503fb000600780053
:1033900085bf9f00f6b79f00bbfd07008fba97005f
:1033a0007fb39700e00f5000050032000600780060
:1033b000c7fd070097ccb300074240000500370067
:1033c0000603b100e90f530020003e0006cdb30014
:1033d00006c242008402fb00898f52001a003d00a1
:1033e0000402fb00cfa2de005fb19700efb19700af
:1033f0000a00be00f4b79f0085bf9f00e7150700d5
:103400007fb297008fba970004034000858348007d
:103410000800e800860f5500878f5d000500360024
:103420002402200044a388000004780010c0b300e8
:103430000600370098427800000478000605be00b8
:103440001dc0b300d0ff37000040eb00e00f560076
:1034500002003200e0cf560004003a009c027800df
:1034600004c3b300954f120001003a00080ee900b2
:10347000e14f500005003200e04f570005003200d8
:1034800060051500e0851d00020037000085eb0097
:103490008085eb000a00be004f0778004f06be0093
:1034a0004f05be004f04be00af00b1000000060093
:1034b0000200fa00889fbe008a9fbe008c1f780021
:1034c00080057800010578000002eb0044a3880025
:1034d0000b0678008c047800090678003c447800dc
:1034e0000800fb00a2bf9f0071fd07002fb99700e5
:1034f000e00f5000f7ff3a00d4c2b300844f5400ed
:103500000300320004c2e900844f540002003a0074
:103510008904e80001003700044478008a0078003c
:10352000090078005cff07009a8f540001003a0000
:103530000b0d78009a8f550003003a00e00f500001
:10354000e08f58000f003a00b4c2b300844f54001b
:1035500004003a00e00f5000e08f580015003d00d5
:1035600008003700d4c2b300844f540011003a0061
:103570000400200005002800840f5000858f5800ab
:103580000a0036002402200044a38800f0ff2f0028
:10359000f1ff27006b424200844f540005003a00bf
:1035a0000000200001002800020037006000100029
:1035b000e08018004f0678004f05be004f04be00a3
:1035c0000080fa00000006000002e9000080eb0025
:1035d000e50f520004003e00040242006545210050
:1035e00065007a0081327a0000000600881f7800aa
:1035f0000002e900e50f52000e003e000402420006
:103600006545210065027a00e00f520002003a0091
:103610001000200026000700e10f420007003200e2
:103620000004eb00e10f520005003200040001002d
:10363000030037000084eb00010037000404780029
:10364000080078004f0478000000060010002000f9
:10365000e6ff070010002000150007000c00fa002c
:1036600000027800820278000000eb00e18f500039
:103670000d0036008100e900f1bf9f00b0bf9f0040
:10368000a4bf9f00c4bf9f00240c2000d4bf9f0094
:1036900003017800850078006c80570071070700ef
:1036a0002fba9700004aeb000080fa0000000600e5
:1036b0000004780096110700080078004f120700f8
:1036c0000c00fa00889fbe0000047800f4ff270079
:1036d000d4bf9f008004eb0099bf9f0088bf9f006c
:1036e000a8bf9f00240c2000b4bf9f007881570022
:1036f000cfb0970070805700b30007000fba970053
:10370000094a78000fba9700080052004f04be0023
:103710000080fa0000000600889fbe008a9fbe005d
:103720000084fb00d4c6b300844f50002200360052
:103730004b062000110009000b84d8008105780099
:10374000720040004300dd00e91a210000804400bf
:103750006022b8000600200007fe23005001be00d2
:103760004000be006b140700aa002000809fbe002e
:10377000110009008a85d800800578004f00be003e
:10378000e9854500c35ddd008b8544003b02be003a
:103790002b03be005f140700809fbe0011000900cc
:1037a0000a84d800010478004f00be004344dd00c5
:1037b0008884440013003700ea4f5000140036009c
:1037c000aa002000110009000a84d8000004780033
:1037d00001057800690444004344dd00e91a210032
:1037e000088444006022b8000600200007fe230081
:1037f0003800be002801be00461407004355dd0016
:103800008a8444003902be002903be000800370044
:103810004344dd00e41a2100080442006022b8009d
:103820000600200007fe23003800be002801be006d
:10383000381407004f05be004f04be00000006000c
:10384000889fbe008a9fbe00d4c6b300e04f5000e0
:1038500029003d000040ea000004fb00844f5000b6
:103860001000340044062000809fbe0011000900b3
:103870000404d800010278004f00be00a900200017
:10388000809fbe00110009000902d80000027800e4
:103890004f00be00690242004322dd00ea1a210007
:1038a00023003700ea4f500010003400a40020002d
:1038b000110009000404d8000104780069004000e8
:1038c0004300dd00e41a2100000042004344dd0013
:1038d000080242005403be004402be005001be0074
:1038e0004000be000b140700340037004344dd00e5
:1038f000e41a21002e0037000004fb00844f500022
:103900001d00340044062000110009000404d80002
:1039100001027800a9002000110009000902d80066
:1039200000027800690242004322dd00ea0f210014
:10393000040245005403be004402be008b0920006f
:103940008a8545003b00be002b01be00f113070035
:10395000809fbe00110009000904d800010478000e
:103960004f00be004344dd00080545003a02be009a
:103970002a03be00dbff3700ea4f50000a00340084
:10398000a4002000811f7800110009000404d80061
:1039900001047800cf007800690040004300dd009a
:1039a000e40f2100c8ff37004344dd00e40f21008d
:1039b000080442003800be002801be004f05be00ca
:1039c0004f04be0000000600ef05b000889fbe0057
:1039d0008a9fbe008c9fbe008e1f78000006780074
:1039e000e19f9f0082af9f000007eb00e5053700d5
:1039f000ef9897008100e800e19f9f0054c2b30058
:103a0000844f500006003a00010378008006eb0066
:103a100007c3b30000c2b300b1c2b3000e00370049
:103a20003c0290000404b200040032001c02780042
:103a3000004a7800040ee800050037000000fb0093
:103a40008c0078006e100700e10f4000cd053200b9
:103a50000e07e800cb05370006027800b642780072
:103a6000d2c2b30082cf52000900320005003c00f0
:103a700080cf52000800320081cf52000c003a0083
:103a80000700370087cf520009003a0006003700d0
:103a90000d30a000f0ff37000d00a000eeff370052
:103aa0000d10a000ecff37000d20a000eaff37004a
:103ab00062836600010032000d00a1006883660089
:103ac000010032000d20a1000503fb000603b10038
:103ad000e90f53000d003e0084027800070020002b
:103ae0006a3bb9003502fb000403b10086034200c3
:103af000050278001503fb000603b100e90f53002f
:103b0000f7ff360097b79f000a0037000003eb006d
:103b100096b79f00a6c2b30086cf520005003a00b8
:103b20008fab97004700780087af9f0090b79f004a
:103b30000402e800e5c2b30094cf120017003a0077
:103b40000de0a000e4c25200d4cf12000300320006
:103b50008402780007002000090037000fa99700b1
:103b6000c201780082af9f00d3af9f000402e8003b
:103b7000c6c6b3000d0037006a38b90080034300a1
:103b8000050278003503fb000603b100e90f53007e
:103b9000f9ff3600d7af9f00f5ff37000dc0a0003a
:103ba0008002eb00d5af9f00f1ff3700840378005f
:103bb000b74278000702780086cf52002d0032000d
:103bc000e79f9f00c4c6b30084cf520014003c009e
:103bd0006842520084cf52002400320009003c00a9
:103be0006c42520084cf52002e0032006b424200e1
:103bf00084cf520099003200e0cf520066053200b7
:103c0000b600370064c6b30084cf52001f003200f4
:103c10006342420084cf5200b0003a0013003700e4
:103c200034c7b30084cf52002200320007003c00aa
:103c30006442520084cf5200170032000442e80070
:103c400084cf5200a5003a001600370054c7b300d5
:103c500084cf5200a60032006342420084cf52005b
:103c60009e003a00e5579f0010003700e5579f007f
:103c7000a1003700f083660005012000010032003a
:103c80000500280085867600c8ff3700e5579f00ad
:103c90000da0a00098003700e5579f000d60a00020
:103ca00095003700e5579f000d50a0000d70a00053
:103cb00091003700e5579f000fab97004602780050
:103cc00086af9f0004047800e00f520001003a0024
:103cd000e83f2100880278000002eb000100370075
:103ce0000402e80065437a00e04f5300fcff3a000d
:103cf00084047800dfab9700e08f530003003200ac
:103d0000898f530001003100870478000002eb0026
:103d10001fb09700890f50000100360009025000c3
:103d2000e8866600ddaf9f008d007800e08f5000d0
:103d30002d003a008406780004c2b300100037005a
:103d4000bc0290000504b200040032009c0278001e
:103d5000844a7800050ee800070037008c007800e0
:103d60000002200084bf9f00a50f07000fba970034
:103d7000e10f4000010032000e07e8008d06e90067
:103d8000e08f5600eeff3a000082eb00160037008d
:103d9000bc0290000504b200090032009c037800c8
:103da0008802780035437800864b7800070ee800db
:103db00005047800e04f53000a003a000a0037007b
:103dc000880278003500fb00050478008c0078003c
:103dd00084bf9f008a0f07000fba9700e10f4000d1
:103de000010032000e07e800890278008504e9002e
:103df000e08f5200e6ff3a005fa99700e00f510004
:103e0000e00432008406780004c2b30010003700da
:103e1000bc0290000504b200040032009c0278004d
:103e2000844a7800050ee800070037008c0078000f
:103e30000002200084bf9f00710f07000fba970097
:103e4000e10f4000010032000e07e8008d06e90096
:103e5000e08f5600eeff3a00ca0437008fa99700a2
:103e60004302780083af9f0004007800cf80de001b
:103e7000010178008201780090af9f00a1af9f0000
:103e8000b2af9f00c3af9f004800de00480add00cc
:103e900000007200e0579f00f082660009003200c7
:103ea000e04f500007003200e14f400005003200b3
:103eb000f0579f00afd29700855f9f002900200038
:103ec000030037002fd39700f6579f0019002000fa
:103ed00078f92f000f04440086ff3700e5579f0054
:103ee00068f92f000f0444001900200081ff3700fb
:103ef000e5579f000d0cb30004702000048266009b
:103f00006c023200040021000482660002003200cc
:103f100067002000d7af9f00708266000900320062
:103f20000faa97004401be004400be0084af9f006a
:103f300090af9f00a1af9f00b2af9f00c3af9f00a3
:103f40000a0037008faa97004500be0085af9f008a
:103f5000ca1107000002be000203be0094af9f001a
:103f6000a5af9f00b6af9f00c7af9f006022b8000b
:103f70006033b8001fa89700afa897003fa997002b
:103f8000cfa997000f110700e00f50000a003d0075
:103f90001fa89700afa897003fa99700cfa9970047
:103fa00003f0a20090af9f00a1af9f00b2af9f00af
:103fb000c3af9f003d00b3000002eb00d48f9f0011
:103fc0006022b8006033b8001fa89700afa8970020
:103fd0003fa99700cfa997005e110700e00f50009e
:103fe000390032001fa89700afa897003fa997009b
:103ff000cfa99700be120700a2f92f000f014100c0
:10400000411207005f8b97000603e9006333b90094
:10401000a500200000027800811f7800110009002f
:104020000503d8000002fd00cf007800d48f9f0068
:10403000e00f520002003d000402e900d48f9f000f
:104040005f8c97000840ea00fdfd07001faa97005b
:10405000afaa97003fab9700cfab97002d12070098
:104060000002be000203be0084a79f0095a79f0028
:10407000a6a79f00b7a79f006022b80006002000f7
:1040800007ff2300cf100700e00f500002003d00a3
:104090000804e9000b0037006022b8000600200089
:1040a000470224000fa097009fa097002fa1970020
:1040b000bfa19700c8100700e00f500002003500b4
:1040c0000804e800d88f9f00dfaa9700f88f5200fd
:1040d0000f003c00054078008ffd07000002be0085
:1040e0000203be001fa89700afa897003fa9970042
:1040f000cfa99700361007000002be000203be00e1
:1041000094af9f00a5af9f00b6af9f00c7af9f00c1
:104110005f8c9700e90f540015003c006022b80046
:104120006033b8001fa89700afa897003fa9970079
:10413000cfa9970007110700e00f500032003200ae
:104140001fa89700afa897003fa99700cfa9970095
:1041500069110700e00f5000e08f5800e00f590090
:10416000e08f590028003a00e10f54002600340087
:104170000400200005002e00b6e0220017012400f4
:104180000fa097009fa097002fa19700bfa19700b5
:104190008c100700e00f500002003d007304540033
:1041a0000100370072045400d88f9f002f589700e9
:1041b000a3fd07000002be000203be0084a79f000b
:1041c00095a79f00a6a79f00b7a79f001fa89700cd
:1041d000afa897003fa99700cfa9970083100700c9
:1041e000451107000205be000004be006000b800d3
:1041f0006011b80090af9f00a1af9f00b2af9f00c9
:10420000c3af9f00170037001fa89700afa8970003
:104210003fa99700cfa99700371107000205be00fc
:104220000004be008b1107000002be000203be00a6
:104230001fa89700afa897003fa99700cfa99700a4
:10424000291207000002be000203be0094af9f00c7
:10425000a5af9f00b6af9f00c7af9f000002eb0065
:10426000d48f9f006126210010c0b30008003700e2
:104270003102be003103be000440e10005c8e10088
:1042800006d0e10007d8e100030039000040e80053
:10429000f44f5000f6ff3a00e0579f005f8a970006
:1042a0009fb29700048252005fab97000602520053
:1042b0000000fb000000520090b79f00e00f530089
:1042c000020032000000e90090b79f0063826600a0
:1042d000030032009fb397008703e90097b79f0060
:1042e000648266004500320062826600e1826600f8
:1042f000e00f5200110032003c0290000404b200b2
:10430000080032001c037800b4c2b300e08f5200f2
:104310000100320004c2e800044b7800060ee800f9
:1043200015003700b0022000e08f5200010032007b
:104330000080e8008c0078000c003700e08f52000d
:10434000200032003c0290000404b200050032005c
:104350009c02780004c2b300844a7800050ee8008d
:10436000050037008c00780000022000240e0700b2
:10437000e10f4000130032000e07e8001100370083
:104380003c0290000404b200040032001c027800d9
:10439000054a7800040ee800070037008c0078001a
:1043a00000032000f5b79f00150e0700ffb297002d
:1043b000e10f4000010032000e07e8008904e90027
:1043c0000600370005c3b300c8a79f00d9a79f0008
:1043d000eaa79f00fba79f009fb49700e08f5400bf
:1043e000e7ff3c0099b79f004fa49700dfa4970018
:1043f0006fa59700ffa597006f00370068826600e1
:104400001f003a00110037003c0290000404b20083
:10441000040032001c027800054a7800040ee8000f
:10442000070037008c00780000022000f5b79f00dd
:10443000f30d0700ffb29700e10f400001003200ca
:104440000e07e8008904e9000600370005c2b30042
:10445000c8a79f00d9a79f00eaa79f00fba79f00be
:104460009fb49700e08f5400e7ff3c0099b79f008e
:104470004fa49700dfa497006fa59700ffa59700b2
:1044800062826600e1826600e00f52001100320095
:104490003c0290000404b200080032001c037800c3
:1044a000b4c2b300e08f52000100320004c2e80041
:1044b000044b7800060ee8003e003700b0022000f2
:1044c000e08f5200010032000080e8008c0078008c
:1044d00035003700e08f5200370032003c02900078
:1044e0000404b200050032009c02780004c2b3004c
:1044f000844a7800050ee8002e0037008c00780012
:1045000000022000280037003c0290000404b200a2
:104510008502fb00e00f5200130032009c0078007f
:10452000c1a79f00c32add00e225210085024100ca
:104530005503be004502be000800be000a01be00d1
:1045400047120700a4002000050020006033b800d7
:104550004a12070005c3b3004fa29700054a400066
:10456000040ee80013003700c32add00e625210011
:10457000850243005503be004502be000800be0090
:104580000a01be0036120700a4002000050020002a
:104590006033b80039120700040320000002420013
:1045a0008c00780004007800950d0700e10f4000b2
:1045b000010032000e07e8006f5297008442e900c4
:1045c000e5579f00e04f5200cfff3a00110037003f
:1045d0003c0290000404b200040032001c02780087
:1045e000084a7800040ee800050037008c007800c7
:1045f00000032000820d0700e10f4000010032009f
:104600000e07e8005f8a97000402e900d48f9f003c
:104610000100370008c3b3005f8a9700e00f520023
:10462000ebff3c00dfab9700f28f53000300340038
:1046300024c1b300e4579f00020037002fd8970031
:10464000e0579f006f5297008402fb00dfa897009d
:1046500085825000c5a79f00e04f52000e00320037
:104660003c0290000404b200050032001c027800f5
:10467000e5c2b300054a7800040ee80005003700e3
:104680008c007800e00220005d0d0700e10f400083
:10469000010032000e07e8006f50970068fc070029
:1046a0000002be000203be001fa89700afa897003b
:1046b0003fa99700cfa99700961007000e1007009a
:1046c000360037003c0290000404b2008502fb0073
:1046d000e00f5200130032001c017800d2af9f009f
:1046e000c32add00e3252100858241005503be0079
:1046f0004502be000800be000a01be00d811070036
:10470000a4002000050020006033b800db11070082
:1047100005c3b3005faa9700054a4000040ee800f5
:1047200013003700c32add00e6252100850243007f
:104730005503be004502be000800be000a01be00cf
:10474000c7110700a4002000050020006033b80056
:10475000ca11070004032000000242008c00780008
:1047600004007800260d0700e10f40000100320030
:104770000e07e800ef5397000702fb004322dd001d
:10478000e0252100040240005403be004402be00a4
:104790000800be000a01be00b81107000205be00f5
:1047a0000004be006f5297008442e900e5579f0065
:1047b000e04f5200c3ff3a0011003700bc029000e6
:1047c0000504b200040032009c027800844a78009c
:1047d000050ee800070037008c0078000003200079
:1047e00084bf9f00060d07000fba9700e10f40003d
:1047f000010032000e07e8008904e90006003700d6
:1048000004c3b300d0af9f00e1af9f00f2af9f00a1
:1048100083b79f00cfa49700e08f5400e7ff3a00d2
:104820005fac9700efac97007fad97008fb5970016
:10483000e8866600530232009fb09700e08f500078
:10484000500234000dc2b3000802be000a03be00cd
:10485000810478003c0090000004b20004003200a3
:104860001c0078000d487800000ee8000d003700ad
:104870008c0078000002200084bf9f00f5b79f00e5
:10488000d6b79f00e7b79f00dd0c07000fba97006f
:10489000ffb297005fb39700efb39700e10f4000be
:1048a000010032000e07e8008904e900e9ff3a0040
:1048b000340237008d027800050cb2002a003a005d
:1048c000e08f560005003d000fa997004205be008d
:1048d0004204be0082af9f0016003700708266005f
:1048e0000e0032000fab97004602be0086af9f005d
:1048f000c4979f00d5979f00160290004fa2de003c
:10490000e4979f00f4979f004f949700df949700df
:104910006f959700ff959700060037000fa8970046
:104920004004780080af9f00cfc4de000905780006
:104930008a057800e00f5400e08f5c00e00f5d0016
:10494000e08f5d0023003d003d00b3006022b80011
:104950006033b8000804520089845a000a055b00dd
:104960008b855b001b003700e08f560005003d0083
:104970008fa897004105be004104be0081af9f0093
:1049800014003700f08266000c0032008faa9700f6
:104990004501be0085af9f0082979f0093979f00bf
:1049a000a4979f00b4979f000f9497009f9497003f
:1049b0002f959700bf959700060037008fab9700a3
:1049c0004704780087af9f00090020000a002000fc
:1049d0000b0020005fa89700e00f500009003a008c
:1049e00011002000d1af9f00e00f5400e08f5c0069
:1049f000e00f5d00e08f5d00020032000001eb007f
:104a0000d2af9f008d017800030cb20093af9f00de
:104a100004042000848f51002c00320003003c006d
:104a2000e08f5100080032003c00370004082000ed
:104a30009faa9700848f520010003200040c2000bf
:104a4000848f520035003a006526210014c0b3005f
:104a50003500be003501be000040e10001c8e100a4
:104a600002d0e10003d8e1002b0039000442e80045
:104a7000f44f5200f6ff3a002700370014c0b3008d
:104a800000012000010020006011b8000040e1009a
:104a900001c8e10002d0e10003d8e1001e003900a6
:104aa000460020000000d0008180d2000281d200a8
:104ab0008381d2000603e900faff3a000442e800cd
:104ac000f04f5200f1ff3a001300370014c0b3005a
:104ad00080002000010020006011b8000040e100cb
:104ae00001c8e10002d0e10003d8e1000a0039006a
:104af000370020000000d0008180d2000281d20067
:104b00008381d2008703e900faff3a000442e800fb
:104b1000f54f5200f1ff3a00e4579f006f509700a5
:104b20000002fb00dfa89700810f520002003d0049
:104b3000e1579f00040037005fa99700840f5100e0
:104b400001003d00d4af9f009fb19700e08f51005e
:104b50000400320063826600020032008301e90033
:104b600093b79f000400240004826600090032000d
:104b70001fb29700dfaa9700850f52000300340090
:104b80000502520094b79f00020037000003eb00bb
:104b900096b79f00ef5397000702fb000000eb0061
:104ba000c0a79f009fb09700848f50000200340080
:104bb00004825000c4a79f00648266004500320052
:104bc000e282660061826600e08f520011003200ce
:104bd000bc0290000504b200080032009c0278007c
:104be000b6c2b300e00f52000100320006c3e80075
:104bf000864a7800050ee80015003700b002200054
:104c0000e00f5200010032000080e8008c007800c4
:104c10000c003700e00f52000e0032003c02900002
:104c20000404b200050032001c02780005c2b30083
:104c3000054a7800040ee800050037008c00780073
:104c400000022000ee0b0700e10f400001003200df
:104c50000e07e8004fa19700e00f510063003200fb
:104c600004c3b30098b79f00a9b79f00bab79f00cd
:104c7000cbb79f00cfa49700bc0290000504b20000
:104c8000040032009c027800844a7800050ee80097
:104c9000070037008c0078000003200084bf9f00cd
:104ca000d70b07000fba9700e10f40000100320058
:104cb0000e07e8008904e900efff3a00c9a79f004a
:104cc0001fb49700afb497003fb59700cfb59700da
:104cd00046003700cfa09700e08f50001e00320042
:104ce000688266001c003a0004c2b30098b79f00b7
:104cf000a9b79f00bab79f00cbb79f00cfa497007a
:104d0000bc0290000504b200040032009c0278004e
:104d1000844a7800050ee800070037008c00780010
:104d20000002200084bf9f00b50b07000fba970058
:104d3000e10f4000010032000e07e8008904e9009d
:104d4000efff3a00c9a79f001fb49700afb49700c8
:104d50003fb59700cfb59700e2826600618266009a
:104d6000e08f520011003200bc0290000504b20036
:104d7000080032009c027800b6c2b300e00f520077
:104d80000100320006c3e800864a7800050ee800fc
:104d900015003700b0022000e00f52000100320081
:104da0000080e8008c0078000c003700e00f520013
:104db0000e0032003c0290000404b20005003200f4
:104dc0001c02780005c2b300054a7800040ee80012
:104dd000050037008c00780000022000880b0700d7
:104de000e10f4000010032000e07e800dfa8970045
:104df0000102e9004221dd00929f9f006323b90078
:104e000086017800839f9f004322dd00e525210075
:104e100085024200f59f9f0070826600f48f9f001c
:104e20008d0278000502b200e58f9f0098b79f00c1
:104e3000a9b79f00bab79f00cbb79f00aa00370061
:104e4000dfa897008100e900d1af9f001fa997005c
:104e500003042000830f51007a00320003003c005d
:104e6000e00f5100080032008500370004082000e0
:104e70009faa9700848f52005d003200040c20002e
:104e8000848f52007e003a00e08f56001f003d00e4
:104e90007f9b97003604be002605be000802be00b8
:104ea0000a03be001fb09700afb097003fb1970054
:104eb000cfb19700ea0f0700e0579f000000fb000a
:104ec000cf80de0001017800820178000802be0078
:104ed0000a03be004b1007001fb29700afb2970045
:104ee0003fb39700cfb397000002520081825a006f
:104ef00002035b0083835b0094b79f00a5b79f000c
:104f0000b6b79f00c7b79f0035003700ff8a9700ec
:104f1000e08f5200220032001fb29700afb297001c
:104f20007f9b97003604be002605be000801be0028
:104f30000400be0084bf9f00f5b79f000ef8070075
:104f4000e0579f000000fb00cf80de000801be009c
:104f5000120f07000fba9700ffb29700000152002e
:104f600081815a00a29f9f00b39f9f008001eb00a8
:104f7000c39f9f000002eb00d49f9f002f989700d3
:104f8000bf9897004f999700df99970090b79f00bf
:104f9000a1b79f00b2b79f00c3b79f0010003700b2
:104fa000ff989700110278001fb1970080027800e7
:104fb000811f7800110009000481d8008002fd00e3
:104fc000cf007800a4002000809fbe0011000900df
:104fd0008482d800010278004f00be00e4579f0091
:104fe000ef5197000343b000e3579f0024003700c0
:104ff000d43e2100ef8a9700e08f5200010032007a
:10500000c43d21001fb09700afb097003fb197009b
:10501000cfb197001f9b97000603e90005003300fe
:105020008301d1000281d3008180d3000080d300ae
:10503000f9ff37006f00600064407800e0579f0080
:105040000f0037001fb29700afb297003fb3970031
:10505000cfb397000f9897000000e90005003300d8
:105060008703d1000683d3008582d3000482d30056
:10507000f9ff3700674262000443b000e4579f0025
:105080003c0290000404b200070032009c02780049
:105090006f529700844a7800050ee800e04f5200f6
:1050a00007003a0007003700ef5097000100fb00af
:1050b0008c007800d20a0700e10f400001003200a6
:1050c0000e07e8001f99970064015100929f9f000e
:1050d0008f999700e3815100839f9f007f9a9700eb
:1050e00068025200f49f9f00dfaa9700e08f5200f1
:1050f00053ff3a001fb49700afb497003fb5970035
:10510000cfb59700e88666001e0032004fa39700d7
:10511000e00f53001b0034000dc2b3000802be00b4
:105120000a03be00cfa497003c0090000004b20028
:10513000040032001c0078000d487800000ee800e2
:105140000d0037008c0078000002200084bf9f0013
:10515000f5b79f00d6b79f00e7b79f00a80a0700e2
:105160000fba9700ffb297005fb39700efb39700b5
:10517000e10f4000010032000e07e8008904e90059
:10518000e9ff3a00ef9b970017407800e0579f0037
:10519000e04f500016fa3a000e0078004f077800f2
:1051a0004f06be004f05be004f04be00ef05b10024
:1051b00000000600889fbe008a9fbe000084fb009e
:1051c000d4c6b300844f5000220036004b062000a6
:1051d000110009000b84d80081057800720040009e
:1051e0004300dd00e91a2100008044006022b8007d
:1051f0000600200007fe23005001be004000be0054
:10520000c40d0700aa002000809fbe001100090005
:105210008a85d800800578004f00be00e9854500ea
:10522000c35ddd008b8544003b02be002b03be0046
:10523000b80d0700809fbe00110009000a84d80045
:10524000010478004f00be004344dd008884440020
:1052500013003700ea4f500014003600aa00200067
:10526000110009000a84d8000004780001057800c4
:10527000690444004344dd00e91a21000884440025
:105280006022b8000600200007fe23003800be00a0
:105290002801be009f0d07004355dd008a844400ad
:1052a0003902be002903be00080037004344dd0078
:1052b000e41a2100080442006022b8000600200021
:1052c00007fe23003800be002801be00910d070034
:1052d0004f05be004f04be0000000600889fbe00c0
:1052e0008a9fbe00d4c6b300e04f500029003d00a5
:1052f0000040ea000004fb00844f5000100034001e
:1053000044062000809fbe00110009000404d8005c
:10531000010278004f00be00a9002000809fbe005f
:10532000110009000902d800000278004f00be00f9
:10533000690242004322dd00ea1a210023003700ff
:10534000ea4f500010003400a400200011000900b2
:105350000404d80001047800690040004300dd0027
:10536000e41a2100000042004344dd00080242002c
:105370005403be004402be005001be004000be0007
:10538000640d0700340037004344dd00e41a2100b7
:105390002e0037000004fb00844f50001d00340035
:1053a00044062000110009000404d800010278001e
:1053b000a9002000110009000902d80000027800ad
:1053c000690242004322dd00ea0f21000402450089
:1053d0005403be004402be008b0920008a854500ac
:1053e0003b00be002b01be004a0d0700809fbe009f
:1053f000110009000904d800010478004f00be0024
:105400004344dd00080545003a02be002a03be0001
:10541000dbff3700ea4f50000a003400a4002000f0
:10542000811f7800110009000404d80001047800ed
:10543000cf007800690040004300dd00e40f210048
:10544000c8ff37004344dd00e40f21000804420098
:105450003800be002801be004f05be004f04be004c
:10546000000006000f07b000889fbe008a9fbe00a4
:105470008c9fbe008e1f780000067800c1979f00a9
:10548000d2af9f000007eb00d1093700cf90970003
:105490008100e800c1979f0054c2b300844f5000c0
:1054a00007003a00010278000003eb00d0c2b3000d
:1054b00001c3b30002c2b30033c2b3000e00370011
:1054c0003c0290000404b200040032001c02780088
:1054d000004a7800040ee800050037000000fb00d9
:1054e0008c007800c6090700e10f4000b8093200bf
:1054f0000e07e800b609370084037800b44278004c
:10550000b8c2b30088cf52000f00320005003c0043
:1055100082cf52000a00320083cf520010003a00be
:105520000b00370080cf52000300320081cf5200c1
:105530000b003a00080037000630a000eeff3700ed
:105540000600a000ecff37000610a000eaff3700bd
:1055500006b0a000e8ff37000620a000e6ff3700f5
:1055600062026300010032000600a10068026300cd
:10557000010032000620a1000502fb000403b10077
:10558000e90f52000d003e00870278000000200065
:105590006a00b9003502fb000403b10000004200bc
:1055a000850378001502fb000403b100e90f5200e7
:1055b000f7ff3600e0af9f000a0037000005eb0060
:1055c000eaaf9f00a4c2b30084cf520005003a00a6
:1055d000dfad97004b007800dbaf9f00e0af9f008e
:1055e0008703e800e4c2b300974f12001c003a00a2
:1055f00006e0a000c6b79f0064425200d74f1200d9
:105600000300320007037800050020000d0037007a
:105610005fa99700c2017800d2af9f00f3af9f004f
:105620008703e8000700780076c6b30007c7b30019
:10563000c1c6b3004fb297000e0037006a28b90008
:1056400080024200860378003602fb000403b100aa
:10565000e90f5200f9ff3600f5af9f00f1ff370068
:1056600006c0a000c6b79f000002eb00f4af9f0089
:10567000ecff3700b0427800c0979f0086cf520001
:105680003300320018003c00c4b79f0034c6b3009a
:1056900084cf5200d00032000e003c007c42520009
:1056a00084cf52004400320006003c00e0cf52009c
:1056b0004c09320004c2e90084cf5200e6003a00ef
:1056c0003500370084c5b30084cf5200e2003a00b1
:1056d0004700370054c6b30084cf52001f00320089
:1056e00028003c001f00370087cf52003f003200e7
:1056f0000a003c0081cf52001c003200c4b79f005a
:10570000f4c6b30084cf5200330032006642520028
:1057100084cf5200d0003a0012003700c4b79f0077
:1057200054c7b30084cf5200d2003200634242001b
:1057300084cf5200040032006542520084cf5200f0
:10574000c5003a0032003700c5479f002c003700e3
:10575000c4b79f00c6479f001b003700c5479f0086
:1057600011003700c5479f00c60037007001620076
:10577000050120000100320005002800050272002a
:10578000bcff3700c5479f00cfb4970009a0a00019
:10579000c9b79f00bb003700c5479f004fb59700b2
:1057a0000a50a000cab79f00cfb597000b80a00099
:1057b000cbb79f00b3003700c5479f004fb097009d
:1057c0000050a000c0b79f00cfb097000190a0008c
:1057d000c1b79f00ab003700c5479f004fb197008e
:1057e0000260a000c2b79f00a6003700c4b79f00a8
:1057f000c5479f00cfb197000350a000c3b79f00db
:105800004fb297000470a000c4b79f009d003700fe
:10581000c5479f00dfaa970045027800d5af9f00db
:1058200084b79f00e00f520002003a008742210037
:1058300087b79f000fb397008002eb00010037008d
:105840008502e80066c27a00e04f5200fcff3a0091
:1058500095b79f007fac9700e00f54000500320021
:105860009fb49700890f54000200310008057800aa
:105870009ab79f001fb297000004eb00efad9700ae
:10588000848f550001003600048455004fb0970006
:105890006805600009c2b3000f003200290037001c
:1058a0003c0290000404b200040032001c027800a4
:1058b000094a7800040ee800050037008c007800e3
:1058c00000022000ce080700e10f40000100320076
:1058d0000e07e8000804e900e00f5400f0ff3a006a
:1058e0000084eb0017003700bc0290000504b200f2
:1058f000090032009c037800880278003543780064
:10590000864b7800070ee80005047800e04f53004e
:105910000a003a0011003700880278003500fb00c9
:10592000050478008c00780084bf9f00b40807004d
:105930000fba9700e10f4000080032000e07e800a0
:1059400006003700880678000a0278000fb4970036
:105950009fb497002fb59700bfb5970089027800d4
:105960008504e900e08f5200dfff3a0088b79f000e
:1059700099b79f00aab79f00bbb79f000d0478009e
:105980000405780009c2b300e00f55000f003a008b
:105990008f0837003c0290000404b200040032007b
:1059a0001c027800094a7800040ee8000500370060
:1059b0008c0078000002200091080700e10f4000f1
:1059c000010032000e07e8000804e900e00f54006f
:1059d000f0ff3a007e083700dfa897004102780008
:1059e000d1af9f0004047800cfc4de000905780021
:1059f0008a0578000800be000a01be004800de00eb
:105a0000480add0000007200c0479f004fb39700b6
:105a10007002630009003200e04f500007003200be
:105a2000e14f400005003200d0479f00e8479f004b
:105a30002700200097b79f0003003700d8479f003a
:105a40001800200098b79f0059f82f00898447005c
:105a500089b79f007fff3700c5479f004af82f0096
:105a60000a8547008ab79f001b0020009bb79f0054
:105a700078ff3700c5479f004fb09700000cb30078
:105a8000c0b79f0004702000cfb097000482600070
:105a90009a053200040021000482600002003200f6
:105aa00062002000f2af9f00cfb1970070826100ca
:105ab000050032005faa97004405be004404be0002
:105ac000d4af9f0006003700dfaa97004500be0054
:105ad000d5af9f00e90a07000004be000205be0022
:105ae0006022b8006033b8000800be000a01be00a2
:105af000340a0700e00f500004003d000bf0a20044
:105b00004fb397003600b300c6b79f000002eb000a
:105b1000c4879f006022b8006033b8000800be0050
:105b20000a01be008b0a0700e00f5000340032006b
:105b30000800be000a01be00ed0b070082f82f002e
:105b40000f014100700b07004f8297000402e9002b
:105b50006323b900a4002000809fbe00110009004b
:105b60000403d800000278004f00be00c4879f00e5
:105b7000e00f520002003d000402e900c4879f00cc
:105b8000cf8697000d40ea00d4fd07000802be0052
:105b90000a03be005f0b07000002be000203be0046
:105ba000d49f9f00e59f9f00f69f9f0087a79f00bf
:105bb0006022b8000600200007ff2300010a07004a
:105bc000e00f500002003d000d02e9000b0037001d
:105bd0006022b80006002000470224005f9897006a
:105be000ef9897007f9997008fa19700fa09070017
:105bf000e00f5000020035000d02e800c4879f004e
:105c0000cf8697004fb297000410b20008003a0008
:105c10004fb297000420b20028033200e48f460000
:105c200003003500ffaa9700858f5600b1023500aa
:105c30007fab9700e00f5300050032004fb2970092
:105c40000420b200020032000603e900f6af9f0014
:105c5000ffab9700f28f53000300360024c1b3005e
:105c6000c4479f00020037006fd89700c0479f00cd
:105c70006022b8006033b8000800be000a01be0010
:105c8000340a0700e00f500063003200cf40970055
:105c900081e79f0001c0560090fd07000002be0092
:105ca0000203be000800be000a01be00cf090700c3
:105cb0000004be000205be00c00a0700100b07006a
:105cc0000002be000203be000800be000a01be00c2
:105cd000850b07006022b8000600200007fe2300a5
:105ce000bd090700e00f5000080035006022b80031
:105cf0000600200007fe23000800be000a01be00c7
:105d0000330907000004be000205be000800be0003
:105d10000a01be00a90a0700909f9f00a19f9f0053
:105d20008001eb00b39f9f000002eb00c49f9f0027
:105d30008fe297008502fb0095af9f000502e80007
:105d40004322dd00e62f2100040043003002be00a4
:105d50002003be0084b79f0095b79f00a6b79f00a1
:105d6000b7b79f001f989700af9897003f9997008b
:105d7000cf9997000400e1000588e1000690e1005a
:105d80000798e1000b0039000400200005002a00fc
:105d90009699290097fb23000800be000a01be0067
:105da000dc0a07000004be000205be000d02e80088
:105db000180037009fa89700430add00e22f21005a
:105dc000040241005403be004402be001f98970025
:105dd000af9897003f999700cf9997000400e10092
:105de0000588e1000690e1000798e1000a00310013
:105df0006022b80006002000470224000800be0010
:105e00000a01be00c30a07000004be000205be006e
:105e10000d02e900c4879f0004a02000cfb09700c6
:105e20008482600004202000848f52004c003a00dd
:105e30007fa99700f40f51000200340043012000b5
:105e4000f3af9f000800be000a01be005b0a070016
:105e5000d0979f00e1979f008002eb00f5979f008d
:105e60000003eb00869f9f00ffae97000800be0076
:105e70000a01be0080b79f0091b79f00a2b79f00a4
:105e8000b3b79f005f949700ef9497007f959700ba
:105e90008f9d9700090037008d06e900a4002000bf
:105ea000050020006033b8000800be000a01be00f3
:105eb000eb0b07000205be000004be00e00f54001b
:105ec000e08f5c00e00f5d00e08f5d000b003200b2
:105ed000a4002000050020006033b8000800be00c8
:105ee0000a01be00e50b0700e00f5000e08f5800ec
:105ef000e00f5900e08f5900e7ff3200fdaf9f002f
:105f0000d8979f00e9979f00fa979f008b9f9f006b
:105f10000fb497009fb497002fb59700bfb59700b7
:105f20004f4097000002fb008d027800848f5200e2
:105f30000b003d0005405000e8fc07000002be00d9
:105f40000203be000800be000a01be0027090700c8
:105f50000004be000205be006fdb9700c6479f002d
:105f6000efab9700658253007fa8970000025200b4
:105f7000e4af9f00e00f500004003a0004802000ce
:105f8000cfb0970004826000030032006fa9970031
:105f90000201e900e2af9f00cfb197006382610088
:105fa000030032006faa97000402e900e4af9f00eb
:105fb000cfb29700648262004700320062836200c1
:105fc0003c02900085037800e1826300e00f5300fb
:105fd000100032000404b200080032001c037800f4
:105fe000b4c2b300e08f52000100320004c2e800e6
:105ff000044b7800060ee80014003700b0022000c1
:10600000e08f5200010032000080e8008c00780030
:106010000b003700e08f5200250032000404b2006c
:10602000050032009c02780004c2b300844a780064
:10603000050ee800050037008c0078000002200003
:10604000ef060700e10f4000190032000e07e800dc
:10605000170037003c0090000004b200040032003a
:106060001c0078000d487800000ee8000d00370095
:106070008c0078000003200084bf9f00f5b79f00cc
:10608000d6b79f00e7b79f00dd0607000fba97005d
:10609000ffb297005fb39700efb39700e10f4000a6
:1060a000010032000e07e8008904e900040037000f
:1060b0000dc3b3000802be000a03be00efac970098
:1060c000e08f5400e3ff3c00e9af9f000404be00f2
:1060d0000605be00490037004fb097006802600017
:1060e00021003a00170037003c0090000004b20085
:1060f000040032001c0078000d487800000ee80013
:106100000d0037008c0078000002200084bf9f0043
:10611000f5b79f00d6b79f00e7b79f00b806070006
:106120000fba9700ffb297005fb39700efb39700e5
:10613000e10f4000010032000e07e8008904e90089
:10614000040037000dc2b3000802be000a03be00ff
:10615000efac9700e08f5400e3ff3c00e9af9f00f5
:106160000404be000605be00cfb097006283600045
:106170003c029000e1826000e00f5300100032000a
:106180000404b200080032001c037800b4c2b3005b
:10619000e08f52000100320004c2e800044b780096
:1061a000060ee80014003700b0022000e08f520015
:1061b000010032000080e8008c0078000b003700fe
:1061c000e08f52000d0032000404b20005003200de
:1061d0009c02780004c2b300844a7800050ee800ef
:1061e000050037008c0078000002200084060700bc
:1061f000e10f4000010032000e07e8000800be0079
:106200000a01be006d09070090a79f00a1a79f008b
:106210008001eb00b3a79f000002eb00c4a79f0022
:106220003c0290000404b2004f4397008602fb003a
:10623000830f5200110032001c047800432add0055
:10624000e52f2100848242005503be004502be00b6
:106250001fa09700afa097003fa19700cfa1970084
:10626000ff0a07000043b000004c7800080ee80069
:10627000e04f500010003a0010003700432add00c4
:10628000e52f2100848242005503be004502be0076
:106290001fa09700afa097003fa19700cfa1970044
:1062a000ef0a07000003b0008c00780054060700d6
:1062b000e10f4000010032000e07e800cf439700d5
:1062c0000702fb00c322dd00e42f2100050242008b
:1062d0005403be004402be001fa09700afa0970069
:1062e0003fa19700cfa19700e40a070080b79f0065
:1062f00091b79f00a2b79f00b3b79f00ffac970074
:10630000e08f540004003a00048020004fb597004d
:1063100004026500720032003c0290000404b200e6
:10632000050032009c027800e4c2b300844a780081
:10633000050ee800050037008c007800e002200020
:106340002f060700e10f4000010032000e07e800b1
:106350004f459700cfb697000d20b200e92f2100de
:1063600044003700e08f56000d0032000fb0970058
:106370009fb097002fb19700bfb19700e00f50007a
:10638000e08f5800e00f5900e08f590004003a00f8
:106390008040eb00c1479f000004eb004d00370038
:1063a000bc0290000504b2000402fb00e08f520022
:1063b000100032001c0478004322dd0004824400f7
:1063c0005403be004402be000fb097009fb0970078
:1063d0002fb19700bfb19700a10a07000043b0009a
:1063e000004c7800080ee800e04f500011003a0021
:1063f000110037004322dd00048244005403be0034
:106400004402be000fb097009fb097002fb19700d5
:10641000bfb19700920a0700040320000002420067
:106420008c00780004007800f5050700e10f4000bb
:10643000010032000e07e8004f4197000202fb0006
:106440004322dd00048244005403be004402be0027
:106450000fb097009fb097002fb19700bfb1970082
:10646000860a070080b79f0091b79f00a2b79f00e0
:10647000b3b79f00cf4297000542e900c4479f0091
:10648000e0cf5200b7ff3a000a02fb00ffaa9700d4
:10649000048452000f0037003c0290000404b20054
:1064a000040032001c027800094a7800040ee8005b
:1064b000050037008c00780000032000d00507009d
:1064c000e10f4000010032000e07e8000804e90077
:1064d0000100370009c3b300e00f5400eeff3a009b
:1064e000cfb297000502b2003c02900008003200d3
:1064f0000404b200030032009c02780054c4b300cc
:10650000070037008c007800500420000900370095
:106510000404b200050032009c02780054c6b300a7
:10652000844a7800050ee800050037008c007800ea
:1065300050062000b2050700e10f400001003200c4
:106540000e07e8004f829700bc029000e00f520057
:106550000d003d000402ea00c4879f000502780098
:106560000404b200050032009c027800d4c2b300db
:10657000844a7800050ee800100037008c0078008f
:10658000d00220000a003700050278000404b2009f
:10659000050032001c027800b6c2b300064a78003b
:1065a000040ee800050037008c007800b0022000df
:1065b00093050700e10f4000010032000e07e800dc
:1065c0003c0290000404b2004f8097000d0032009e
:1065d0009c027800a4002000811f780011000900af
:1065e0000400d80000027800cf0078000443b00017
:1065f000844a7800050ee800e04f520009003a0096
:1066000009003700a4002000110009000400d80090
:106610000003b0008c00780079050700e10f40000e
:10662000010032000e07e8003c0290000404b200b2
:106630004f8097000d0032009c027800a4002000db
:10664000811f7800110009000400d80001027800c1
:10665000cf0078000443b000844a7800050ee800bb
:10666000e04f52000a003a000a003700a400200060
:10667000110009000400d800010078000003b000f8
:106680008c0078005e050700e10f40000100320039
:106690000e07e800cfb39700688263004c05320014
:1066a0006fac9700e00f54004905340008c2b300f6
:1066b000efac97003c0290000404b20004003200ea
:1066c0001c027800084a7800040ee8000500370034
:1066d0008c0078000002200049050700e10f40000f
:1066e000010032000e07e8008904e900f1ff3a00da
:1066f00037053700e08f560004003d000d82ea00a8
:106700007fa8970004004000f0af9f000800be0083
:106710000a01be00f807070080b79f0091b79f00ed
:10672000a2b79f00b3b79f00e12f21000040eb000c
:106730000802be000a03be0094af9f00a5af9f00f1
:10674000b6af9f00c7af9f000c0037003102be00fc
:106750003103be000fb497009fb497002fb5970088
:10676000bfb597000440e10005c8e10006d0e10094
:1067700007d8e100030039000040e800f44f500062
:10678000f2ff3a001fac9700afac97003fad970007
:10679000cfad97000002fb007fa8970004005000d7
:1067a000f0af9f00f80f500009003c006fd8970031
:1067b00080fa07000002be000203be000800be000f
:1067c0000a01be00820607000004be000205be00ea
:1067d0006fd89700c1fa07000002be000203be0096
:1067e00094af9f00a5af9f00b6af9f00c7af9f00bb
:1067f0000fb097009fb097002fb19700bfb19700df
:10680000140807000002be000203be000800be001c
:106810000a01be00b40807000002be000203be0069
:106820001fa89700afa897003fa99700cfa997008e
:1068300038080700b0070700ffae97000802be0047
:106840000a03be0084b79f0095b79f00a6b79f00bc
:10685000b7b79f000205be000004be000900370064
:10686000a4002000050020006033b8000800be002e
:106870000a01be007a0907000205be000004be003e
:106880008d06e900e08f560019003200a4002000b8
:10689000050020006033b8000800be000a01be00f9
:1068a00076090700e00f5000e08f5800e00f590014
:1068b000e08f5900eaff32000d003700ffaa970071
:1068c000f88f52000f003c000540780039fa0700ad
:1068d0000002be000203be000800be000a01be00a6
:1068e0003b0607000004be000205be00050037009d
:1068f000fdaf9f000fb497009fb497002fb597008e
:10690000bfb59700cf869700e98f560011003c0075
:106910006022b8006033b8000800be000a01be0063
:106920000c070700e00f50002c0032000800be00ea
:106930000a01be0070070700e00f5000e08f58000a
:10694000e00f5900e08f590024003a00e18f560013
:10695000220034000400200005002e00b6e02200d2
:10696000170124005f989700ef9897007f99970090
:106970008fa1970093060700e00f500002003d0032
:10698000f386560001003700f2865600cd879f003f
:106990000f48970051fa07000002be000203be0034
:1069a000d49f9f00e59f9f00f69f9f0087a79f00b1
:1069b0000800be000a01be008c0607004e07070053
:1069c00080b79f0091b79f00a2b79f00b3b79f0009
:1069d0006044b8006055b800110037000800be00e0
:1069e0000a01be004407070080b79f0091b79f00cf
:1069f000a2b79f00b3b79f00960707000002be0032
:106a00000203be000800be000a01be0036080700ef
:106a10000004be000205be000002eb00c4879f0018
:106a20006130210010c0b3000802be000a03be009e
:106a3000d4a79f00e5a79f00f6a79f0087af9f0000
:106a4000100037003104be003105be0098af9f0032
:106a5000a9af9f00baaf9f00cbaf9f000fb29700c6
:106a60009fb297002fb39700bfb397000820e100b3
:106a700009a8e1000ab0e1000bb8e1000300390009
:106a80000040e800f44f5000eeff3a005fa497008a
:106a9000efa497007fa597008fad9700c0479f0098
:106aa0004f829700efaa9700048252007fab9700b5
:106ab000860252000002fb0004825200e4af9f00f5
:106ac00004802000cfb397000482630094af9f003e
:106ad00002003a00e00f5300030032006fa8970055
:106ae0000000e900e0af9f00cfb097006382600034
:106af000030032006fa997000201e900e2af9f0096
:106b0000cfb1970064826100470032006282610069
:106b1000e1826100e00f5200110032003c0290005f
:106b20000404b200080032001c037800b4c2b300b1
:106b3000e08f52000100320004c2e800044b7800ec
:106b4000060ee80015003700b0022000e08f52006a
:106b5000010032000080e8008c0078000c00370053
:106b6000e08f5200260032003c0290000404b20084
:106b7000050032009c02780004c2b300844a780009
:106b8000050ee800050037008c00780000022000a8
:106b90001b040700e10f4000190032000e07e80057
:106ba000170037003c0090000004b20004003200df
:106bb0001c0078000d487800000ee8000d0037003a
:106bc0008c0078000003200084bf9f00f5b79f0071
:106bd000d6b79f00e7b79f00090407000fba9700d8
:106be000ffb297005fb39700efb39700e10f40004b
:106bf000010032000e07e8008904e90004003700b4
:106c00000dc3b3000802be000a03be00efac97003c
:106c1000e08f5400e3ff3c00e9af9f000404be0096
:106c20000605be0076003700cfb29700688262008a
:106c300021003a00170037003c0090000004b20029
:106c4000040032001c0078000d487800000ee800b7
:106c50000d0037008c0078000002200084bf9f00e8
:106c6000f5b79f00d6b79f00e7b79f00e403070082
:106c70000fba9700ffb297005fb39700efb397008a
:106c8000e10f4000010032000e07e8008904e9002e
:106c9000040037000dc2b3000802be000a03be00a4
:106ca000efac9700e08f5400e3ff3c00e9af9f009a
:106cb0000404be000605be004fb3970062026300e5
:106cc000e1026300e00f5200110032003c0290002c
:106cd0000404b200080032001c037800b4c2b30000
:106ce000e08f52000100320004c2e800044b78003b
:106cf000060ee80015003700b0022000e08f5200b9
:106d0000010032000080e8008c0078000c003700a1
:106d1000e08f52003a0032003c0290000404b200be
:106d2000050032009c02780004c2b300844a780057
:106d3000050ee800050037008c00780000022000f6
:106d4000af030700e10f40002d0032000e07e800fe
:106d50002b0037003c0290000404b2008502fb00c7
:106d6000e00f5200110032009c067800c32add00bb
:106d7000e72f2100858243005503be004502be0077
:106d80000800be000a01be0035080700a40020006c
:106d9000050020006033b8003808070004c3b300c2
:106da000844e40000d0ee80013003700c32add00ba
:106db000e62f2100850243005503be004502be00b8
:106dc0000800be000a01be0025080700a40020003c
:106dd000050020006033b8002808070004032000e5
:106de000000242008c007800040078008403070051
:106df000e10f40000c0032000e07e8000a003700e7
:106e00000800be000a01be00d0a79f00e1a79f00b6
:106e1000f2a79f0083af9f000fb497009fb4970025
:106e20002fb59700bfb597004f4297008442e90005
:106e3000c5479f00e04f5200c6ff3a0011003700df
:106e40003c0290000404b200040032001c027800ee
:106e50000d4a7800040ee800050037008c00780029
:106e60000003200066030700e10f4000010032002c
:106e70000e07e8004f8297000402e900c4879f00d4
:106e8000050037005fa49700efa497007fa5970047
:106e90008fad97000dc3b3004f829700e00f5200f3
:106ea000e7ff3c00ffa89700f28f5000030034007a
:106eb00024c1b300c4479f00020037006fd9970078
:106ec000c2479f00cf4297000502fb00ffa9970031
:106ed00084865100e0cf520003003a001faa9700b9
:106ee000e00f52000e0032003c0290000404b20099
:106ef000050032009c027800e4c2b300844a7800a6
:106f0000050ee800050037008c007800e002200044
:106f10003b030700e10f4000010032000e07e800cc
:106f20004f409700edf807000002be000203be00cc
:106f30000800be000a01be0076060700ee05070045
:106f400080b79f0091b79f00a2b79f00b3b79f0083
:106f5000e92f2100390037003c0290000404b20000
:106f60008502fb00e00f5200120032001c04780082
:106f7000c32add00858244005503be004502be00e1
:106f80000fb097009fb097002fb19700bfb1970047
:106f9000b3070700a4002000050020006033b800fc
:106fa000b60707000ac3b3000a4c4000080ee80009
:106fb00012003700c32add00858244005503be005d
:106fc0004502be000fb097009fb097002fb1970009
:106fd000bfb19700a2070700a40020000500200011
:106fe0006033b800a50707000003b0008c007800ec
:106ff00003030700e10f4000010032000e07e80024
:10700000cf4597000b02fb004322dd0004824400c1
:107010005403be004402be000fb097009fb097001b
:107020002fb19700bfb197009407070080b79f006a
:1070300091b79f00a2b79f00b3b79f004f42970040
:107040008442e900c5479f00e04f5200c2ff3a006a
:107050000f0037003c0290000404b200040032002c
:107060001c027800084a7800040ee800050037008a
:107070008c00780000032000e1020700e10f4000cf
:10708000010032000e07e8008d06e900010037001c
:1070900008c3b300e08f5600eeff3a00cfb297006e
:1070a00068826200ca0232006fab9700e00f5300a3
:1070b000c702340008c2b300860478003c02900086
:1070c0000404b200040032001c027800084a780070
:1070d000040ee800050037008c0078000002200054
:1070e000c7020700e10f4000010032000e07e80070
:1070f0008904e900f1ff3a00b5023700cfb29700ea
:10710000050cb20040003a00cfb39700e08f530067
:1071100005003d005fa897004005be004004be008a
:10712000d0af9f0011003700cfb097007082600091
:10713000130032005faa97004401be00d4af9f0045
:10714000b28f9f00c38f9f008402780015029000c9
:107150004fa2de00d48f9f00e48f9f003f8c9700ea
:10716000cf8c97005f8d9700ef8d970088b79f00b9
:1071700099b79f00aab79f00bbb79f000b003700cd
:10718000dfac970049027800d9af9f000400780077
:10719000cf80de00010178008201780080b79f0077
:1071a00091b79f00a2b79f00b3b79f000fb297009f
:1071b0009fb297002fb39700bfb39700e00f520024
:1071c000e08f5a00e00f5b00e08f5b0034003d0071
:1071d000cfb297003500b300c5b79f006022b8005a
:1071e0006033b8000fb497009fb497002fb5970095
:1071f000bfb597000804520089845a000a055b0055
:107200008b855b0022003700cfb49700e08f5400dd
:1072100005003d005faa97004401be004400be0087
:10722000d4af9f000e0037004fb39700f002630009
:10723000100032005fad97004a04be00daaf9f0035
:10724000f8879f00898f9f00948f9f00a48f9f00d5
:107250007f8097008f8897001f899700af899700dc
:1072600080b79f0091b79f00a2b79f00b3b79f0060
:107270000b003700dfa8970041027800d1af9f00d4
:1072800004047800090020000a0020000b00200000
:1072900088b79f0099b79f00aab79f00bbb79f0010
:1072a000ffac9700e08f54000d003a001a00200058
:1072b000faaf9f000fb097009fb097002fb19700d3
:1072c000bfb19700e00f5000e08f5800e00f590069
:1072d000e08f5900020032008000eb00f1af9f0008
:1072e0004fb19700020cb20092af9f00040420003f
:1072f000840f51003400320003003c00e00f5100c5
:107300000800320048003700040820009fa99700b9
:10731000848f510014003200040c2000848f51002f
:1073200041003a006130210010c0b3003102be00bc
:107330003103be000fb497009fb497002fb597009c
:10734000bfb597000440e10005c8e10006d0e100a8
:1073500007d8e100330039000040e800f44f500046
:10736000f2ff3a002f00370010c0b30004012000e4
:10737000050020006033b8000fb497009fb4970059
:107380002fb59700bfb597000440e10005c8e100a4
:1073900006d0e10007d8e1002200390049002000b2
:1073a0000402d0008582d2000683d2008783d200f7
:1073b0008904e900faff3a000040e800f04f50006d
:1073c000edff3a001700370010c0b3008400200022
:1073d000050020006033b8000fb497009fb49700f9
:1073e0002fb59700bfb597000440e10005c8e10044
:1073f00006d0e10007d8e1000a003900390020007a
:107400000402d0008582d2000683d2008783d20096
:107410008904e900faff3a000040e800f54f500007
:10742000edff3a00c0479f004f4597000a02fb005e
:10743000ffad97008b0f520002003d00cb479f002d
:10744000040037007fa89700840f500001003d0022
:10745000f4af9f00efa89700e08f500005003200c6
:107460004fb1970063026100020032008100e90021
:10747000e1af9f0004002400cfb1970004826100b7
:10748000090032006faa9700ffaa9700850f5200eb
:107490000300340005025200e4af9f0002003700f1
:1074a0000003eb00e6af9f00448c2000cfb39700b1
:1074b000848263004408b100848f520006003a00c1
:1074c0006fac9700e00f5400110032000804e9008f
:1074d000e8af9f000e003700048c2000cfb4970067
:1074e000848264000404b100848f520008003a00d2
:1074f0006fad9700e20f5500030034000a85e900e4
:10750000eaaf9f00020037008005eb00ebaf9f0061
:107510004f4097000002fb008000eb00d1a79f00c6
:107520006fa99700840f510002003400040251003b
:10753000d4a79f00cfb19700648261006000320041
:1075400062826100e1826100e00f520010003200af
:107550003c0290000404b200080032001c037800d2
:10756000b4c2b300e08f52000100320004c2e80050
:10757000044b7800060ee8003a003700b002200005
:10758000e08f5200330032000080e8003100370005
:10759000e08f5200090032003c0290000404b20067
:1075a000030032009c02780004c2b30022003700be
:1075b0008c0078000002200027003700048c200097
:1075c0004fb39700840263000404b100848f52001b
:1075d00025003a003c0290000404b200050032008d
:1075e0009c02780004c3b300844a7800050ee800ca
:1075f000050037008c0078000003200080010700a0
:10760000e10f4000010032000e07e8003c0290004c
:107610000404b2004fb397000602b200e00f52001c
:10762000080032009c02780084c7b300e00f5300ca
:107630000100320084c5b300844a7800050ee800da
:107640000800370080072000e00f530001003200df
:10765000800520008c00780069010700e10f4000e0
:10766000010032000e07e800dfa39700e08f53000f
:107670008800320008c3b300870478003c02900001
:107680000404b200040032001c027800084a7800aa
:10769000040ee800050037008c007800000320008d
:1076a00057010700e10f4000010032000e07e8001b
:1076b0008904e900f1ff3a00d9a79f00750037005f
:1076c0005fa49700e00f540015003200cfb497007c
:1076d0006882640012003a0008c2b300dfa4970079
:1076e0003c0290000404b200040032001c02780046
:1076f000084a7800040ee800050037008c00780086
:10770000000220003e010700e10f400001003200ae
:107710000e07e8008904e900f1ff3a00d9a79f00ad
:107720004fb5970062026500e1026500e00f52006c
:10773000110032003c0290000404b2000800320044
:107740001c037800b4c2b300e08f52000100320085
:1077500004c2e800044b7800060ee800150037006c
:10776000b0022000e08f5200010032000080e800eb
:107770008c0078000c003700e08f52000e003200c1
:107780003c0290000404b200050032009c02780024
:1077900004c2b300844a7800050ee80005003700f3
:1077a0008c0078000002200015010700e10f400066
:1077b000010032000e07e800048c2000cfb59700ce
:1077c000848265000408b100848f520009003a00e9
:1077d0003c0290000404b200030032009c027800d6
:1077e00004c3b3001f0037008c00780000032000a2
:1077f0002400370004882000848f520025003a00be
:107800003c0290000404b200050032009c027800a3
:1078100004c3b300844a7800050ee8000500370071
:107820008c00780000032000f5000700e10f400005
:10783000010032000e07e8003c0290000404b20090
:107840004fb397000602b200e00f5200080032006a
:107850009c02780084c7b300e00f5300010032009f
:1078600084c5b300844a7800050ee800080037009c
:1078700080072000e00f5300010032008005200047
:107880008c007800de000700e10f400001003200ac
:107890000e07e8007fa897000003e900c230dd0072
:1078a000e1af9f006332b90004017800f28f9f00be
:1078b0004333dd00e42f210084064300cfb197005d
:1078c000f0816100e3879f004fb297000402b2008d
:1078d000d4879f00a4003700ffaa97008502e90023
:1078e000f5af9f001fab970007042000870f5300e0
:1078f0007600320003003c00e00f53000800320025
:1079000081003700040820001fac9700840f54004a
:1079100059003200040c2000840f54007a003a0011
:10792000cfb49700e08f54001e003d003d04be0020
:107930002d05be000802be000a03be000fb097006e
:107940009fb097002fb19700bfb197004405070083
:10795000c0479f000000fb00cf80de0001017800df
:10796000820178000802be000a03be00a5050700d8
:107970000fb297009fb297002fb39700bfb3970045
:107980000002520081825a0002035b0083835b0085
:1079900084b79f0095b79f00a6b79f00b7b79f0019
:1079a00031003700ef829700e08f52002100320053
:1079b0000fb297009fb297003d04be002d05be0098
:1079c0000801be000400be0084bf9f00f5b79f0001
:1079d00069ed0700c0479f000000fb00cf80de007c
:1079e0000801be006d0407000fba9700ffb29700b0
:1079f0000003520081835a0086979f0097979f004b
:107a00008003eb00a7979f000004eb00b8979f004e
:107a10000f9097009f9097002f919700bf9197002c
:107a200080b79f0091b79f00a2b79f00b3b79f0098
:107a30000d0037001d0278008fb09700800278009b
:107a4000110009008480d8008002fd00a4002000fd
:107a5000809fbe00110009008482d80001027800d6
:107a60004f00be00c4479f004f4197000243b00043
:107a7000c2479f002400370074412100df81970036
:107a8000e08f510001003200644021000fb09700e8
:107a90009fb097002fb19700bfb19700efaa970052
:107aa0008502e900050033008301d1000281d30083
:107ab0008180d3000080d300f9ff37006f006000a1
:107ac00064407800c0479f000f0037000fb2970056
:107ad0009fb297002fb39700bfb397007f8c97009a
:107ae0000804e900050033008703d1000683d300b2
:107af0008582d3000482d300f9ff37006742620019
:107b00000443b000c4479f003c0290000404b2004c
:107b1000070032009c0278004f429700844a7800a8
:107b2000050ee800e04f520007003a00070037005a
:107b3000cf4497000900fb008c007800300007005c
:107b4000e10f4000010032000e07e8006fad970022
:107b500064055500eaaf9f00ff8d9700e38555004f
:107b6000fb8f9f00e88656007fa89700e00f50002b
:107b700059ff3a00cfb097006882600014003200cd
:107b80005fa19700e00f51001100340008c2b3005c
:107b9000820478003c0290000404b2000400320029
:107ba0001c027800084a7800040ee800050037003f
:107bb0008c0078000002200011000700e10f400057
:107bc000010032000e07e8008904e900f1ff3a00e5
:107bd000cf91970013407800c0479f00e04f5000be
:107be0002af63a000e0078004f0778004f06be00d4
:107bf0004f05be004f04be000f07b1000000060095
:107c0000889fbe000104780038029000e202620002
:107c10008084eb003b003200040378000620b200b1
:107c20009802900002003a00e08f520035003a00be
:107c30000490a0003404980080047800f90fb2008a
:107c4000e08f520002003a00a8029000050c780074
:107c5000ea8f540005003a000408b20003003a001d
:107c600088007800d0002000e5ff0700180290008f
:107c7000d8029000850f52000b0032000402e80089
:107c80001404980018027800094a7800040ce800ef
:107c900015c0b30024462100054a7800ea8f54003d
:107ca00018003a0005003700880078000940780085
:107cb0007f0007008004780012003700380290002f
:107cc0000410b2000f00320018019000a8009000cc
:107cd00048009000e100070018029000840f500057
:107ce00004003200380290000403b300340498000a
:107cf0008084eb000002eb0014049800280290003e
:107d0000040c7800090078004f04be000000060053
:107d100054a38000e00f5200010032000400010073
:107d20000043210004000700c043210002000700b7
:107d30008044210000003700889fbe008a1f780021
:107d40000004780038029000630262000080eb00bb
:107d50002a003200080078002b0007003805900048
:107d600084ef2f000402650034049800280090007e
:107d7000e00f500004003200e804650002003a0001
:107d80009a0007002904980048009000a800070006
:107d9000e10f400019003200b80490000902b2005f
:107da0000080eb0015003a00000021000000650093
:107db0001200320060a38000e00f50000f0032007c
:107dc000042a2000902a9000888f520006003a0072
:107dd000d400070064a38000890442000000eb0087
:107de000902c9800050037004905b0004005b00010
:107df000848f5400f3ff3a000000eb004f05780039
:107e00004f04be0000000600881f780000047800c0
:107e100038009000000278001420b200e10f5200f8
:107e200005003a000002eb001404980028029000bc
:107e3000040c780019003700800278002520b20079
:107e40000000eb0024202000848f520016003a002e
:107e5000a8009000808f500013003200180190009d
:107e6000800f510010003200480090007b00070096
:107e700018029000840f5000030032003802900076
:107e80000403b300340498000002eb0014049800cb
:107e900028029000040c7800380090000002b20024
:107ea000010032000080eb004f0478000000060063
:107eb0000200fa00889fbe00a0ff9f000104780026
:107ec00038029000840278000504b20002003200fb
:107ed0000000fb0035003700e202620005003a00b6
:107ee0000403b30034049800150498000080eb00ec
:107ef0002e003700d8049000e08f540006003a00ae
:107f000012002000e6805700480090005300070050
:107f10001904980023003700a8029000e08f520057
:107f200008003a005546210025049800050c780009
:107f30002500200055049800150498000430a00086
:107f40003404980018019000a800900048009000a8
:107f500042000700280290008082eb001504980080
:107f6000affa9700054a7800040ce8002ffa970052
:107f7000ea4f52000b003a00380290000410b200a1
:107f80000800320018019000a800900048009000fe
:107f9000320007000002eb0014049800a8029000d1
:107fa000050c78002ffa97000400fb004f04be0078
:107fb0000080fa000000060070a38000e00f50006f
:107fc000030032001002780074a38800020037001a
:107fd000200020005c000700e10f400002003a0092
:107fe000946e260044a388000000060074a380005d
:107ff0000408780070a388000000060004118000c7
:10800000e00f520006003d001511800004402000e2
:1080100004826200020032002302ab00feff320045
:108020000040da00feff370000c0da000000060062
:108030000a00fa0014002000b4bf9f00c0bf9f00d8
:108040006a805700f8ff07004fb897000080fa00d9
:108050000000060000c0da00000006000a00fa0076
:10806000e20f500022003e0084a38000e10f520086
:10807000060032008723200046232000242320000e
:1080800005232000e08f530004003a0087222000df
:108090004622200024222000052220000000280083
:1080a0001500600003003a00800b780007002800ec
:1080b000958a7300054020009482620001003a0016
:1080c00014a0a00082027800060037009403780014
:1080d0000710b200fdff3200b103fb00070b780070
:1080e0008502e900e08f5200f8ff3a0008003700ef
:1080f00034002000b4bf9f00c0bf9f00d1bf9f00cd
:10810000e2bf9f006a805700d2ff07006fb9970057
:10811000020078000080fa000000060000c0da00cb
:10812000000006000a00fa0054002000b4bf9f00bf
:10813000c0bf9f006a805700f8ff07005fb8970034
:108140000080fa0000000600889fbe0080047800ce
:1081500090a38000e00f500004003a000e000700da
:108160000084eb00e00f50000800350098a3800069
:10817000e08f5400050032000900440006000700ab
:10818000e00f500001003d000084eb000800780083
:108190004f04be0000000600e00f500004003a004b
:1081a0004447210094a388000002780006003700ad
:1081b0000082eb0045472200850f500002003e0080
:1081c00090a388000002eb00040078000000060085
:1081d0002800fa00889fbe008a9fbe008c9fbe00c8
:1081e00007067800878669000c003b0003047800ce
:1081f0008704780008f0a10009f0a100840f500066
:10820000858f5800860f5900890f5c0003003300ea
:108210000cf0a20001003a000cf0a100fe000700e3
:108220006400e1005f003200780147006408e1006b
:10823000610032006c014700748557003200be00b7
:108240001201be003a04be001a05be001e039000d3
:10825000be0a90008503530006003d000004fd00a7
:108260008104fd000205fd008305fd008703ea008f
:10827000050378000df8a300040032006004140028
:10828000e0841c0060051d00e0851d006022b80030
:108290007d0320000d38e1008006eb000b00390063
:1082a0004433dd00f300b20083017300390037006e
:1082b000848272000d027800e10664008b85d10093
:1082c0000a85d3008984d3000884d3008703e9009a
:1082d000f7ff3b0008004000898048000a01490080
:1082e0008b81490004003b0060001000e080180012
:1082f00060011900e08119000358a3000900320051
:108300008d82720084827200610260008301d1005c
:108310000281d3008180d3000080d3000603e800ef
:108320001b0037000348a30017003a000600e000d6
:10833000170034000603e9000d00a3000000480008
:108340008180480002014900838149000348a3005d
:108350000f003a000600e000090034000603e900bf
:1083600000004000818048000201490083814900eb
:1083700001003a000003eb000348a300f5ff3200c0
:108380006022b800020037008482720061826600b9
:108390007500070003f0a1000cf0a70003f0a00097
:1083a000b1003700640147006408e10002003a00b0
:1083b0000df8a300a9003a003200be001201be0071
:1083c000a90037008f1fd100440307008f87e90001
:1083d0000000e00000000600809feb003f03070064
:1083e0008f87e9000000e000000006002800fa0086
:1083f000889fbe008a9fbe008c9fbe0003866b00d4
:10840000850007006400e100440032006408e100d8
:108410004a0032006100e100460032006108e100dc
:1084200049003200ec0647006000b8003d02be0083
:108430003d03be00f48657006011b8003d04be0045
:108440003d05be007d0320000b0037000000a000aa
:108450008d06e900130032000402420085824a00c2
:1084600006034b0087834b000000400081804800da
:1084700002014900838149000802520089825a00a2
:108480000a035b008b835b00f0ff3b0008024200a5
:1084900089824a000a034b008b834b008d06e9005a
:1084a000edff3a008482720086827200f707b20004
:1084b0008782720001003200150020001e04900027
:1084c0003e0b900006035400e63fb0000368a30093
:1084d000070032000000a7000500a0008301d100c2
:1084e0000281d3008180d3000080d3000603e8001e
:1084f0008301d1000281d3008180d3000080d300aa
:108500000002eb000482d2001700070003f0a10074
:108510000cf0a70003f0a0005300370064024700ee
:108520006408e1004d0032003400be003401be009a
:10853000f6ff37006108e100480032006011b80022
:108540006000b800f1ff370003ff270002002000a1
:10855000fbff3700801feb00e00207008f87e90078
:108560000000e00000000600180020005700200076
:10857000080453000d003d000600200097fc2f006a
:108580000740e1001e003400848272006102600036
:108590008301d1000281d3008180d3000080d30009
:1085a0000804e800f8ff3a0047002000610460007a
:1085b00005047400040464000d00320061004000f2
:1085c000e080480060014900e081490003b8a5004f
:1085d000070032000603e8006538e10004003a00b5
:1085e0008301d1000281d3008180d3000080d300b9
:1085f000f87f20000830e100030035000803780010
:108600006000b8006011b8004433dd00f300b20030
:108610008301730000000600680447000294be0056
:108620000094be00fc0447008694be008494be0003
:1086300009007800f202070008007800f002070045
:1086400099007800814f70000b003b000800be00cd
:10865000cb0207004f00b10003003700f3ff2700f3
:10866000f2ff2f006110b9004f06be004f05be009b
:108670004f04be000080fa0000000600810378006d
:108680007cea07000001be006000b8000478a30087
:1086900013003a006220e10015003e000d00390091
:1086a0008301d1000281d3008180d3008301d100f6
:1086b0000281d3008180d3008301d1000281d300e5
:1086c0008180d3000538b000c42add00f300b20079
:1086d0008381720007f0a70003f0a00000000600ed
:1086e000f3ff2700f2ff2f006110b900fbff3700f6
:1086f00003ff2700f7ff37001400fa00889fbe0031
:108700008a9fbe008c9fbe000004be000205be0012
:10871000680047000a90be000890be00b80207003b
:108720000070a7000bf0a1000bf8a30020003a0096
:108730009e0990000e099000fe0090006e009000cf
:108740009e0290003443200084825200c6ff320013
:108750000a003c00b4fc2f000428e100140034009f
:108760008301d1000281d3008180d3000080d30037
:108770008502e800faff3a00bbff3700b400200092
:108780000428e10007003c00000040008180480010
:1087900002014900838149008502e900faff3a009d
:1087a000b1ff37000300280002002000010037005d
:1087b0006011b8006000b800abff37001400fa0089
:1087c000889fbe008a9fbe008c9fbe000004be0032
:1087d0000205be00680047000a90be000890be0077
:1087e000870207000070a7000bf0a1000bf8a300a0
:1087f00016003a009e029000304320008082520012
:10880000b0fe2f000028e1000d003c00b0fc2f005e
:108810000028e1000d0034001e0990008e08900031
:108820007e0090000501b0000201d1008180d300dc
:108830000080d3008502e800fbff3a008aff370082
:10884000010028000000200087ff37006000b8000a
:1088500085ff3700889fbe0000827000040271000f
:10886000048271002400320036432000c50020003d
:108870008383cf000a0039000541b1008283cf0015
:10888000070039000541b1008183cf0004003900a1
:108890000541b1008083cf00010039000541b100de
:1088a00085c353006022b800120032000a003b006a
:1088b00084827200610260008301d1000281d300d2
:1088c0008180d3000080d3000603e8008743e800de
:1088d000f7ff3a00070037000000400081804800a1
:1088e00002014900838149000603e9008743e9004a
:1088f000f9ff3a001cff07004f04be00000006000d
:108900006011b800d3ff3700e701070005097800c0
:10891000000006002800fa00889fbe008a9fbe0063
:108920008c9fbe0003866b003bff07000028a3005e
:1089300064003a000128a30067003a000008a30081
:1089400062003a000108a30065003a001e00900092
:10895000be08900081064000ed3fb100f480570052
:10896000ee019000111ab8008e099000311bb8007a
:108970009e099000311cb800511db800f4855700c5
:1089800046000700fe0190003a0007008b85e800d2
:108990003e0007008e09900040000700ee019000a5
:1089a000340007008b85e800380007008e0990002e
:1089b000400007009e0990001b18b8008904400081
:1089c0000a854800fe019000340007008b85e8000e
:1089d00038000700ee019000300007008e0990007b
:1089e0001b18b800890440000a8548000a98a300b3
:1089f00008003a000402420085824a0006034b0048
:108a000087834b0008044c0089844c000a054d0004
:108a10008d06e90084827200850273004c3add0005
:108a2000850272000100320015002000443ade0089
:108a30001400b2004538de00cb45dd000b007000ad
:108a4000c540de00cb4ddd008b8070004549de0067
:108a5000cb55dd000b017100c551de000d03780020
:108a6000c1fe070003f0a1000cf0a70003f0a00076
:108a7000fdfe37001b18b800850240000683480041
:108a8000e0834b0060044c00070037001b18b8005f
:108a90000603400087834800faff37001b18b80020
:108aa0008703400008844800e0844c0060054d00c6
:108ab000000006001b18b800080440008984480024
:108ac000faff37000108a300e4fe3a005800be0098
:108ad0005801be00e3ff37000008a300dffe3a00a4
:108ae00009047800f9ff370007f0a200b8fd37004d
:108af0001400fa00889fbe008a9fbe008c9fbe00b3
:108b00000005be000206be00680047000c90be00d3
:108b10000a90be00ba0107006400e1001a003200aa
:108b200016003e006100e1001a0032006e04900061
:108b3000fe0490000e0b90009e0b90006011b80098
:108b40009e0590000b38b100d50120008281710094
:108b5000610164008703d1000683d3008984d300b8
:108b60000884d3008502e900f8ff3a0090e8070086
:108b70000df0a70001f0a000bbfe3700f1ff2700b9
:108b8000f0ff2f00b8fe370001f82700000020009a
:108b9000f7ff37006000b800f5ff3700020ab900a0
:108ba000001bb9000200b8008100420081004300b0
:108bb00000000600889fbe008a9fbe003004be00f1
:108bc0002005be000404440085844c0006054d00c9
:108bd00087854d000898be000a90be000440e10061
:108be00005c8e10006d0e10007d8e100020031002d
:108bf000680040001008e8004f05be004f04be00aa
:108c0000000006001000fa00889fbe008a9fbe0088
:108c10000605be000404be003002be002003be00f4
:108c2000c4b79f00d5b79f00e6b79f00f7b79f0076
:108c30000802520089825a000a035b008b835b00a2
:108c400084bf9f0095bf9f00a6bf9f00b7bf9f0036
:108c50000498be000698be00110020004fb2970095
:108c6000dfb297006fb39700ffb397000820e100d1
:108c700009a8e1000ab0e1000bb8e10001003900e9
:108c80008000eb00108810004f05be004f04be00ae
:108c90000080fa00000006001400fa00889fbe0061
:108ca0008a9fbe008c9fbe003f0007000605be00e5
:108cb0000404be000006eb00ccb79f00bcb79f00c9
:108cc000acb79f009cb79f008cb79f000d0420009d
:108cd0004fb39700bfb29700860343002fb29700af
:108ce000e00f530004003d003d0007000f0040006e
:108cf000b0ff070003003700390007000f004000f5
:108d0000c0ff0700cfb2970095bf9f00e08f5200d1
:108d1000090035002b00070014002000050020008a
:108d20006033b8000000720081807200020173009d
:108d3000838173001c0007000c06e8008d0f5600ad
:108d4000e3ff3a001fba9700e00f520005003d0014
:108d50000802be000a03be0000fe2f000f00400004
:108d600094ff07004faa9700e00f520008003a0056
:108d70000fb497009fb497002fb59700bfb5970029
:108d8000d8b79f00e9b79f00fab79f008bbf9f003d
:108d90000c0007004f06be004f05be004f04be008a
:108da0000080fa0000000600010007000000060035
:108db00090b79f00a1b79f00b2b79f00c3b79f00b5
:108dc0000000060001000700000006001fb0970029
:108dd000afb097003fb19700cfb1970000000600f9
:108de0004f2bde0087037300a7b79f004f23de00e1
:108df000858242008502730095b79f00ffaa970005
:108e00004f2bde00040242000402730084b79f006f
:108e10006faa97004f23de0085824200850273000f
:108e2000f5af9f00e9ff07004f18de000402420083
:108e300000027200e4af9f00e4ff07000000400062
:108e4000818048000201490083814900d8ff070062
:108e50000802be000a03be0000fe2f00000006004c
:108e6000881f780018002000881f78008aff0700fc
:108e70008f87e9004f04780000000600801feb0098
:108e800085ff07008f87e90000000600889fbe006d
:108e90008a9fbe00e00f5000e08f5800e00f59009d
:108ea000e08f59000c003d006044b8006055b800e8
:108eb0000000540081805c0002015d0083815d0040
:108ec000180020001500070008003d0018000700ea
:108ed0000004eb00050037000004eb000f00070062
:108ee00002003d001200070018002000dcff070010
:108ef000e00f5400060032006022b8006033b80072
:108f00000000520081805a0002015b0083815b00f7
:108f10004f05be004f04be0000000600e00f5200e7
:108f2000e08f5a00e00f5b00e08f5b00000006005e
:108f30006044b8006055b8000402540085825c00ab
:108f400006035d0087835d0000000600889fbe0069
:108f50008a9fbe008c1f7800e00f5000e08f580001
:108f6000e00f5900e08f59000d003d006044b8004b
:108f70006055b8000000540081805c0002015d0073
:108f800083815d001c0020000820e10009a8e100a9
:108f90000ab0e1000bb8e1000d003d000800370009
:108fa0000006eb00e00f5200e08f5a00e00f5b007c
:108fb000e08f5b0006003d006044b8006055b800db
:108fc0000402540085825c0006035d0087835d0017
:108fd000aaff0700e00f5600060032006022b8002a
:108fe0006033b8000000520081805a0002015b002b
:108ff00083815b004f0678004f05be004f04be0022
:1090000000000600889fbe008a9fbe008c1f78006b
:109010000006eb00e00f5000e08f5800e00f590011
:10902000e08f590007003d006044b8006055b8006b
:109030000000540081805c0002015d0083815d00be
:109040001c002000e00f5200e08f5a00e00f5b0090
:10905000e08f5b0007003d006044b8006055b80039
:109060000402540085825c0006035d0087835d0076
:109070000c00a20089000700e00f56000600320035
:109080006022b8006033b8000000520081805a00ae
:1090900002015b0083815b004f0678004f05be0034
:1090a0004f04be00000006000003be00f1e7070009
:1090b0006220e100020032000600be00050005004b
:1090c000e507b100f107b20004f0230084807000ce
:1090d00007f0a70001f0a00024000500889fbe0053
:1090e0008a9fbe008c9fbe000404be000605be0021
:1090f000809fbe00829fbe002f00070004067800fc
:109100000800be000a01be002b000700840678009c
:109110004f03be004f02be008d4f76007fb0970018
:1091200013003300f0ff2f008b8f6b0006003b0015
:109130000d0666000c00a7000a00370007f0a60025
:10914000100020000a003700880f5200898f5a0053
:109150008a0f5b008b8f5b0003003900100020003a
:1091600001003e000000200007f0a7000000ea0018
:109170004f06be004f05be004f04be0000000600b3
:10918000e48240001078a30007003200640240002f
:109190001178a3003400be001401be0004003200a8
:1091a0000330a700000006003500be001501be0018
:1091b0000330a0000000060005ff270005826100c3
:1091c000070032000428e1000100320024000500fd
:1091d0000600070001003a004400050004080500ed
:1091e00002000700f9ff3a00140005006f826100d9
:1091f0008102700085027100850272000000060085
:10920000800078005002be005003be004439de00ea
:10921000f700b200f37f2000030161000900320073
:109220000218e10016003a00850172008301730004
:10923000838173000008200015003a0040002000e0
:10924000130037008501720083017300838173006e
:1092500005003a0004a8be0006a8be0010002000c9
:109260000b0037000201e9000402420085824a0037
:1092700006034b0087834b000748a300f9ff320029
:109280000740a00004a8be0006a8be0020002000e1
:10929000800098009200980000000600889fbe00a1
:1092a0008a9fbe008c9fbe000404b8000506b8006b
:1092b0008904460060854e000606b8000a0546008f
:1092c000e0854e000706b8008b054600040eb80086
:1092d000890446000a854e00e0854d00050eb80061
:1092e0000a0546008b854e00060eb8008b05460029
:1092f0000416b8000a0546008b854e000516b80016
:109300008b054600041eb8008b0546000800be0011
:109310000a01be004f06be004f05be004f04be004e
:049320000000060043
:020000040000fa
:10932400766f00006e000000766f00006666000035
:10933400006f00006e0000006f6600006600000011
:10934400666f00006e000000666f00006666000035
:109354000061000061000000617200000061000013
:109364006e000000616d00000061000070000000ec
:109374007376000000670000660000006763000069
:10938400007700000064000000680000007800001e
:109394000071000000740000657300007400000098
:1093a40056490000434f0000523100005f54000052
:1093b400454d000050000000646500006720000077
:1093c4004300000056490000434f000052320000a1
:1093d4005f540000454d0000500000005649000055
:1093e400434f0000523300005f540000454d00001d
:1093f400500000004845000041540000534900005b
:109404004e4b000000340000385600005f3100006d
:109414005f4300005552000052000000616d0000df
:109424007073000000340000385600005f31000003
:109434005f5600004f4c000054000000766f00009f
:109444006c7400007300000034380000565f0000a4
:10945400325f000043550000525200000034000007
:10946400385600005f3200005f5600004f4c000089
:109474005400000032340000565f000043550000e1
:109484005252000000320000345600005f560000c3
:109494004f4c000054000000332e000033560000ef
:1094a4005f4300005552000052000000332e0000bc
:1094b400335600005f5600004f4c0000540000007b
:1094c400414d0000425f0000485500004d0000007f
:1094d4002552000048000000414d0000425f00009a
:1094e400544500004d500000004700004e44000069
:1094f4005f460000415500004c5400000075000018
:10950400616d00007073000000460000414e0000d1
:109514003031000020000000464100004e300000c1
:109524003220000000560000494300004f52000062
:10953400303100002000000056490000434f000075
:109544005230000032200000004600004f4300006b
:1095540045300000315f0000524500004c410000de
:1095640059200000004600004f4300004530000031
:10957400325f0000524500004c41000059200000b9
:1095840000340000385600005f3000003100000055
:1095940034380000565f0000303100005f52000094
:1095a4004554000000340000385600005f300000cd
:1095b4003200000034380000565f000030320000f2
:1095c4005f5200004554000000470000465f000061
:1095d400544500005354000000470000465f00005b
:1095e40054450000535400005f52000045540000ed
:1095f400000d00000a0000000d0a000044450000b0
:1096040042550000472000004d4500004e55000023
:10961400202d000020540000797000006520000017
:1096240061200000636f00006d6d0000616e00003a
:10963400643a00000d0a00000a00000068200000df
:10964400666f0000722000007468000069730000f7
:1096540020680000656c0000702000006d6500004b
:109664007373000061670000650d00000a000000cc
:1096740078200000746f0000206700006f20000055
:1096840062610000636b0000207400006f20000022
:109694006d610000696e0000206d0000656e0000c1
:1096a400750d00000a0a0000007600006f6e0000cd
:1096b4005b3100002d3200005d200000746f00005b
:1096c40020740000757200006e2000006f6e0000b0
:1096d4002061000020760000696300006f720000c2
:1096e4000d0a0000007600006f660000665b000053
:1096f400312d0000325d0000207400006f20000056
:1097040074750000726e0000206f00006666000031
:109714002061000020760000696300006f72000081
:109724000d0a0000006f00006e5b0000312d000088
:10973400325d0000207400006f200000747500008a
:10974400726e0000206f00006e2000006120000097
:10975400464f000043450000207000006f77000072
:109764006572000020720000656c000061790000e1
:109774000d0a0000006f0000666600005b31000007
:109784002d3200005d200000746f00002074000082
:10979400757200006e2000006f66000066200000f5
:1097a40061200000464f0000434500002070000087
:1097b4006f7700006572000020720000656c000085
:1097c400617900000d0a0000006600006f6e000061
:1097d4005b3100002d3200005d200000746f00003a
:1097e40020740000757200006e2000006f6e00008f
:1097f4002061000020660000616e00000d0a000078
:10980400006600006f660000665b0000312d0000fa
:10981400325d0000207400006f20000074750000a9
:10982400726e0000206f0000666600002061000078
:1098340020660000616e00000d0a00000a000000ae
:10984400617200005b3000002d310000345d0000c7
:10985400207400006f200000726500006164000045
:10986400206100006e200000616e0000616c000049
:109874006f670000207000006f720000740d00001c
:109884000a00000061610000207400006f200000e5
:109894007265000061640000206100006c6c0000cf
:1098a400206100006e6100006c6f00006720000002
:1098b400706f000072740000730d00000a00000055
:1098c40061700000207400006f20000072650000c9
:1098d40061640000206100006e6100006c6f000094
:1098e4006720000070610000726100006d65000077
:1098f40074650000727300000d0a0000006100002e
:109904006e5b0000312d0000393900005d2000003d
:10991400746f000020730000657400002061000073
:109924006e6100006c6f0000672000006e7500001f
:109934006d41000076670000202800006e7500006d
:109944006d6200006572000020730000616d00000c
:10995400706c000065730000207400006f2000002c
:1099640061760000657200006167000065290000ef
:109974000d0a0000006100006d5b0000312d000045
:10998400393900005d200000746f0000207300006e
:1099940065740000206100006e6100006c6f0000bf
:1099a4006720000061760000674d0000732000000e
:1099b400286d0000732000006265000074770000c9
:1099c400656500006e200000736100006d7000008a
:1099d4006c650000732900000d0a0000007300008c
:1099e40076200000746f00002072000065610000a2
:1099f400642000007379000073740000656d00003a
:109a0400207300007461000074750000732000006e
:109a140076650000637400006f7200002028000067
:109a2400706f00007765000072200000626900001a
:109a340074730000206f00006e2900000d0a0000fe
:109a440000670000665b0000302d0000355d0000fb
:109a5400207400006f200000736500007420000073
:109a6400677200006f7500006e64000020660000dd
:109a7400617500006c7400002063000068610000e0
:109a84006e6e0000656c00000d0a000000670000a7
:109a9400635b0000302d0000363300005d200000c1
:109aa400746f0000207300006574000020470000fc
:109ab40046200000636f00006e740000726f0000a7
:109ac4006c20000072650000676900007374000078
:109ad4006572000020280000696e00002064000008
:109ae40065630000696d0000616c00002c200000bb
:109af400736f000072720000792900000d0a0000e3
:109b040000770000207400006f20000072650000e0
:109b14006164000020770000617400006572000039
:109b2400206100006c610000726d0000730d000084
:109b34000a0a0000006400005b3000002d390000b8
:109b44005d200000746f0000207300006574000045
:109b5400206400006562000075670000206f00004b
:109b64007574000070750000742000006c650000be
:109b7400766500006c0d00000a0000000d0a00006c
:109b84004261000064200000706100007261000006
:109b94006d65000074650000723a00002025000025
:109ba400750d00000a000000456e00007465000099
:109bb4007220000061200000636f00006d6d0000e2
:109bc400616e0000643a0000202000000054000090
:109bd400757200006e6900006e670000206f00005f
:109be4006e20000056690000636f000072200000c0
:109bf400257500000d0a0000005400007572000075
:109c04006e6900006e670000206f00006666000049
:109c140020560000696300006f72000020250000d8
:109c2400750d00000a00000054750000726e0000fb
:109c3400696e0000672000006f6e0000204600007f
:109c44004f43000045200000726500006c61000075
:109c540079200000257500000d0a00000054000062
:109c6400757200006e6900006e670000206f0000ce
:109c740066660000204600004f43000045200000b7
:109c8400726500006c6100007920000025750000f9
:109c94000d0a000000540000757200006e69000097
:109ca4006e670000206f00006e2000004661000017
:109cb4006e200000257500000d0a0000005400000d
:109cc400757200006e6900006e670000206f00006e
:109cd4006666000020460000616e0000202500003a
:109ce400750d00000a0000004368000020250000f4
:109cf4003264000020200000252d000031320000d5
:109d0400732000002535000075200000636e0000fc
:109d14007473000020250000362e00003366000016
:109d24002041000044430000207600006f6c0000d6
:109d34007473000020250000362e000033660000f6
:109d440020250000730d00000a000000426100009d
:109d54006420000063680000616e00006e6500000e
:109d64006c2000006e7500006d62000065720000da
:109d74000d0a0000006e0000756d000041760000c1
:109d8400672000003d200000257500002c20000005
:109d940061760000674d0000732000003d20000044
:109da400257500000d0a00000053000065740000d2
:109db400206e0000756d00004176000067200000f1
:109dc400746f000020250000750d00000a000000db
:109dd400536500007420000061760000674d0000a8
:109de40073200000746f000020250000750d000032
:109df4000a000000537400006174000075730000d1
:109e04002056000065630000746f0000722000009b
:109e14003d2000003078000025780000205b000021
:109e2400200000004e4f00004e45000020000000be
:109e34005d0d00000a000000576100007465000019
:109e440072200000416c0000617200006d2000006f
:109e540056650000637400006f720000203d00002e
:109e64002030000078250000780d00000a00000072
:109e740042610000642000004746000020430000c7
:109e8400686100006e6e0000656c0000206e0000ca
:109e9400756d000062650000720d00000a0000008c
:109ea4004746000020430000686100006e6e000019
:109eb400656c0000207300006574000020740000cd
:109ec4006f200000746f0000202500007520000042
:109ed40028250000732900000d0a00000047000037
:109ee40046200000436f00006e740000726f000093
:109ef4006c2000007265000067200000736500009c
:109f040074200000746f00002030000078250000e9
:109f1400780d00000a00000054650000737400000e
:109f2400204300006f6d00006d6100006e6400004e
:109f34002c20000070610000726d0000203d0000c4
:109f440020250000752c00002064000069670000d3
:109f540069740000732000003d2000002575000096
:109f64000d0a000000000000302000002d20000039
:109f74005361000076650000206300006f6e0000ee
:109f8400666900006720000063680000616e0000dd
:109f94006765000073200000616e0000642000000b
:109fa4007265000073650000740d00000a00000073
:109fb400312000002d200000536800006f7700005e
:109fc40020620000756900006c64000020640000d9
:109fd4006174000065200000616e000064200000d0
:109fe400636f00006e660000696700000d0a0000e0
:109ff40000320000202d0000205300006574000092
:10a00400205300006c6100007665000020490000c8
:10a01400440d00000a000000332000002d20000041
:10a0240053650000742000004d6f0000646200005e
:10a034007573000020620000617500006472000006
:10a0440061740000650d00000a0000003420000067
:10a054002d2000005365000074200000626c000095
:10a06400696e00006b7900002064000065620000e6
:10a0740075670000207300007461000074650000bf
:10a084000d0a000000350000202d000020530000c0
:10a0940065740000207000006f7700006572000096
:10a0a40020720000657300006574000020730000d6
:10a0b40074610000746500000d0a000000360000a1
:10a0c400202d000020530000657400002062000071
:10a0d4006f6100007264000020730000657200006c
:10a0e400696100006c2000006e7500006d62000064
:10a0f400657200000d0a000000370000202d0000ea
:10a1040020530000657400002064000065660000b0
:10a11400617500006c7400002047000046200000b8
:10a1240063680000616e00006e6500006c730000df
:10a1340020730000616d0000706c00006564000015
:10a144000d0a000000440000202d000020440000ff
:10a154006562000075670000204d0000656e000018
:10a16400750d00000a00000046610000696c0000e3
:10a1740065640000207400006f2000007265000018
:10a1840061640000206300006f6e000066690000d7
:10a19400672c000020750000736900006e670000e2
:10a1a4002064000065660000617500006c740000a6
:10a1b400206300006f6e000066690000670d0000f8
:10a1c4000a000000496e0000766100006c6900001e
:10a1d40064200000636f00006d6d0000616e00007c
:10a1e400642c00002000000074720000792000003c
:10a1f400273f000027200000666f00007220000047
:10a20400686500006c7000002e0d00000a0000005c
:10a21400313500003a310000363a0000343700008e
:10a224000041000070720000203200003120000064
:10a234003230000031350000000d00000a4d0000ee
:10a2440065640000697500006d200000566f000011
:10a254006c7400006167000065200000436f00001b
:10a264006e760000657200007465000072200000c4
:10a27400535700002052000065760000202500009e
:10a28400752e0000253000003275000020250000e6
:10a29400732c000020250000730d00000a0000004c
:10a2a4005479000070650000203f00002066000023
:10a2b4006f720000206d0000656e0000750d0000d7
:10a2c4000a0d00000a000000534c00004156000033
:10a2d40045200000494400003a20000020200000ee
:10a2e40020200000257500000d0a00000042000037
:10a2f4004155000044200000524100005445000034
:10a304003a20000020200000202500006c75000089
:10a314000d0a0000004200004c4900004e4b0000b2
:10a32400592000004445000042550000473a00000f
:10a334002000000052450000534500005420000056
:10a34400504f000057450000523a00002020000002
:10a35400307800002530000032780000202800000a
:10a364002000000056490000434f00005231000015
:10a374002000000056490000434f00005232000004
:10a3840020000000524500004c41000059310000fb
:10a3940020000000524500004c41000059320000ea
:10a3a40020000000464100004e3100002000000063
:10a3b400464100004e320000200000004e6f0000b5
:10a3c4006e65000020000000290d00000a00000056
:10a3d4004746000020430000545200004c3a00005d
:10a3e4002020000020200000202000003078000001
:10a3f40025300000327800000d0a000000530000f0
:10a4040045520000494100004c2000004e55000018
:10a414004d3a000020200000202500006c7500004b
:10a424000d0a0000000d00000a000000456e000047
:10a434007465000072200000534c00004156000077
:10a4440045200000494400003a2000000049000073
:10a454006e760000616c0000696400002049000011
:10a46400443a000020250000752c000020760000ee
:10a47400616c00006964000020720000616e0000dd
:10a484006765000020690000732000005b31000054
:10a494002c330000325d00000d0a0000004500006e
:10a4a4006e740000657200002042000041550000f7
:10a4b4004420000052410000544500003a200000ae
:10a4c400004900006e760000616c000069640000c1
:10a4d4002042000041550000442000005241000089
:10a4e400544500003a200000256c0000750d000062
:10a4f4000a000000566100006c690000642000003e
:10a504007261000074650000732000006172000035
:10a51400650d00000a0000003936000030300000ec
:10a5240020310000393200003030000020330000b8
:10a534003834000030300000203500003736000089
:10a5440030300000206f0000722000003131000024
:10a5540035320000303000000d0a000000450000d4
:10a564006e74000065720000204200004c49000037
:10a574004e4b0000592000004445000042550000a5
:10a58400472000005b300000203d0000206f0000e9
:10a5940066660000207c000020310000203d0000a1
:10a5a400206f00006e5d00003a20000000490000aa
:10a5b4006e760000616c0000696400002073000086
:10a5c40074610000746500003a20000025640000f6
:10a5d4002c2000005b300000203d0000206f0000b4
:10a5e40066660000207c000020310000203d000051
:10a5f400206f00006e5d00000d0a000000450000a1
:10a604006e74000065720000207000006f77000017
:10a61400657200002073000074610000746500001e
:10a6240020610000742000005245000053450000e2
:10a63400542c000020680000657800000d0a00001a
:10a644005b4200006974000073200000302c00009d
:10a65400312000003d20000056690000636f0000b7
:10a6640072200000312c0000322000007c20000009
:10a674004269000074730000203200002c33000093
:10a68400203d000020520000656c0000617900004c
:10a69400203100002c320000207c00002042000009
:10a6a4006974000073200000342c00003520000081
:10a6b4003d200000466100006e200000312c0000a7
:10a6c400325d00000d0a0000004900006e760000b3
:10a6d400616c000069640000207300007461000074
:10a6e400746500003a200000307800002530000036
:10a6f400327800000d0a0000004500006e7400006e
:10a7040065720000204200006f6100007264000066
:10a714002053000065720000696100006c20000095
:10a724004e7500006d620000657200003a20000062
:10a73400004500006e7400006572000020470000b0
:10a74400726f0000756e0000642000004661000016
:10a75400756c00007420000063680000616e0000e6
:10a764006e6500006c730000206f00006e20000016
:10a7740061740000207200006573000065740000bd
:10a78400205b000042690000747300002030000068
:10a794002d35000020760000616c00006964000023
:10a7a4005d0d00000a00000000c1000081400000af
:10a7b40001c000008041000001c000008041000091
:10a7c40000c100008140000001c000008041000081
:10a7d40000c100008140000000c100008140000071
:10a7e40001c000008041000001c000008041000061
:10a7f40000c100008140000000c100008140000051
:10a8040001c000008041000000c100008140000040
:10a8140001c000008041000001c000008041000030
:10a8240000c100008140000001c000008041000020
:10a8340000c100008140000000c100008140000010
:10a8440001c000008041000000c100008140000000
:10a8540001c000008041000001c0000080410000f0
:10a8640000c100008140000000c1000081400000e0
:10a8740001c000008041000001c0000080410000d0
:10a8840000c100008140000001c0000080410000c0
:10a8940000c100008140000000c1000081400000b0
:10a8a40001c000008041000001c0000080410000a0
:10a8b40000c100008140000000c100008140000090
:10a8c40001c000008041000000c100008140000080
:10a8d40001c000008041000001c000008041000070
:10a8e40000c100008140000000c100008140000060
:10a8f40001c000008041000001c000008041000050
:10a9040000c100008140000001c00000804100003f
:10a9140000c100008140000000c10000814000002f
:10a9240001c000008041000000c10000814000001f
:10a9340001c000008041000001c00000804100000f
:10a9440000c100008140000001c0000080410000ff
:10a9540000c100008140000000c1000081400000ef
:10a9640001c000008041000001c0000080410000df
:10a9740000c100008140000000c1000081400000cf
:10a9840001c000008041000000c1000081400000bf
:10a9940001c000008041000001c0000080410000af
:10a9a40000c100008140000000c00000c10100009f
:10a9b400c303000002c20000c606000007c700006f
:10a9c40005c50000c4040000cc0c00000dcd00003f
:10a9d4000fcf0000ce0e00000aca0000cb0b00000f
:10a9e400c909000008c80000d818000019d90000df
:10a9f4001bdb0000da1a00001ede0000df1f00006f
:10aa0400dd1d00001cdc000014d40000d51500007e
:10aa1400d717000016d60000d212000013d300008e
:10aa240011d10000d0100000f030000031f100001e
:10aa340033f30000f232000036f60000f73700006e
:10aa4400f535000034f400003cfc0000fd3d00003e
:10aa5400ff3f00003efe0000fa3a00003bfb00000e
:10aa640039f90000f838000028e80000e92900005e
:10aa7400eb2b00002aea0000ee2e00002fef00006e
:10aa84002ded0000ec2c0000e424000025e500007e
:10aa940027e70000e626000022e20000e32300008e
:10aaa400e121000020e00000a060000061a100009e
:10aab40063a30000a262000066a60000a76700006e
:10aac400a565000064a400006cac0000ad6d00003e
:10aad400af6f00006eae0000aa6a00006bab00000e
:10aae40069a90000a868000078b80000b9790000de
:10aaf400bb7b00007aba0000be7e00007fbf00006e
:10ab04007dbd0000bc7c0000b474000075b500007d
:10ab140077b70000b676000072b20000b37300008d
:10ab2400b171000070b0000050900000915100001d
:10ab3400935300005292000096560000579700006d
:10ab440055950000945400009c5c00005d9d00003d
:10ab54005f9f00009e5e00005a9a00009b5b00000d
:10ab6400995900005898000088480000498900005d
:10ab74004b8b00008a4a00004e8e00008f4f00006d
:10ab84008d4d00004c8c000044840000854500007d
:10ab9400874700004686000082420000438300008d
:10aba4004181000080400000757300005263000082
:10abb4007642000075660000666500007250000071
:10abc4006f730000203c0000204d0000425f000035
:10abd40053450000525f000050440000555f0000e0
:10abe400534900005a4500005f4d000041580000e1
:10abf400002e00002e2f00002e2e00002f6d0000ce
:10ac04006f64000062750000732f0000727400000e
:10ac1400752f00006d62000072740000752e000034
:10ac240063000000655300006e640000537400006c
:10ac340061740000652000003d3d000020530000c9
:10ac440054410000544500005f540000585f000068
:10ac5400494400004c4500000065000052630000b8
:10ac6400765300007461000074650000203d00000c
:10ac74003d2000005354000041540000455f000093
:10ac8400525800005f490000444c00004500000099
:10ac94002820000065520000637600005374000011
:10aca40061740000652000003d3d00002053000059
:10acb40054410000544500005f520000585f0000fa
:10acc400494e00004954000020290000207c000067
:10acd4007c200000282000006552000063760000fc
:10ace4005374000061740000652000003d3d0000c5
:10acf4002053000054410000544500005f520000fe
:10ad0400585f000052430000562000002920000034
:10ad14007c7c0000202800002065000052630000b5
:10ad2400765300007461000074650000203d00004b
:10ad34003d2000005354000041540000455f0000d2
:10ad4400525800005f450000525200004f5200006c
:10ad54002029000000000000757300005263000009
:10ad640076420000756600006665000072500000bf
:10ad74006f730000203c0000204d0000425f000083
:10ad840053450000525f000050440000555f00002e
:10ad9400534900005a4500005f4d0000415800002f
:10ada400002e00002e2f00002e2e00002f6d00001c
:10adb4006f64000062750000732f0000617300006f
:10adc40063690000692f00006d6200006173000078
:10add40063690000692e00006300000065530000f1
:10ade4006e6400005374000061740000652000006c
:10adf4003d3d000020530000544100005445000034
:10ae04005f540000585f0000494400004c450000b6
:10ae14000065000052630000765300007461000076
:10ae240074650000203d00003d20000053540000e4
:10ae340041540000455f0000525800005f49000083
:10ae4400444c00004500000028200000655200002a
:10ae540063760000537400006174000065200000f4
:10ae64003d3d0000205300005441000054450000c3
:10ae74005f520000585f000052430000562000005b
:10ae8400292000007c7c00002028000020650000b0
:10ae94005263000076530000746100007465000082
:10aea400203d00003d2000005354000041540000a8
:10aeb400455f0000525800005f5700004149000000
:10aec400545f0000454f00004620000029000000a8
:10aed40030000000000000000040000000100000ee
:10aee400005000000020000000600000003000005e
:10aef400007000000010000000500000002000005e
:10af04000060000061640000634300006f6e000095
:10af14007665000072740000283000007825000077
:10af2400782c000020250000752900000d0a00007f
:10af340000610000647300003833000034780000be
:10af4400436f00006e7600006572000074280000f4
:10af540025750000292000003d2000002575000013
:10af640020280000436f00006e76000020250000ba
:10af74007520000063680000616e00002025000059
:10af8400752900000d0a0000000000007563000030
:10af94004e42000069740000732000003c3d000034
:10afa40020380000002e00002e2f00002e2e00005e
:10afb4002f6d00006f64000062750000732f0000a5
:10afc400667500006e630000746900006f6e000017
:10afd400732f00006d62000075740000696c00003e
:10afe400732e0000630000004f4e00000d0a0000a5
:10aff400004f0000464600000d0a0000000000005b
:020000040000fa
:10b004000600fa00200798002e029000245d8800b4
:10b014002e0090002200070003003700000000000b
:10b0240001003700000000000002eb001407980044
:10b034000e82e800840078002e009000380107009a
:10b0440000027800040f78001e027800e00f52001e
:10b05400f2ff3200b1af2c002e0090000107070070
:10b064001e027800940290001e0290008400780072
:10b074002e0090000500010000027800e20f42005b
:10b08400e8ff3a008000eb002e009000b5010700b5
:10b094002e00900067d907000080fa000000060027
:10b0a4000200fa00000f7800e1af2c001e007800c7
:10b0b400ec06070001b22c001e007800e906070028
:10b0c400a1b32c001e007800e606070071b52c0021
:10b0d4001e007800e306070051b72c001e0078001c
:10b0e400e006070051b92c001e007800dd060700b9
:10b0f400d1bb2c001e007800da06070071be2c00bc
:10b104001e007800d706070031c02c001e0078000e
:10b11400d406070021c22c001e007800d1060700c7
:10b1240041c42c001e007800ce06070021c62c0066
:10b134001e007800cb06070011c82c001e00780002
:10b14400c8060700d1cb2c001e007800c5060700f6
:10b1540011cf2c001e007800c206070031d22c004b
:10b164001e007800bf06070091d42c001e00780052
:10b17400bc06070031d82c001e007800b906070071
:10b18400d1d92c001e007800b60607000002eb009f
:10b19400040078000080fa00000006000e00fa00a7
:10b1a4004007980051079800620798004e029000eb
:10b1b400040f78005e029000140798006e0290005d
:10b1c400340798006e029000e00f52000c003c001f
:10b1d4000002eb002c0037004e429000e04f52007a
:10b1e40002003a000002eb00270037001e0fe800bf
:10b1f4001e0290000402e8001407980001003700c2
:10b204000000000014c0b300be029000e08f5200a2
:10b2140001003c000042eb00be0290008502e90000
:10b2240035079800e04f5200120032001e027800e9
:10b23400144278000402fb000400780023de0700b7
:10b2440000027800444798001e02900014427800df
:10b254000402fb00040078001cde070000027800f2
:10b2640054479800ce4290005e42900084cf520032
:10b27400d9ff32004e4290008402fb005e429000ef
:10b284000402fb0004825200040078000080fa00eb
:10b29400000006000800fa00200798003107980013
:10b2a4000002eb00040f78000002eb001407980082
:10b2b4000f0037001e0278006a22b90004027800e9
:10b2c400040f78002e029000144278000402fb0060
:10b2d4001e02420005fd2f00050f4200140020004d
:10b2e400140798002e0290000402e8002407980036
:10b2f4002e029000144278000402fb000403b10003
:10b30400e90f5200ebff36001e029000e00f5200de
:10b31400020032003e0290001e0a78001e029000d5
:10b32400040078000080fa00000006000c00fa0017
:10b33400500798000002eb00040f780064ba200064
:10b34400140798002d0037001e02900014027800a4
:10b3540004007800c8df0700000278002407980082
:10b364001e029000140278002e01900084007800e0
:10b374000080200089ff070000027800e00f5200df
:10b384001a003a001e02900024029000e00f5200be
:10b3940002003a001e0290001c003700ae0290002a
:10b3a4000480200004824200e802470085007800ff
:10b3b40004007800b7ff0700000278003407980003
:10b3c4003e029000e00f5200060034005e0290003e
:10b3d400e00f520003003200ce0290005e029000a3
:10b3e400050a78001e029000080037001e0fe800ce
:10b3f4001e0290006a024200140798001e027800a0
:10b40400f30f5200d0ff36000002eb000400780076
:10b414000080fa00000006000600fa00000f780021
:10b4240011079800220798001e0290002402900041
:10b43400e00f520002003a001e0290001f00370085
:10b444002e029000e00f520002003a000002eb00ce
:10b454001a0037002e029000940278001e02900019
:10b4640034029000848f5200080039002e029000ac
:10b47400940278001e02900044029000848f5200cf
:10b4840002003e001e0290000c0037002e029000c5
:10b4940014027800841f780004dc2c00841f7800d8
:10b4a4000090200085e00700e48757000190200009
:10b4b4001e007800eb0507000002eb000400780092
:10b4c4000080fa00000006000400fa00100798004b
:10b4d40014002000040f78000a0037001e0fe80053
:10b4e4009e029000a4002000809fbe00110009006d
:10b4f4008482d80000027800810278004f00be00e8
:10b50400140798001e029000e90f5200f3ff3e005a
:10b514001e027800040078000080fa000000060093
:10b524000e00fa00500798006107980061dd2c00b6
:10b534005e009000cb050700021020008000eb00a5
:10b544000080200045df07000002eb00040f7800b4
:10b554000480200014079800630037001e02900046
:10b56400840078005e0090007605070000027800f1
:10b57400e00f52005c0032001e029000144278007a
:10b58400844078005e0090008b0507001e02900046
:10b5940014427800ea4f5200040032001e02900068
:10b5a40014427800ed4f520012003a009e029000bf
:10b5b4000042eb00844a78006e0090005bff0700b5
:10b5c40000027800240798002e029000e00f520039
:10b5d40002003a000002eb00480037006e019000c0
:10b5e400ae0090005e0090008bff07000002780020
:10b5f400420037001e0fe8001e0290000402e8001b
:10b60400140798009e0290000042eb00844a7800e0
:10b614006e00900045ff07000002780024079800a0
:10b624002e029000e00f52002f0032002e029000f4
:10b6340024029000e00f520002003a002e02900013
:10b644002e0037002e0290001402780004007800c7
:10b6540009df070000027800340798002e029000ea
:10b66400440290000400780097ff0700000278006d
:10b6740044079800be0290004e02900004824200eb
:10b684009e0f520006003c006e019000ae00900038
:10b694005e00900060ff070000027800170037008a
:10b6a4002e02900044029000f30f52000e003e0060
:10b6b4003e0290000402e8009e0f52000a003c0083
:10b6c4006e02900014027800e10f5200060036006a
:10b6d4006e019000ae0090005e0090004eff0700e7
:10b6e40000027800050037009e027800e40f200075
:10b6f400848f520099ff36000002eb0004007800aa
:10b704000080fa00000006000400fa0004508000e3
:10b71400e00f520002003c000002eb000e00370074
:10b7240068025700040f78009e0178004eb9970014
:10b734000110200000902000c7df070000027800fd
:10b7440014079800245d8000019020000400780014
:10b75400440507001e029000040078000080fa00ef
:10b76400000006000400fa00000f7800110798009a
:10b774001e029000045088000002eb0004007800d0
:10b784000080fa00000006000000fa000450800067
:10b79400040078000080fa00000006000000fa00af
:10b7a400e4ff2f00040078000080fa000000060087
:10b7b4000400fa00000f7800110798001e029000a0
:10b7c400841f780094de2c00841f780000902000f1
:10b7d400badf0700e4875700019020001e007800bc
:10b7e400200507001e0290001100200004007800cc
:10b7f400611307000002eb00040078000080fa00e7
:10b80400000006000400fa00000f780011079800f9
:10b814001e029000841f7800f4df2c00841f78003f
:10b8240000902000a5df0700e48757000190200066
:10b834001e0078000b0507001e0290008000eb003c
:10b84400040078004c1307000002eb0004007800a9
:10b854000080fa00000006000400fa00000f7800df
:10b86400110798001e029000841f780064e12c00e8
:10b87400841f78000090200090df0700e4875700c1
:10b88400019020001e007800f60407001e029000bc
:10b894001100200004007800651307000002eb008b
:10b8a400040078000080fa00000006000400fa009a
:10b8b400000f7800110798001e029000841f780082
:10b8c40014e32c00841f7800009020007bdf070025
:10b8d400e4875700019020001e007800e10407006f
:10b8e4001e0290008000eb00040078005013070053
:10b8f4000002eb00040078000080fa00000006005b
:10b904000400fa00000f7800110798001e0290004e
:10b91400841f7800d4e42c00841f78000090200059
:10b9240066df0700e4875700019020001e007800be
:10b93400cc0407001e0290001100200004007800cf
:10b94400e01207000002eb00040078000080fa0017
:10b95400000006000400fa00000f780011079800a8
:10b964001e029000841f780014e62c00841f7800c7
:10b974000090200051df0700e48757000190200069
:10b984001e007800b70407001e0290008000eb0040
:10b9940004007800cb1207000002eb0004007800da
:10b9a4000080fa00000006000c00fa00889fbe0028
:10b9b4008a1f7800300798004107980052079800c2
:10b9c4004e0290006c22b90084027800e4c6200084
:10b9d400048f42005e029000050020000400be00b7
:10b9e400f0dc07000002be00020020000304240073
:10b9f4000400be002bdd07000002be000200200090
:10ba0400037824000400be0095dc07000002be0099
:10ba140014079800250798004e029000ed0f52007d
:10ba24004c003a0082eb210053fd23001e009000dd
:10ba3400ae0090001bdd07000002be001407980052
:10ba4400250798001e02780014059000f251280082
:10ba5400b3012c001e009000ae00900011dd070021
:10ba64000002be001e019000ae0190000400be0062
:10ba74000cdd07000002be001e019000ae01900024
:10ba84000400be0007dd07000002be000404be007f
:10ba940002002000031a24001e009000ae00900053
:10baa40000dd07000002be001e019000ae01900000
:10bab4000400be00fbdc07000002be000401be005f
:10bac4000800be0009dc07000002be000404be003a
:10bad40082142600432924001e009000ae0090002a
:10bae400f0dc07000002be000401be000800be0036
:10baf400fddb07000002be00723d2a00632f240014
:10bb04000400be00f9db07000002be001e0378003b
:10bb1400160378008a1f7800849fbe001e029000de
:10bb2400ae029000849fbe005e029000841f7800e5
:10bb3400861f78004e029000841f780064e72c0072
:10bb4400841f780000902000dcde0700f287570095
:10bb5400230037001e027800140490001e027800af
:10bb6400b4029000240290001e019000ae019000e7
:10bb74000400be00cbdc07000002be000403be00cc
:10bb84001e027800d4029000440290000401be001a
:10bb94000600be00d5db07000002be001e037800cd
:10bba40016037800881f7800849fbe001e02900050
:10bbb400ae029000849fbe005e029000841f780055
:10bbc400861f78004e029000841f780064e72c00e2
:10bbd400841f780000902000b8de0700f287570029
:10bbe400019020003e0090001e0407004f057800dd
:10bbf4004f04be000080fa00000006000600fa00b0
:10bc040010079800210798002e029000ee0f5200b2
:10bc14000400360081ea2c001e0090001104070085
:10bc24000f0037002e0290000402b0001100200023
:10bc340004007800980a07002e0290000402b00065
:10bc440004007800040b070000027800040f780059
:10bc54001e017800ae0090001e00900052ff070005
:10bc64000002eb00040078000080fa0000000600e7
:10bc74000400fa0010079800f100200000022000e0
:10bc8400850a07000002eb00040f78000a00370061
:10bc9400050220001e82420004007800ee0a07001c
:10bca40000027800040178009e0078001e009000d5
:10bcb4003dff07001e0fe8001e027800ee0f520041
:10bcc400f3ff36000002eb00040078000080fa0065
:10bcd400000006000600fa00200798000003200078
:10bce400dd0a070000027800040f7800100320002a
:10bcf400d90a070000027800140798001e02900079
:10bd0400841f78009e1f7800d4eb2c00841f7800d9
:10bd14000090200069de0700e687570001902000ac
:10bd24002e009000cf0307000002eb00040078000f
:10bd34000080fa00000006000600fa0010079800d0
:10bd4400210798001e0290004822de000442780079
:10bd5400044f78001e0290000442780014479800b3
:10bd640012002000ae0090000e007800e60a0700e2
:10bd740000027800040078000080fa000000060049
:10bd84000400fa00000f7800110798000103200056
:10bd94001e009000e8ff07001e029000841f780038
:10bda40074ed2c00841f78000090200043de07000f
:10bdb400e4875700019020001e007800a9030700c3
:10bdc4000002eb00040078000080fa000000060086
:10bdd4000400fa00000f78001107980011032000f6
:10bde4001e009000d4ff07001e029000841f7800fc
:10bdf400a4ee2c00841f7800009020002fde0700a2
:10be0400e4875700019020001e0078009503070086
:10be14000002eb00040078000080fa000000060035
:10be24000600fa002007980031120700000278008b
:10be3400140798001e029000841f7800c4ef2c00a1
:10be4400841f7800009020001cde0700e487570060
:10be5400019020002e009000820307001e02900033
:10be6400e00f520004003a0041f12c002e00900033
:10be74007c030700170037000002eb00040f780072
:10be8400110037001e02780015002000042add008e
:10be9400840278001e02900004826200e00f5200c7
:10bea400080032001e0278008402420024d22000de
:10beb4000482420014027800840078002e0090006e
:10bec400680307001e0fe8001e027800e50f520009
:10bed400ecff3600a1f12c002e0090006103070056
:10bee4000002eb00040078000080fa000000060065
:10bef4000400fa0010079800f00120000115070063
:10bf040000027800040f78009e1f7800e4f12c00f2
:10bf1400841f780000902000e8dd0700e4875700c4
:10bf2400019020001e0090004e0307000002eb0069
:10bf3400040078000080fa00000006000400fa0003
:10bf4400000f7800110798001e029000e50f5200c0
:10bf540005003600a1f32c001e0078004103070001
:10bf64000082eb00130037001e009000e00e070073
:10bf74001e02900084024200e4d2200004824200a7
:10bf840014027800841f78001e029000841f780039
:10bf940024f52c00841f780000902000c7dd0700e2
:10bfa400e6875700019020001e0078002d0307004b
:10bfb4000002eb00040078000080fa000000060094
:10bfc4000400fa00000f7800110798009e02900008
:10bfd400f40320000482620004007800090f0700c3
:10bfe4009e029000f403200004826200841f780003
:10bff40014f72c00841f780000902000afdd0700a8
:10c00400e4875700019020001e0078001503070004
:10c014000002eb00040078000080fa000000060033
:10c024000400fa00000f7800110798001e00900029
:10c0340025fd070000027800841f78001e0290008e
:10c04400841f7800e4f82c00841f780000902000fe
:10c054009add0700e6875700019020001e00780053
:10c06400000307000002eb00040078000080fa00df
:04c0740000000600c2
:020000040000fa
:10c07800e01000000e00000000000000fc100000ae
:10c0880002000000020000007e0e000042100000c6
:10c098002200000000000000f4100000040000006e
:10c0a80000000000f810000004000000000000007c
:10c0b8007a0e00000a010000000000006410000071
:10c0c8002200000000000000840f00004200000071
:10c0d8000200000002001100009a8a000400da0041
:10c0e80087030000006e100000546d000600f40085
:10c0f8006c170000d06e010000c67f000500ac0080
:10c10800800f00004681020000f686000000000053
:10c118000000000000000000000000000000000017
:10c12800000000000000000000000000c410000033
:10c138001c00000002000000e803010000b6cf0068
:10c14800dacffb00cf0ed00028d04500d061d00058
:10c158007fd0a500d0000000000000000000000013
:10c168003a0d00004001000000000000020a000033
:10c17800a201000000000000ee1000000600000010
:10c1880000000000c60f0000400000000200000090
:10c198000a000a0000000000000000000001000082
:10c1a8000000020000000000030002000000000080
:10c1b800020001000003000000000300000100006d
:10c1c8000100000000010000010001000002000061
:10c1d8000100030000010000040001000005000048
:10c1e8000100060000000000061000003c000000ee
:10c1f800000000008610000020000000020000007f
:10c208000a006400000a00000a0004000008000098
:10c218001000200000400000800001000002000023
:10c22800040008000010000020000000a610000014
:10c238001e000000000000000008000002020000cc
:10c2480000000000a40b000096010000020000009e
:10c2580003009200c9da5b0001000100000200003f
:10c2680096c904005c01000001000200009bc9009f
:10c278002e5c01000001000002009e00c9585c000d
:10c288000100010000020000a2c982005c01000058
:10c298000100020000a6c900ac5c0100000100001a
:10c2a8000200ab00c93a5e00000000000000000078
:10c2b800aec900005e01000000000f0000b1c90017
:10c2c800c25e0100000100006300b400c9ea5e001c
:10c2d8000100010000630000b7c96c005e000000a7
:10c2e8000000000000bac900125f00000000000052
:10c2f8000000bd00c9a05f000100000000050000ab
:10c30800c0c9e2005f01000000003f0000c3c9008f
:10c318007a5f0000000000000000c500c9b45b009f
:10c328000100000000090000c7c9520058000000c1
:10c338000000000000c9c900d05b00000000000038
:10c348000000cb00c9d05b00000000000000000026
:10c35800cdc91200600100000100fa0000d2c90036
:10c36800dec9ec00510542000000000000e4c900ed
:10c37800dec9ec00510542000000000000f0c900d1
:10c38800dec9ec00510542000000000000fcc900b5
:10c39800dec9ec0051054200000000000005ca009b
:10c3a80010caa40070854000000000000015ca00f3
:10c3b80020ca000000a04100000000000026ca00ba
:10c3c80010caa40070854000000000000031ca00b7
:10c3d80020ca000000a0410000000000003cca0084
:10c3e80010ca7b00148e3f00000000000045ca0000
:10c3f80020ca00000020410000000000004eca00d2
:10c4080010ca7b00148e3f00000000000058ca00cc
:10c4180020ca9a0099993f00000000000062ca00f3
:10c428006acae1007a474200cdcc1600c26eca0043
:10c43800dec9000000164200cdcc1600c277ca0043
:10c4480081ca0000c026440000007a00c487ca00e0
:10c458008eca9500ca9eca00a7cab500cac3ca0038
:10c46800cacad500cadcca00e7caef00ca00000081
:10c478009e1300003e000000020000002c20660011
:10c48800756e630074696f006e3a200000006100e9
:10c4980073736500727469006f6e20002225730043
:10c4a8002220660061696c0065643a0020666900b4
:10c4b8006c65200022257300222c20006c696e0018
:10c4c800652025006425730025730a00000000001c
:10c4d800561400000c000000000000006214000068
:10c4e80006000000000000003014000026000000d4
:10c4f800020000006314000000631400090000003b
:10c508000002000065140000006514000e0201001e
:10c518000000000000000000000000000602020009
:10c528000000000030140000681400000200000041
:10c5380000000000dc1300002a00000002000000d8
:10c548003031320033343500363738003941420053
:10c55800434445004600300031323300343536005c
:10c5680037383900616263006465660000286e0030
:10c57800756c6c00290000005e120000a00000002d
:10c5880002000000010000000000000000000a0096
:10c59800000000000000000000640000000000002f
:10c5a80000000000e8030000000000000000100088
:10c5b800270000000000000000a086000100000025
:10c5c8000000000040420f00000000000000800052
:10c5d80096980000000000000000e100f50500004a
:10c5e8000000000000ca9a003b00000000000000a4
:10c5f800e40b5400020000000000e8007648170031
:10c60800000000000010a500d4e8000000000000b1
:10c61800a0724e0018090000000040007a10f300d4
:10c628005a0000000080c600a47e8d0003000000b0
:10c6380000c16f00f2862300000000008a5d7800c8
:10c648004563010000006400a7b3b600e00d0000d8
:10c6580000e889000423c7008a00000006140000cf
:10c668002a00000002000000303132003334350067
:10c67800363738003941420043444500460030000f
:10c68800313233003435360037383900616263009f
:10c698006465660000286e00756c6c002900000057
:10c6a800fe120000a00000000200000001000000cf
:10c6b8000000000000000a00000000000000000068
:10c6c800006400000000000000000000e803000013
:10c6d800000000000000100027000000000000001b
:10c6e80000a08600010000000000000040420f008a
:10c6f8000000000000008000969800000000000084
:10c708000000e100f50500000000000000ca9a00e2
:10c718003b00000000000000e40b54000200000091
:10c728000000e80076481700000000000010a5008f
:10c73800d4e8000000000000a0724e0018090000b4
:10c74800000040007a10f3005a0000000080c60084
:10c75800a47e8d000300000000c16f00f286230054
:10c76800000000008a5d7800456301000000640055
:10c77800a7b3b600e00d000000e889000423c70055
:10c788008a000000fe1000006001000002000000a6
:10c798000000000000000000f03f00000000000062
:10c7a8000000240040000000000000000059400084
:10c7b80000000000000040008f4000000000000062
:10c7c8000088c30040000000000000006af8400034
:10c7d80000000000008084002e41000000000000de
:10c7e800d01263004100000000008400d797410088
:10c7f800000000000065cd00cd41000000002000d1
:10c808005fa002004200000000801d00af15440038
:10c818000000000040593e002946000000000000ca
:10c828000000f0007f0000000000000000f07f0022
:10c838000000000000000000f07f00000000000081
:10c848000000f0007f0000000000000000f07f0002
:10c858000000000000000000f07f00000000000061
:10c868000000f0007f0000000000000000f07f00e2
:10c878000000000000000000f07f00000000000041
:10c888000000f0003f00000000a0990099b93f00a7
:10c898000000000040e17a00843f00000000e00052
:10c8a8004d6250003f00000000e0e200361a3f00f1
:10c8b8000000000080b5f800e43e00000000a00081
:10c8c800f7c6b0003e00000000a0f200d77a3e0094
:10c8d80000000000e08e7900453e00000000e00006
:10c8e8000b2e11003e00000000e0df007cdb3d0065
:10c8f8000000000000a19c00c73b000000000000f1
:10c908004c48b40039000000000020006ca137003a
:10c91800000000000000000000000000000000000f
:10c9280000000000000000000000000000000000ff
:10c9380000000000000000000000000000000000ef
:10c9480000000000000000000000000000000000df
:10c9580000000000000000000000000000000000cf
:10c9680000000000000000006a140000020000003f
:10c97800000000006c14000002000000000000002d
:10c988006e14000002000000000000007014000097
:10c998000200000002000000010000007214000004
:0cc9a80002000000000000000000000081
:020000040000fa
:10c9b4000200fa000002eb00040f780022003700a6
:10c9c400a5a120001e0278004722dd0084824200d7
:10c9d4001e0278004323dd0024a02000040243004b
:10c9e400050a78001e027800c322dd0044a020005e
:10c9f400048242008002eb00050a78001e027800df
:10ca0400c322dd0064a02000048242008002eb0007
:10ca1400050a78001e027800c322dd0084a02000ed
:10ca240004824200f5072000050a78001e027800ff
:10ca340084024200a4b92000048242008002eb0078
:10ca4400050a78001e0fe8001e027800e20f52006b
:10ca5400dbff340000582200010020007a010700a7
:10ca640000027800c412880051e2a80050a2a90074
:10ca74005062a900841280000410a1000420a100c7
:10ca8400841288005002a9000440200094128800f7
:10ca94008e40a9008e60a900640680000480a10075
:10caa4000490a00004a0a00064068800640680002e
:10cab40004c0a10004d0a00004e0a1006406880022
:10cac4009e40a8009e60a90000582200010020009a
:10cad4005d01070000027800c411880031e2a8005b
:10cae40030a2a9003062a900841180000410a100c2
:10caf4000420a100841188003002a9000440200011
:10cb04009411880087c0a90087e0a90094058000db
:10cb14000480a1000490a00004a0a0009405880053
:10cb24009405800004c0a10004d0a00004e0a1008a
:10cb34009405880097c0a80097e0a9000080fa0037
:10cb4400000006000600fa0010079800210798006c
:10cb54001e0090002101070000027800e00f52003f
:10cb64000e003200ddd407001e0290000402e9002a
:10cb7400c322dd0024a02000048242008400780047
:10cb84002e0090004010070000027800040f780087
:10cb9400dfd407001e02780004003700ae029000c4
:10cba4000042eb00844a78000002eb0004007800a5
:10cbb4000080fa00000006000600fa001007980042
:10cbc400414798000002eb00040f78001d00370075
:10cbd4001e029000e20f52000c003200e30f5200dc
:10cbe40017003a009512800004202000048262009d
:10cbf400e00f52000f003a004e4290000482fb0006
:10cc0400a41288001400200013003700951180003e
:10cc14000420200004826200e00f520007003a0062
:10cc24004e4290000482fb00a411880014002000ee
:10cc34000900370000000000010037000000000078
:10cc44001e0fe800743e20009e027800848f52007c
:10cc5400dfff34000002eb00040078000080fa00db
:10cc6400000006000600fa0010079800210798004b
:10cc74000002eb00040f78000b0037001e0278005e
:10cc8400ae0290000482420014427800844078008e
:10cc94001e009000c8ff070000027800e00f520059
:10cca400010032001e0fe8001e027800ae02900060
:10ccb4000482420014427800e04f5200efff3a0031
:10ccc4000002eb00040078000080fa000000060077
:10ccd4000600fa00000f7800110798002207980058
:10cce4009e0090001e007800deff07002e029000d8
:10ccf400e00f520002003200647f2d000100370073
:10cd0400b47f2d00840078001e007800d5ff070052
:10cd14000002eb00040078000080fa000000060026
:10cd24000400fa00100798001e009000ab000700f2
:10cd340000027800e00f52001100320067d40700af
:10cd44001e0290000402e900c322dd0024a020009a
:10cd540004824200040078000810070000027800f2
:10cd6400040f78006ad407001e02780004f0a700bc
:10cd74000402ea000402e9004f22de000100370049
:10cd84000002eb00040078000080fa0000000600b6
:10cd94000400fa00100798001e0090008f0007009e
:10cda40000027800e00f52000d0032004bd407005f
:10cdb4001e0290000402e900c322dd0024a020002a
:10cdc4000482420004007800da0f070000027800b1
:10cdd400040f78004ed407001e02780001003700cb
:10cde4000002eb00040078000080fa000000060056
:10cdf4000400fa00100798001e029000e20f52008f
:10ce040003003200e30f5200070032000c00370029
:10ce1400941180004922de00614262000482fb001a
:10ce2400040f780008003700941280004922de00c5
:10ce3400614262000482fb00040f780002003700a4
:10ce440014002000040f78001e027800040078000b
:10ce54000080fa00000006000200fa00000f7800cb
:10ce64001e0078005d00070000027800e00f520009
:10ce7400060032001e02780084024200a4b9200099
:10ce84000482420014027800010037000002eb0023
:10ce9400040078000080fa00000006000200fa0096
:10cea400000f78001e0078004c0007000002780094
:10ceb400e00f5200060032001e0278008402420095
:10cec400a4b92000048242008002eb00050a780025
:10ced4000080fa00000006000400fa001007980021
:10cee4001e0090003d00070000027800e00f520091
:10cef40023003200f9d307001e0290000402e90067
:10cf0400c322dd0024a02000048242000400780033
:10cf14007e0f07001e029000e20f5200060032004e
:10cf2400e30f52000d00320012003700b4118000ec
:10cf3400040f780001003700000000009411800005
:10cf440061026200e00f5200f8ff3a000900370066
:10cf5400b4128000040f78000100370000000000c4
:10cf64009412800061026200e00f5200f8ff3a0060
:10cf740000000000e6d307000000000001003700b5
:10cf8400000000000080fa00000006000200fa0021
:10cf9400000f78001e027800e20f520003003200f6
:10cfa400e30f5200060032000a0037003342a900a2
:10cfb400000000003342a800000000000500370014
:10cfc4005342a900000000005342a80000000000e2
:10cfd400000000000080fa00000006000200fa00d1
:10cfe400000f78001e027800e30f520003003200a5
:10cff4001e027800e20f520002003a0014002000e2
:10d00400010037000002eb00040078000080fa0001
:10d01400000006000200fa00000f78001e02e8007b
:10d024004422dd00050020000401be0000002200af
:10d03400c10120004cd707000002be000400be005e
:10d044000080fa00000006000400fa00008fbe0011
:10d054001e02be00e00f5200e08f5a0002003a00a8
:10d064000082eb000f00370004202c001500200084
:10d074001e03be00840f5300858f5b000200360040
:10d084000002eb00070037001e01be0000202c0048
:10d0940011002000b7d707000002be000402780088
:10d0a4000402e900040078000080fa000000060091
:10d0b400849fbe000000fa00045d8000155d8000be
:10d0c40061024200e0824a00045d8800155d880028
:10d0d40087e0a9000080fa004f02be00004006006d
:10d0e400849fbe000000fa001500370064508000e1
:10d0f4008402e800845080008482620074508000be
:10d10400848f520003003a0014002000e45c88007d
:10d114000b00370055508000645080008482420028
:10d12400b411800004427800844a7800645080007e
:10d134008402e80084508000048262006450880005
:10d144009411800061026200e00f5200e7ff3a0090
:10d1540087c0a9000080fa004f02be00004006000c
:10d16400849fbe000000fa00045d8000155d80000d
:10d1740061024200e0824a00045d8800155d880077
:10d184008e60a9000080fa004f02be000040060035
:10d19400849fbe000000fa0015003700a4508000f0
:10d1a4008402e800c450800084826200b45080008d
:10d1b400848f520003003a0014002000f45c8800bd
:10d1c4000b00370095508000a450800084824200f8
:10d1d400b412800004427800844a7800a45080008d
:10d1e4008402e800c450800004826200a4508800d5
:10d1f4009412800061026200e00f5200e7ff3a00df
:10d204008e40a9000080fa004f02be0000400600d4
:10d214000a00fa0020479800314798002207980036
:10d2240033079800440798000002eb00040f7800cd
:10d234002ad30700a4c0b30004007800edf0b700bf
:10d244004e02900071c0b3002e019000be01900008
:10d254003e4090006ed2070000027800e10f5200b9
:10d264000300320034002000040f78000700370068
:10d2740000e22400ee10070000027800e10f5200e3
:10d284000200320034002000040f780020d307008d
:10d294001e027800040078000080fa0000000600f6
:10d2a4000000fa000dd307008000eb0010002000fe
:10d2b40048d207000002eb001487880014d307004b
:10d2c4000000eb000a1107000080fa0000000600cd
:10d2d4000000fa0001d307008000eb000000eb001f
:10d2e4003cd20700e410070009d307000080fa00cd
:10d2f400000006000800fa001007980021079800b3
:10d30400320798000002eb00040f7800f3d2070004
:10d3140025878000f40f2000848f5200050036001a
:10d324008001eb00e26a2d00316d2d00d009200050
:10d33400aed7070024878000e20f520015003600a4
:10d3440025878000e4878000850078000400780049
:10d354008601070000427800e04f52000d003a00b9
:10d36400e4878000144278009e029000844a78008a
:10d37400248780008482e9003e029000050a780038
:10d38400e48780008402e8002e029000050a7800f9
:10d394000200370054002000040f7800dcd207009c
:10d3a4001e027800040078000080fa0000000600e5
:10d3b4000a00fa0040479800310798004207980095
:10d3c4000002eb00040f7800c4d207001487800029
:10d3d400e00f520020003a003e0290000402e900ef
:10d3e4004487880014002000548788004487800004
:10d3f400ce429000054a7800558780004e02900086
:10d404000482420054878800558780004487800046
:10d414008500780004007800540107000042780079
:10d4240024479800e5878000548780008482420066
:10d434002e439000864a78000402e800548788004e
:10d444001400200004878800110020000000eb0075
:10d45400e0d107000200370054002000040f7800d8
:10d46400abd207001e027800040078000080fa00a6
:10d47400000006000400fa000002eb00040f78002c
:10d4840004878000e00f5200050032008001eb00a9
:10d49400026f2d00316d2d00400e200053d7070080
:10d4a40063024700040078003ad207001487800022
:10d4b400e10f520005003200e10f52005c00390018
:10d4c400e20f52003e00320066003700641007008d
:10d4d400be429000a4c3b30084cf520005003a00ba
:10d4e4000002eb00348788000002eb0024878800e8
:10d4f4005c0037003e429000ed4f520003003a00ba
:10d504002400200014878800560037003e42900013
:10d5140004407800e00007000042780024479800a7
:10d5240034878000e00f520003003200e10f520004
:10d53400130032004b00370025878000f40f2000d1
:10d54400848f52000a003e00e58780002487800013
:10d55400848242002e429000460020000622dd0014
:10d56400844a7800140020003487880013003700b0
:10d574000002eb00148788003f1007000f003700fb
:10d58400e5878000268780000602780084834200b5
:10d59400e587800004824200944278002e42900085
:10d5a40004c27200844b78000602e80024878800d5
:10d5b4000002eb00348788000000000029003700d7
:10d5c400be429000d40e21001442780084cf520051
:10d5d40008003a00281007000002eb0014878800b6
:10d5e400100020004210070000027800040f7800a9
:10d5f4001c003700be429000a4c3b30084cf520085
:10d6040008003a000002eb00348788000002eb00b7
:10d614002487880014002000148788001010070055
:10d62400100037000002eb00148788000d0037005b
:10d63400be429000a4c3b30084cf520008003a0055
:10d64400071007000002eb00248788000002eb00ab
:10d6540034878800140020001487880001003700f4
:10d66400000000001e027800040078000080fa0028
:10d67400000006000400fa000002eb00040f78002a
:10d6840014878000e00f5200050032008001eb0097
:10d69400b2702d00316d2d00f0142000d3d6070098
:10d6a40004878000050020004600200007002000b9
:10d6b400860f5200878f5a0058003e000460010014
:10d6c40052003700030037000c0037003c003700dd
:10d6d40042003700a4c3b300244798002e429000b0
:10d6e40004407800a3d107002400200004878800a8
:10d6f4000002eb003487880048003700548780001c
:10d70400e00f52002900320034878000e00f5200fd
:10d7140003003200e10f5200100032003f003700d6
:10d7240044878000144278000482fb004422de0017
:10d734000442780004407800730007000042780037
:10d74400244798002e4290000440780089d10700b5
:10d7540014002000348788001300370044878000b9
:10d76400144278006f4262000440780066000700ab
:10d7740000427800244798002e429000044078002c
:10d784007cd10700448780000402e80044878800b5
:10d794000002eb0034878800548780000402e9000b
:10d7a40054878800000000001c003700d0c0b3007c
:10d7b40070d1070034002000048788001700370068
:10d7c400d40e2100144278000440780069d1070087
:10d7d4004400200004878800100037000002eb009a
:10d7e4000487880030002000c10f07000002780081
:10d7f400040f78008000eb0010002000f5d0070033
:10d804000002eb0004878800040037008000eb006e
:10d8140010002000efd00700000000001e02780076
:10d82400040078000080fa00000006000000fa00fe
:10d83400148780000402e900e10f520003003e0057
:10d844000002eb00148788000e0037001487800064
:10d85400e10f52000800320014878000e20f5200ea
:10d86400070032008001eb0062722d00316d2d0043
:10d87400701a20005dd60700000000000100370088
:10d88400000000007c0f07000002eb000400780099
:10d894000080fa00000006000200fa00004f780041
:10d8a400f4c2b3009e42780084cf520007003600d1
:10d8b40094c3b3009e42780084cf520003003e001c
:10d8c40004cdb3001e4242000c00370004c4b30070
:10d8d4009e42780084cf52000700360064c4b3002f
:10d8e4009e42780084cf520003003e0094ccb300e3
:10d8f4001e4242000100370000c2eb0004407800e1
:10d904000080fa00000006000200fa00004f7800d0
:10d914001e427800e94f520003003e0005c3b300e5
:10d924001ec242000e0037001e427800e94f52002a
:10d93400060036001e427800ef4f520003003e00fe
:10d9440075c3b3001ec24200050037008001eb001e
:10d95400a2762d00316d2d00001d200023d6070076
:10d96400044078000080fa00000006000600fa0077
:10d9740010079800210798000042eb00044f78003c
:10d98400060037001e029000144278001e4f420029
:10d994001e0290000402e800140798002e02900072
:10d9a40004f0a7000402ea000402ea004f22de00a9
:10d9b40004427800ae0290008502e9002507980031
:10d9c400e04f5200efff3a001e4278000442ea00a2
:10d9d400044f78001e427800044078000080fa006a
:10d9e400000006000a00fa0030079800410798007a
:10d9f4000002eb00040f78004e029000140278003d
:10da0400e50f520021003a003e0290000402e800b3
:10da1400144278000482fb004822dd0014079800b9
:10da24003e0290000482e800144278000482fb0065
:10da34009e02900004827200140798001e02900057
:10da44000402e800140798003e02900063024200ba
:10da540013002000120020009e00900004007800b3
:10da64006ccb070000027800240798002e02900077
:10da7400e00f5200070032002e0090004c0c07000b
:10da840000027800040f7800020037003400200000
:10da9400040f78001e027800040078000080fa0069
:10daa400000006000e00fa00500798006107980075
:10dab4000002eb00040f78006e029000140278005c
:10dac400e50f5200470036005e0290000402e800b1
:10dad400144278000482fb004822dd0014079800f9
:10dae4005e0290000482e800144278000482fb0085
:10daf4009e02900004827200140798001e02900097
:10db04000402e800140798005e02900063024200d9
:10db1400144278000482fb004822dd0024079800a8
:10db24005e02900064024200144278000482fb000a
:10db3400ae02900004827200240798005e029000f6
:10db44006502420094427800654798002e029000d6
:10db5400e00f520020003200ae0290008407200043
:10db6400848f52001c003e002e0290000442780074
:10db740004424200844278006e42900084cf5200f6
:10db840015003a005e029000660242001300200075
:10db94002e0190009e009000040078001dcb070029
:10dba40000027800440798004e029000e00f5200f3
:10dbb400050032004e009000fd0b070000027800c3
:10dbc400040f7800090037006e0290005500200011
:10dbd400050a78000500370034002000040f78009f
:10dbe4000200370034002000040f78001e02780081
:10dbf400040078000080fa00000006000e00fa001d
:10dc040050079800610798000002eb00040f7800a9
:10dc14006e02900014027800e50f520059003a0099
:10dc24005e0290000402e800144278000482fb00c3
:10dc34004822dd00140798005e0290000482e80088
:10dc4400144278000482fb009e0290000482720059
:10dc5400140798001e0290000402e80014079800bc
:10dc64005e02900063024200144278000482fb00ca
:10dc74004822dd00240798005e02900064024200fe
:10dc8400144278000482fb00240798002e029000be
:10dc9400e00f520038003200ae029000d40720009a
:10dca400848f520034003e005e02900034079800d6
:10dcb4006e0290008002eb00050a7800be0290001c
:10dcc40034c0b300844a78003e0290000402e800a5
:10dcd400340798006e029000140278008402e80071
:10dce4006e029000050a78002e029000044278002b
:10dcf40004424200be029000844a78003e02900032
:10dd04000402e800340798006e02900014027800c0
:10dd14008402e8006e029000050a78008001eb009e
:10dd24002e0190009e0090003e009000b9ca0700aa
:10dd340000027800440798004e029000e00f520061
:10dd4400050032004e009000990b07000002780095
:10dd5400040f78000d0037006e02900094027800e2
:10dd64002e02900004024200848242006e0290005f
:10dd7400050a78000500370034002000040f7800fd
:10dd84000200370034002000040f78001e027800df
:10dd9400040078000080fa00000006001400fa0075
:10dda400000f9800110f98000002eb00040f780098
:10ddb4001e0a900014027800e90f52009700360002
:10ddc4000e0a90000402e800144278000482fb006a
:10ddd4004822dd00240798000e0a90000482e8001f
:10dde400144278000482fb00ae02900004827200a8
:10ddf400240798002e0290000402e80024079800eb
:10de04000e0a900063024200144278000482fb0070
:10de14004822dd00340798000e0a90006402420094
:10de2400144278000482fb00be0290000482720057
:10de3400340798000e0a90006502420014427800ec
:10de44000482fb004822dd00440798000e0a90007b
:10de540066024200144278000482fb00ce02900065
:10de640004827200440798004e0290000402e80005
:10de7400440798000e0a900067024200144278009a
:10de84000482fb004822dd00540798000e0a90002b
:10de940068024200144278000482fb00de02900013
:10dea40004827200540798000e0a9000690242002e
:10deb40094427800454f98003e029000e00f5200d3
:10dec40054003200be029000d4072000848f520018
:10ded40050003e005e029000e00f52004d00320000
:10dee400de02900094072000848f520049003e0017
:10def4005e02900004024200840278004e4a9000c0
:10df04000482fb00848f520042003a000e0a900003
:10df14006a024200130020005e019000ce009000cf
:10df2400040078003bca0700000278001407980038
:10df34001e029000e00f52002e003a000e0a9000dc
:10df4400740798001e0a90008002eb00050a78000e
:10df5400fe02900074c1b300844a78007e029000ef
:10df64000402e800740798001e0a90001402780066
:10df74008402e8001e0a9000050a78003e02900020
:10df84000442780004424200fe029000844a780071
:10df94007e0290000402e800740798001e0a9000b4
:10dfa400140278008402e8001e0a9000050a780032
:10dfb4008001eb003e019000ae0090007e009000d6
:10dfc40014ca070000027800140798001e0290008b
:10dfd400e00f520007003a001e0a900094027800f5
:10dfe4003e02900004024200848242001e0a900015
:10dff400050a78001e029000e00f5200070032006c
:10e004001e009000ea0a070000027800040f78005e
:10e014000200370034002000040f78001e0278004c
:10e02400040078000080fa00000006000c00fa00ea
:10e034001007980041479800524798003407980009
:10e0440045079800530798000002eb00040f78007e
:10e054004e429000e04f5200060032004e429000c3
:10e06400e04f5200030032004e429000e94f42005c
:10e074000300360024002000040f78004e0037000f
:10e084004e40900064f0b7001e029000e00f520072
:10e0940003003200e10f52001c003200360037004a
:10e0a4004468270054838800a46927006483880097
:10e0b400e470270044838800c46a270074838800be
:10e0c4000002eb008483880044782700948388004e
:10e0d40024802700a483880044862700b483880012
:10e0e40045062100954278005e0290003e019000b2
:10e0f400ce019000de40900005407800c802070081
:10e1040000027800040f78001d00370024952600d3
:10e1140054838800a496260064838800a49d260066
:10e1240044838800c4972600748388000002eb00af
:10e1340084838800c4a3260094838800c4b3260083
:10e14400a483880084c12600b48388004506210086
:10e15400954278005e0290003e019000ce0190004e
:10e16400de4090000540780029fc0700000278009a
:10e17400040f78000200370024002000040f780008
:10e184001e027800e00f52000b003a00510d070008
:10e1940000027800e00f520003003a00340020002f
:10e1a400040f7800040037001e02900034838800b6
:10e1b40014002000247c88001e02780004007800eb
:10e1c4000080fa00000006000800fa0040479800aa
:10e1d400310798004e429000e04f52005400320044
:10e1e4004e429000e04f5200510035003bcf0700f3
:10e1f4003e029000e00f52002d0032000002eb00be
:10e20400040f78001f0037001e0278004222dd0050
:10e214008482e80064f8200004824200140278003a
:10e22400e00f5200090032001e0278004222dd0095
:10e234008482e80064f8200004824200940278009a
:10e244003e029000848f52000d003a001e027800b6
:10e25400c222dd0064f8200004824200ce42900015
:10e26400054a78001e027800c222dd0084f82000ee
:10e2740004824200be029000050a780004003700c0
:10e284001e0fe8001e027800ef0f5200deff34007c
:10e294001e027800f00f5200020032000002eb0070
:10e2a4000100370044002000140798001e003700c6
:10e2b4000002eb00040f7800160037001e027800fd
:10e2c400c222dd0064f820000482420094427800f7
:10e2d4004e42900084cf52000d003a001e02780096
:10e2e400c222dd0064f82000848242000042eb0078
:10e2f400844a78001e027800c222dd0084f82000df
:10e30400048242008002eb00050a78000400370012
:10e314001e0fe8001e027800ef0f5200e7ff3400e2
:10e324000002eb0014079800f9ce07000200370042
:10e3340024002000140798001e02900004007800b6
:10e344000080fa00000006000200fa000002eb0060
:10e35400040f7800247c8000e10f520006003a008c
:10e3640084838000e00f5200050032008483800023
:10e37400040001000200370064002000040f78004c
:10e384001e027800040078000080fa0000000600f5
:10e394000200fa000002eb00040f7800247c8000e5
:10e3a400e10f520005003a0054838000040001008c
:10e3b4000002eb00247c8800020037006400200087
:10e3c400040f78001e027800040078000080fa0030
:10e3d400000006000200fa00247c8000e00f5200d6
:10e3e40007003a0064838000040001001400200048
:10e3f400247c88000002eb00040f7800080037003a
:10e40400247c8000e10f520003003a000002eb007c
:10e41400040f78000200370064002000040f780025
:10e424001e027800040078000080fa000000060054
:10e434000600fa000002eb0014079800247c800018
:10e44400e00f520002003200640020008500370013
:10e454006402470004007800af0c07000002780053
:10e46400e10f52007e003a002e02900005002000c9
:10e474003600200007002000860f5200878f5a00c4
:10e4840077003e00046001006e0037000200370090
:10e49400180037006b0037007483800002082100e5
:10e4a400e1072100c00721000400010000027800f8
:10e4b400140798001e029000e00f520063003a0017
:10e4c400c5072100954278004406210014427800d3
:10e4d40084cf520004003200c407210014427800a3
:10e4e400e04f52005b003a0020002000800c07003f
:10e4f4005b003700f4838000144278000002fd00c2
:10e5040082f0b7000002fd0014002000248488007b
:10e514000002eb00040f78001e0037001e02780092
:10e52400c222dd0064f82000048242001442780014
:10e53400e04f52001b0032001e027800c222dd00b0
:10e5440064f82000048242009442780024082100e8
:10e554001442780084cf52000d003a001e02780065
:10e564004222dd008482e80064f820000482420034
:10e5740094027800f48380000108210004007800ec
:10e58400050001000002780024848800060037009a
:10e594001e0fe8001e027800ef0f5200dfff340068
:10e5a4000100370000000000c40721001442780075
:10e5b400e04f52002900320024848000e00f520012
:10e5c400140032000002eb0004848800f48380000d
:10e5d40006848000860342002508210095427800c5
:10e5e40004c8b30004c27200844b78000602e80039
:10e5f40004848800f48380000584800005034200bd
:10e604002484800004427800044b78000502e8006a
:10e61400048488004783800006848000f58380009a
:10e624004406210014427800060178008500780031
:10e6340004407800070001000002780014079800e5
:10e64400070037000000000005003700000000004c
:10e654000300370000000000010037000000000044
:10e664000002eb00040078000080fa0000000600bd
:10e674000000fa00dcc2a800dce2a800dd22a80049
:10e68400dd42a800f0e2a800f102a800f122a800ef
:10e694000080fa00000006001000fa00889fbe0007
:10e6a400600798007107980037f4070000027800ab
:10e6b400e00f5200080032007e029000841f7800b0
:10e6c4006e029000841f780044782d00841f780027
:10e6d4000df40700e6875700ee0290007e029000da
:10e6e40004824200ff0f520055003600ee029000f3
:10e6f400e4022000848f520053003e00c203200035
:10e704008000eb0060002100d4d207006e0290006c
:10e71400040f78000002eb00540798007e0290007a
:10e72400140798006e029000ff0f52000a003e008a
:10e7340004022000040f7800050220006e029000fd
:10e744000482520054079800fe0290005e0290007a
:10e7540004825200140798001e0290009e02420098
:10e76400f4022000848f520003003600f4022000db
:10e774001e0252001407980004fe2f001e0f4200d0
:10e784000002eb0024079800280037002e029000b6
:10e79400e00f520003003200447e80000400780041
:10e7a4005b0407001e027800340798000002eb00a7
:10e7b40044079800160037003e029000c222dd0094
:10e7c40064002100048242001404be003e00900054
:10e7d400ba00070000027800050020000802420089
:10e7e40089824a003e039000c233dd0066002100a6
:10e7f40006834300048bbe004e0290000402e8002e
:10e80400440798003e0290000402e8003407980090
:10e81400ce0290001e029000848f5200e6ff390061
:10e824002e0290000402e80024079800347e800041
:10e83400ae029000848f5200d4ff390003003700e9
:10e844000000000001003700000000004f04be007b
:10e854000080fa00000006000200fa00000f7800b1
:10e86400347e8000e00f520002003a000002eb0008
:10e87400220037001e027800ff0f520012003600fb
:10e88400e40220009e027800848f52000e003e00b5
:10e8940005fe2f001e824200c222dd00640021001a
:10e8a400048242001403be00347e80000500200070
:10e8b4000401be000600be00aed107000002be0087
:10e8c400040278000d003700040320009e02780043
:10e8d400848f520002003a00347e80000700370023
:10e8e400140320009e027800848f520002003a0034
:10e8f400447e8000010037000002eb000400780031
:10e904000080fa00000006000c00fa0030079800ae
:10e914004107980052079800347e8000140798003d
:10e92400447e80002407980031003700ce02900016
:10e93400f4022000848f520027003600ce0290009b
:10e9440014032000848f520023003e003e029000f6
:10e95400144278000482fb00040f78003e02900009
:10e964000402e800340798001e0278004822dd0003
:10e97400040f78003e029000144278000482fb00e9
:10e984001e0f42003e0290000402e8003407980083
:10e994001e027800e00f520002003a00140020002a
:10e9a400040f7800ce02900004032000848f5200ec
:10e9b40003003a001e02780014079800060037008e
:10e9c400ce02900014032000848f520002003a000b
:10e9d4001e027800240798005e0290000402e900f9
:10e9e400540798004e0290000402e800440798007f
:10e9f4005e029000e00f5200ccff3a009e029000ad
:10ea04002e02900004aab90084027800a40f20000a
:10ea1400848f520006003e001e029000347e88005f
:10ea24002e029000447e88000002eb0001003700b3
:10ea340024002000040078000080fa000000060092
:10ea44000200fa00000f78001e0278000500200082
:10ea54003600200007002000860f5200878f5a00de
:10ea64000d003e000460010003003700040037007d
:10ea74000500370006003700dcc2a9000600370095
:10ea8400dce2a90004003700dd22a90002003700ff
:10ea9400dd42a900000000000080fa00000006002a
:10eaa4000000fa00dcc2a800dce2a800dd22a80015
:10eab400dd42a8000080fa00000006000a00fa0007
:10eac400400798004e029000ef0f520002003600fb
:10ead4000002eb003e0037004e029000c222dd002f
:10eae400a4fc200004824200140f78004e0290001f
:10eaf4004222dd008482e800a4fc2000048242005b
:10eb040094027800150798001e027800e10f520065
:10eb140006003a001e02900084024200c4762d00d2
:10eb2400048242001402780005003700c5772d00e6
:10eb34001e02900004024200048242001402780083
:10eb440024079800d6ff07001e007800bcff0700ca
:10eb5400ae02900004702800048272000400780061
:10eb640014cd0700000278004922dd003407980024
:10eb74000000eb000fcd0700000278004722de0002
:10eb8400be0290000482720034079800c4ff07009c
:10eb9400fdf2070000027800e10f52000b0036007e
:10eba4001e029000841f78009e1f7800be02900011
:10ebb400851f78004e029000841f7800b4792d00e0
:10ebc400841f7800d0f20700ea8757003e029000c5
:10ebd400040078000080fa00000006000200fa0039
:10ebe400dce2a90000702b00f2cc070000027800e0
:10ebf4004922dd00040f78000000eb00edcc070093
:10ec0400000278004722de001e0f7200dce2a90039
:10ec14001e027800040078000080fa00000006005c
:10ec24000e00fa0060479800714798004207980068
:10ec340053079800640798000002eb00040f780063
:10ec4400a6cc07006e02900081c0b3004e01900074
:10ec5400de0190007e409000edcb070000027800ba
:10ec6400e10f52000300320034002000040f78004a
:10ec74001f0037004e039000de03900004b0240010
:10ec840005002000840f5300858f5b0005003600cb
:10ec9400340220000500200014079800250798007e
:10eca4000b0037004e029000de0290000402420086
:10ecb40085824a000401be0000fa27007101200089
:10ecc400acd007000002be00140798002507980086
:10ecd4001e02900004007800550a07000002780024
:10ece400e10f52000200320034002000040f7800cb
:10ecf40087cc07001e027800040078000080fa0028
:10ed0400000006000000fa0074cc07000002eb00cb
:10ed1400e47388008000eb0010002000adcb0700f6
:10ed24004f0a07007acc07000080fa0000000600b2
:10ed34000000fa0069cc07008000eb000000eb0043
:10ed4400a4cb07004c0a070071cc07000080fa002e
:10ed5400000006000a00fa00200798003107980016
:10ed6400420798000002eb00140798000002eb0031
:10ed7400040f780059cc0700157c8000f40f2000a4
:10ed8400848f5200050036008001eb00625d2d0087
:10ed9400b15f2d00200a200014d10700147c8000ec
:10eda400e30f520015003600147c800084007800c4
:10edb400e0e72000ef09070000027800e00f5200ae
:10edc4000e003a00e4e7200014427800ae029000fe
:10edd400844a7800147c8000e30252004e029000c2
:10ede400050a78003e029000f5e72000050a780045
:10edf400140020001407980002003700540020007b
:10ee0400040f780042cc07001e027800040078004a
:10ee14000080fa00000006000a00fa00404798004b
:10ee240031079800420798000002eb00040f7800b5
:10ee34002acc0700e4738000e10f52002a003a0054
:10ee44003e0290000402e900f47b880014002000d4
:10ee5400047c8800f47b8000ce429000054a780050
:10ee6400057c80004e02900004824200047c8800ed
:10ee7400057c8000f47b8000850078000400780025
:10ee8400bc0907000002780014079800057c800084
:10ee94001e02900004427800e6e720000683420048
:10eea400044b78000502e800047c8800057c80009f
:10eeb4001e0290004822de0004427800e6e72000ab
:10eec40006834200044b78000502e800047c8800b5
:10eed40014002000d4738800110020000000eb000f
:10eee4003ccb07000200370054002000040f7800d8
:10eef40007cc07001e027800040078000080fa00a6
:10ef0400000006000400fa000002eb00040f780081
:10ef1400d4738000e00f5200050032008001eb0042
:10ef240042612d00b15f2d00f00e2000afd007002c
:10ef34000e82e8000400780096cb0700e47380009a
:10ef4400050020003600200007002000860f520034
:10ef5400878f5a0026003e0004600100030037003a
:10ef6400060037001200370002003700bc09070012
:10ef74001f003700ba0907001d0037000002eb002c
:10ef8400147c8800157c80002e429000e6e7200067
:10ef940006834200044b78000502e800147c8800d4
:10efa40024002000e4738800ad0907001000370036
:10efb400157c8000f40f2000848f520008003e006e
:10efc400157c80002e429000e6e720000683420074
:10efd400044b78000502e800147c88000200370026
:10efe40034002000e47388009d090700000000003d
:10eff4001e027800040078000080fa000000060079
:10f004000200fa000002eb00040f7800e4738000b1
:10f01400e10f5200050032008001eb00f2622d0086
:10f02400b15f2d00a012200070d00700d4738000bf
:10f03400e00f520003003200e10f520005003200dd
:10f044001c0037008000eb0010002000e1ca07001c
:10f0540018003700047c8000e00f52000b003200df
:10f06400f47b8000144278000440780041cb070010
:10f07400f47b80000402e800f47b8800047c8000b8
:10f084000402e900047c88000a00370030002000f4
:10f094009709070000027800040f78008000eb0055
:10f0a40010002000cbca07000002eb00d4738800d4
:10f0b400000000001e027800040078000080fa00be
:10f0c400000006000200fa000002eb00040f7800c2
:10f0d400e4738000e20f520009003200e30f520093
:10f0e4001a003200e00f52000a003a000000eb0060
:10f0f4007f09070000027800040f7800140037002d
:10f10400100020007a09070000027800040f78003c
:10f114000f003700e4738000e00f52000c0032004f
:10f12400e4738000e20f520009003200e4738000af
:10f13400e30f5200060032008001eb00a2642d00b0
:10f14400b15f2d004016200028d007000000000009
:10f154004909070014002000e47388001e027800a7
:10f16400040078000080fa00000006001200fa0093
:10f1740070079800010f98000e0a9000e00f5200eb
:10f18400040034008e0a900004402000848f520052
:10f19400020034000082eb00420037000e0a9000a7
:10f1a4008402e90024002000809fbe0011000900b1
:10f1b4008402d80000027800810278004f00be006b
:10f1c4000402e800240798000002eb0014079800ea
:10f1d4000002eb00040f78002d00370004802000ab
:10f1e4001e02420004024200cfa2de00340798004f
:10f1f40045079800be0290004e02900085007800fa
:10f2040004007800020107000002be0054079800c1
:10f21400650798002e4a9000fe029000844a780008
:10f224007e0290000402e800740798001e02900019
:10f234000402e800140798009e0290000e0a900051
:10f24400848f520002003a000002eb0015003700e0
:10f254003e4a9000fe029000844a78007e029000ac
:10f264000402e800740798001e0290000402e800fb
:10f27400140798009e0290000e0a9000848f52009a
:10f2840002003a000002eb00060037001e0fe800ff
:10f294002e0290009e027800848f5200cfff35002a
:10f2a4000002eb00040078000080fa000000060071
:10f2b4001200fa0070079800010f98000e0a9000df
:10f2c400e00f5200040034008e0a90000440200035
:10f2d400848f5200020034000082eb005200370099
:10f2e4000e0a90008402e90024002000809fbe00e2
:10f2f400110009008402d80000027800810278001d
:10f304004f00be000402e800240798000002eb004e
:10f31400140798000002eb00040f78003d0037004a
:10f32400048020001e02420004024200cfa2de003c
:10f3340034079800450798001e0290000402e80074
:10f34400140798000e0a90000402e8009e02900040
:10f35400848f520007003d007e0290001442780022
:10f36400244f98007e0290000402e800740798007d
:10f374000200370000c2eb00244f98001e029000e8
:10f384000402e800140798000e0a90000402e80042
:10f394009e029000848f520007003d007e02900080
:10f3a40014427800344f98007e0290000402e80072
:10f3b400740798000200370000c2eb00344f980035
:10f3c4000042eb00444f98000042eb00544f980079
:10f3d400de0390006e039000be0290004e02900087
:10f3e4008701780006017800850078000400780021
:10f3f400520007003f0007009e0290000e0a900092
:10f40400848f5200020035000002eb000600370032
:10f414001e0fe8002e0290009e027800848f520096
:10f42400bfff35000002eb00040078000080fa0002
:10f43400000006000400fa0004002100050020007a
:10f44400048fbe009e0278001e02900085007800a2
:10f45400040078004a0007000080fa00000006005b
:10f464000c00fa000002eb00040f78000002eb002d
:10f4740014079800170037001e029000040242008f
:10f484000500200024079800350798003e029000ec
:10f49400044278000002fd0032e0b7000002fd00e3
:10f4a4002e0290001402ba00440798002e02900025
:10f4b4001482ba00540798004e029000de029000b5
:10f4c400040278001e0f42001e0290000402e800ad
:10f4d400140798009e029000f4bf2a00848f520003
:10f4e400e5ff36001e027800040078000080fa0070
:10f4f400000006000000fa0034002400043b8800e9
:10f5040054052000343b8800a40a2000343b8800c2
:10f5140061e7a800000000000000000000000000f7
:10f52400053b80000400280004826200e00f5200c2
:10f53400fbff3a000080fa00000006000800fa0011
:10f54400000f7800110798002207980033079800ed
:10f554001e027800044278000400780032e0b7000c
:10f564001e029000be029000050abb001e0290001d
:10f57400ae029000058abb000080fa00000006007d
:10f584000600fa00100798002107980024032000c1
:10f59400144278000482fb00040f78001e029000dd
:10f5a400044278000002fd0032e0b7000002fd00d2
:10f5b40024042400043b88002e029000ae02900034
:10f5c400050abb0054052000343b8800a40a20002f
:10f5d400343b880061e7a800000000000000000040
:10f5e40000000000053b8000040028000482620043
:10f5f400e00f5200fbff3a001e027800044278003c
:10f604000400780032e0b7000080fa000000060031
:10f614000800fa0020079800310798002e02900095
:10f62400044278000400780032e0b7003e02900003
:10f634001402ba00040f78003e0290001482ba004b
:10f64400140798001e02be000400be000080fa00e9
:10f65400000006000000fa000002eb0084088800a5
:10f664000002eb0034088800f47f2400640888005a
:10f6740084e0a90094e0a80011e1a8000080fa0049
:10f68400000006000000fa00fc00070000027800f9
:10f69400040078000080fa00000006000200fa006e
:10f6a400000f78001e02780014027800040078002d
:10f6b4000080fa00000006000200fa00000f780043
:10f6c4001e007800680007001e0078000200070092
:10f6d4000080fa00000006000200fa00000f780023
:10f6e4001e0378006022b800340398004503980094
:10f6f400db0007000002be001e037800140398001c
:10f70400250398000080fa00000006000600fa00b5
:10f7140020079800d20007000002be00048fbe003c
:10f724002e02900014027800e00f520023003200f1
:10f734002e029000a402900014029000be0f52000a
:10f74400ae8f5a000f0036002e0290003403900052
:10f75400c40390002e029000a402900014029000b2
:10f764003e014200ae814a000202be00060242008f
:10f7740087824a002e0390003403980045039800c2
:10f784000e0037002e02900034039000c403900052
:10f794002e029000a4029000140290003e01120078
:10f7a400ae811a000202be000602420087824a00ad
:10f7b4002e03900034039800450398002e02900015
:10f7c4001e03be0016029800270298002e02900025
:10f7d400c4029000340290006a2bb900060378003a
:10f7e4006020b90080037800070343008402780096
:10f7f400a4002000042ab800050343008602780010
:10f804000400be000080fa00000006000200fa00b6
:10f81400000f78001e007800bcff07001e0278006d
:10f8240015002000050a78001e027800c40290002a
:10f83400340290006a2bb900060378006020b900f6
:10f84400800378000703430084027800a4002000aa
:10f85400042ab80005034300860278000400be00b1
:10f864000080fa00000006000200fa00000f780091
:10f874001e007800a5ff07001e0278008002eb003e
:10f88400050a78001e027800c40290003402900039
:10f894006a2bb900060378006020b9008003780061
:10f8a4000703430084027800a4002000042ab8005f
:10f8b40005034300860278000400be000080fa00bd
:10f8c400000006000600fa00200798006400070004
:10f8d4000003be002e02900005002000041f430018
:10f8e40005974b00000000005d0007000002be0009
:10f8f4003e031200ae831a000602be00e00f52005f
:10f90400e08f5a00f8ff3c000080fa000000060077
:10f914000200fa00000f7800743e20009e02780076
:10f92400848f52000c0036001e027800e902420067
:10f93400a4002000811f7800110009008482d800ef
:10f944000002780081027800cf007800040078007b
:10f95400dcff0700160037001e027800e00f52009b
:10f964001300320004022000940888000002eb0017
:10f97400540888001e0278007d22b9000402780031
:10f98400740888008500a90013e1a800010037006d
:10f99400000000002504800004102000048262009e
:10f9a400e00f5200faff320013e1a9008500a9001c
:10f9b4000080fa00000006000200fa00000f780040
:10f9c400743821009e027800848f52000c003600a7
:10f9d400443820009e024200843e2000811f7800ab
:10f9e400110009008482d8000002780081027800a6
:10f9f400cf00780004007800c5ff07001600370028
:10fa04001e027800f40f5200130036000002eb00cf
:10fa1400940888000002eb0054088800c4fe270004
:10fa24001e02420004024200740888008500a900f6
:10fa340013e1a80001003700000000002504800045
:10fa44000410200004826200e00f5200faff32002a
:10fa540013e1a9008500a9000080fa000000060057
:10fa64000000fa0005000700848780009587800065
:10fa74000400be000080fa00000006000200fa0044
:10fa84007687800084878000958780000402780050
:10fa9400040f53001e0278006123b800848780009d
:10faa400958780000602420087824a008487880086
:10fab400958788001e027800040078000080fa0010
:10fac40000000600841f78000000fa000002eb002a
:10fad40034088800748780000402e8007487880072
:10fae40084e0a9000080fa004f027800004006007c
:10faf4000200fa00000f78001e027800e50f5200a1
:10fb040008003e001e02780084024200e40821003e
:10fb14000482420014027800641688001e027800f1
:10fb2400548588000002eb00748588000002eb0015
:10fb3400648588006022b8008485880095858800e3
:10fb44000080fa00000006000200fa0054858000dc
:10fb5400040fe8000d0037001e0278008402420002
:10fb6400a4092100048242009402780034858000b4
:10fb740004826200e00f5200030032001e0078008d
:10fb8400dbff07001d0037001e0fe8001e0278008f
:10fb9400e50f5200f0ff3600448580000402e800bf
:10fba400448588000002eb00040f78000d00370044
:10fbb4001e02780084024200a4092100048242004b
:10fbc400940278003485800004826200e00f5200c1
:10fbd400030032001e007800c5ff0700070037004d
:10fbe4001e0fe800548580009e027800848f520026
:10fbf400efff36000002eb00641688000080fa0074
:10fc0400000006000200fa00000f7800f403200050
:10fc14001e026200348588005485800084024200fc
:10fc2400a4092100048242009402780034858000f3
:10fc340004826200e00f520001003a00c2ff070094
:10fc44000080fa00000006000000fa000000eb004b
:10fc5400a7ff07000002eb004485880080ff07002f
:10fc64000002be00a4858800b58588000080fa00e3
:10fc7400000006000200fa00000f78001e0278005f
:10fc8400f80f52000a0036001e027800fe0f5200e0
:10fc940007003e009e0278007982520084024200ee
:10fca400840b210004824200140278001f003700f4
:10fcb4001e0278006123b800d4fe2f00f5ff2f0048
:10fcc4000602420087824a005600200007002000f6
:10fcd400860f5200878f5a0013003e000460010013
:10fce400050037000600370007003700080037001a
:10fcf400090037000a003700348480000b00370005
:10fd040044848000090037005484800007003700d1
:10fd140034858000050037004485800003003700e7
:10fd240054858000010037000002eb0004007800d5
:10fd34000080fa00000006000400fa00000f7800ba
:10fd4400110798001e0278006123b800d4fe2f002a
:10fd5400f5ff2f000602420087824a005600200069
:10fd640007002000860f5200878f5a002e003e00a5
:10fd740004600100050037000c0037001f00370045
:10fd84002100370026003700250037001e029000ae
:10fd9400e00f5200030032001e02900034848800f9
:10fda4002800370024002000270037001e0290009e
:10fdb400e90f52000f0036001e029000e5024200d7
:10fdc400a4002000809fbe00110009008482d80096
:10fdd40000027800810278004f00be00648488002d
:10fde400648480006a22b900040278004484880094
:10fdf4001400370024002000130037001e02900076
:10fe0400548488000f0037009e029000f403200001
:10fe140004826200040078007aff070009003700ba
:10fe240024002000080037001e027800f80f52005a
:10fe340002003600240020000300370014002000d4
:10fe4400010037000002eb00040078000080fa0093
:10fe5400000006000400fa00881f780000ff070075
:10fe64000002be00048fbe0034858000e00f520003
:10fe74003d003200a4858000b58580003e03520019
:10fe8400ae835a000602be00e00f5200e08f5a0013
:10fe940037003c0064848000050020003e034200db
:10fea400ae834a000602be00a4858800b58588009a
:10feb4007585800054848000848f520007003100cf
:10fec400748580000402e8007485880075858000cc
:10fed40054848000848f5200270039003ffb0700c0
:10fee400000278006123b800848580009585800035
:10fef4000602420087824a0084858800958588002e
:10ff0400648580000402e8006485880065858000bb
:10ff140034848000848f5200180039006485800086
:10ff2400e00f52000e003200588580008685800064
:10ff34009785800064858000050020000401be00d0
:10ff44000600be000bcc07000002be00840278004d
:10ff540008034400840b210004024300050a7800ce
:10ff6400f9fe070005003700000000000300370019
:10ff74000000000001003700000000004f0478007a
:10ff84000080fa00000006001000fa0060079800e4
:10ff9400710798000002eb00140798007e0290009d
:10ffa40014027800e50f520064003a006e029000db
:10ffb4000402e800144278000482fb004822dd00b9
:10ffc400240798006e0290000482e800144278002e
:10ffd4000482fb00ae0290000482720024079800a1
:10ffe4002e0290000402e800240798006e0290009c
:10fff40063024200144278000482fb004822dd00c0
:020000040001f9
:10000400340798006e0290006402420014427800a3
:100014000482fb00be029000048272003407980040
:100024003e029000e00f520041003200be029000f8
:10003400f47c2000848f52003d003e006e0290004c
:10004400440798007e0290008002eb00050a7800c5
:10005400ce02900014c0b300844a78004e0290008f
:100064000402e800440798007e029000140278001d
:100074008402e8007e029000050a78003e029000a7
:1000840067026200e00f5200050032003e02900059
:100094004322de0004427800044fe80003003700e6
:1000a4003e0290004322de00044f78004e0290008e
:1000b4001e4a78004e0290000402e80044079800ab
:1000c4007e029000140278008402e8007e02900010
:1000d400050a78008001eb003e019000ae0090001c
:1000e4004e009000b2c20700000278005407980046
:1000f4005e029000e00f5200050032005e009000a6
:10010400ab02070000027800140798000d003700c6
:100114007e029000940278001e4378000682fb0061
:10012400848242007e029000050a780005003700b0
:100134003400200014079800020037003400200027
:10014400140798001e029000040078000080fa0052
:10015400000006000c00fa004007980051079800c0
:100164000002eb00040f78005e0290001402780095
:10017400e50f52003e003a004e0290000402e800ef
:10018400144278000482fb004822dd001407980022
:100194004e0290000482e800144278000482fb00be
:1001a4009e02900004827200140798001e029000c0
:1001b4000402e800140798004e0290006402420012
:1001c40014427800e04f520026003a004e0290009c
:1001d4006302420014427800e14f420005003200fd
:1001e4004e0290006302420014427800e04f520035
:1001f4001c003a000042eb00744798004e02900045
:100204006302420014427800e14f420003003a00c6
:1002140014c0b30064479800020037000042eb00aa
:100224006447980066024700130020001200200073
:100234009e009000040078005dc207000002780070
:10024400240798002e029000e00f52000a003200aa
:100254002e0090005602070000027800040f780078
:100264000500370034002000040f78000200370036
:1002740034002000040f78001e0278000400780087
:100284000080fa00000006001000fa0060079800e1
:10029400710798000002eb00140798007e0290009a
:1002a40014027800e50f5200500036006e029000f0
:1002b4000402e800144278000482fb004822dd00b6
:1002c400240798006e0290000482e800144278002b
:1002d4000482fb00ae02900004827200240798009e
:1002e4002e0290000402e800240798006e02900099
:1002f40063024200144278000482fb004822dd00bd
:10030400340798006e0290006402420014427800a0
:100314000482fb00be02900004827200340798003d
:100324006e0290006502420094427800054f9800e6
:100334003e02900067026200e00f520005003200a6
:100344003e0290004322de0004427800044fe8009d
:10035400030037003e0290004322de00044f780081
:100364003e029000e00f52001d003200be029000d9
:10037400047b2000848f520019003e000e4a900036
:100384009e42780084cf520015003a006e0290001d
:1003940066024200130020003e019000ae0090006f
:1003a4000400780002c20700000278005407980095
:1003b4005e029000e00f5200050032005e009000e3
:1003c400fb010700000278001407980009003700b9
:1003d4007e02900055002000050a780005003700d1
:1003e4003400200014079800020037003400200075
:1003f400140798001e029000040078000080fa00a0
:0404040000000600ee
:020000040000fa
:020000040001f9
:100408000000fa000082eb00641988000002eb008b
:1004180044168800d8c2a900d8e2a900d902a900c8
:10042800d922a900d942a900d962a9000002eb008b
:1004380044178800f0c2a900f403200004178800bc
:10044800f042a800f062a800f102a8000002eb0048
:10045800641688000082eb00e41688000002eb00b6
:10046800641788000080fa00000006000200fa0005
:10047800000f7800000000001e027800e00f520014
:1004880002003200f4c2a80001003700f4c2a9003b
:10049800000000000080fa00000006000000fa00da
:1004a80000000000a41780004622de0061426200be
:1004b8000482fb00040078000080fa0000000600b7
:1004c8000400fa00000f7800110798001e02780057
:1004d800e10f52000e003a001e02900004f0a7003f
:1004e8000402ea000402ea004f22de000442780017
:1004f8000482fb006102620066178000e5ff2f009e
:1005080085026300048272006417880011003700b6
:100518001e027800e20f52000e003a001e02900000
:1005280004f0a7000402ea000402ea004f22de00f9
:10053800044278000482fb00610262000402420067
:1005480066178000d5ff2f008502630004827200c1
:10055800641788000080fa00000006000000fa0016
:100568001417800063026200040078000080fa001b
:10057800000006000400fa00000f78001107980038
:100588001e027800e10f52000f003a001e02900090
:1005980004f0a7000402ea000402e9004f22de008a
:1005a800044278000482fb00610262004222dd00fe
:1005b80066178000b5ff2f00850263000482720071
:1005c80064178800110037001e027800e20f5200fd
:1005d8000e003a001e02900004f0a7000402ea0090
:1005e8000402e9004f22de00044278000482fb0086
:1005f800610262004322dd006617800075ff2f004c
:100608008502630004827200641788000080fa0083
:10061800000006000000fa00141780006c02620057
:10062800040078000080fa00000006000400fa00c8
:10063800000f7800110798001e027800e10f5200a1
:100648000f003a001e02900004f0a7000402ea001e
:100658000402ea004f22de00044278000482fb0014
:10066800610262004422dd0066178000f5fe2f005b
:100678008502630004827200641788001100370045
:100688001e027800e20f52000e003a001e0290008f
:1006980004f0a7000402ea000402ea004f22de0088
:1006a800044278000482fb00610262004522dd00fa
:1006b80066178000f5fd2f00850263000482720032
:1006c800641788000080fa00000006000000fa00a5
:1006d800141780008402780004032000048262005a
:1006e800040078000080fa00000006000000fa000c
:1006f8001417800084027800f40f2000048262003e
:10070800040078000080fa00000006000000fa00eb
:10071800941780004222de00630262000400780021
:100728000080fa00000006000200fa00000f7800be
:100738001e02780014027800e00f52000500320013
:100748001e0278009402780004022000848f520070
:10075800020036000082eb002e0037001e027800ef
:10076800a4029000140290000660290007002000ef
:10077800860f5200878f5a001c003200066029003d
:1007880007002000860f5200878f5a000b003e009a
:100798000658220007002000860f5200878f5a0053
:1007a8001400320006b0240007002000860f520013
:1007b800878f5a00110032000a00370006102e00f9
:1007c80007002000860f5200878f5a000d00320064
:1007d80006202c0017002000860f5200878f5a0031
:1007e8000a0032000082eb000a0037000000000017
:1007f8000700370000000000050037000000000077
:10080800030037000000000001003700000000006e
:100818000002eb00040078000080fa0000000600e7
:100828001600fa00200f98000e82e800210120002f
:10083800040078004cfa07000e82e800010120004d
:10084800040078004400070000027800040f7800d4
:100858001e0a90009e0f5200020032000082eb0038
:10086800080037000e82e8000201200084007800aa
:100878002e08900071ca07002e089000aaff0700f2
:1008880000027800040078000080fa0000000600ea
:100898001400fa00100f98001e089000a2ff07002d
:1008a80000027800e00f5200020032000082eb00e4
:1008b80010003700020120009e0890000e0078000a
:1008c8005eca07000e0278000101200004007800cb
:1008d8002100070000027800040f9800d4fa0700ee
:1008e8000e02780021012000040078006ffa07004a
:1008f8000002eb00040078000080fa000000060007
:100908001200fa00220120008000eb000e0078009f
:1009180051ca0700a4aa2a00040f78000e02780022
:1009280001012000040078000b0007000002780095
:10093800040f9800befa07000e027800210120007b
:100948000400780059fa07000002eb000400780060
:100958000080fa00000006000800fa00200798004e
:10096800310798000002eb00140798000002eb0022
:10097800040f7800090037001e027800ae029000cc
:1009880004824200144278000402fb009e02900098
:1009980004824200140798001e0fe8003e029000ef
:1009a8009e027800848f5200f3ff35001e029000eb
:1009b800040078000080fa00000006001000fa0029
:1009c8005007980061079800624f9800734f98008d
:1009d8007e4a90000482fb00040f78006e4a900063
:1009e800e84f5200050036008001eb00827c2d00a4
:1009f800517d2d0080032000fbc907006e02900086
:100a08004322de00140798001e0290004322dd00f6
:100a1800ee02900004825200240798002e029000f3
:100a28009e027800042add00040f78006e4a9000c8
:100a38000482fb0015002000042add000402e900fe
:100a4800340798001e0290004322dd00ee02900059
:100a580004825200be029000042add003407980088
:100a6800de0290001e0290000482420014427800c8
:100a78000482fb00440798001e0290000402e8006c
:100a8800de02900004824200144278000482fb00d7
:100a98004822dd00ce0290000482720044079800cc
:100aa8003e0290008482ea004e02900004826200b6
:100ab8001e02720044079800de0290001e02900099
:100ac800848242004e02900004427800844a7800f2
:100ad8001e0290000402e800de02900084824200b8
:100ae8004e0290004822de0004427800844a7800d2
:100af8000080fa00000006000e00fa004007980087
:100b080051079800424f98005e0290004322de0091
:100b1800040f78001e0278004322dd00de029000f8
:100b280004825200140798004e4a90000482fb0089
:100b380015002000042add000402e90024079800bb
:100b48004e0290001e024200144278000482fb000c
:100b5800340798001e02e800ce029000048242008a
:100b6800144278000482fb004822dd00be02900097
:100b780004827200340798001e029000be029000a2
:100b8800042ade0034079800be0290002e0290006e
:100b980004826200340798003e0290000442780004
:100ba800044078000080fa00000006000400fa0003
:100bb800100798001e029000e10f52000800320052
:100bc800e10f520003003900e70f5200070032001e
:100bd800090037000002eb00040f78000900370015
:100be80024002000040f780006003700640020006d
:100bf800040f78000300370044002000040f780039
:100c0800000000001e027800040078000080fa004e
:100c1800000006000400fa00004f78001107980051
:100c28001e0090004200070000027800e00f52000a
:100c3800020032000002eb000f0037001e02900095
:100c4800940278001e029000140290000482420070
:100c58001e4a78001e029000140290008402e800e8
:100c68001e02900034029000848262001e029000ee
:100c78001502980014002000040078000080fa0093
:100c8800000006000400fa00000f78001107980021
:100c98001e0090003800070000027800e00f5200a4
:100ca800050032009e0278000042eb00844a78007a
:100cb8000002eb00110037001e0290009402780039
:100cc8001e02900024029000048242001442780020
:100cd8009e027800844a78001e0290002402900048
:100ce8008402e8001e0290003402900084826200b0
:100cf8001e029000250298001400200004007800cd
:100d08000080fa00000006000200fa00000f7800d8
:100d18001e0278008002eb00250298001e0278006f
:100d28008002eb00150298000080fa00000006001f
:100d38000200fa00000f78001e02780014029000ea
:100d48008402e8001e027800340290008482620067
:100d58001e02780024029000848f520002003a009c
:100d680014002000010037000002eb0004007800a6
:100d78000080fa00000006000200fa00000f780068
:100d88001e027800a40290001e027800140290004f
:100d9800848f520002003a0014002000010037003e
:100da8000002eb00040078000080fa000000060052
:100db8000200fa00000f78001e02780094029000ea
:100dc8001e02780024029000848252001e027800dd
:100dd8003402900004826200040078000080fa0067
:100de800000006001000fa006007980071079800dc
:100df8000002eb00140798007e02900014027800ad
:100e0800e50f520063003a006e0290000402e80009
:100e1800144278000482fb004822dd002407980071
:100e28006e0290000482e800144278000482fb00fd
:100e3800ae02900004827200240798002e029000ef
:100e48000402e800240798006e0290006302420042
:100e5800144278000482fb004822dd003407980021
:100e68006e02900064024200144278000482fb0083
:100e7800be02900004827200340798003e0290007f
:100e8800e00f520040003200be029000f47c2000c7
:100e9800848f52003c003e006e0290004407980088
:100ea8007e0290008002eb00050a7800ce029000d6
:100eb80024c0b300844a78004e0290000402e8007f
:100ec800440798007e029000140278008402e8002b
:100ed8007e029000050a78003e02900067026200d8
:100ee800e00f5200050032003e0290004322de006f
:100ef80004427800044fe800030037003e029000e7
:100f08004322de00044f78004e0290001e4a78000b
:100f18004e0290000402e800440798007e02900008
:100f2800140278008402e8007e029000050a780026
:100f38003e019000ae0090004e009000f8bf070000
:100f480000027800540798005e029000e00f5200fb
:100f5800050032005e00900014ff070000027800d0
:100f6800140798000d0037007e0290009402780064
:100f78001e4378000682fb00848242007e029000b5
:100f8800050a78000500370034002000140798008f
:100f98000200370034002000140798001e02900059
:100fa800040078000080fa00000006000e00fa0035
:100fb80050079800610798000002eb00040f7800c2
:100fc8006e02900014027800e50f52005a003a00b1
:100fd8005e0290000402e800144278000482fb00dc
:100fe8004822dd00140798005e0290000482e800a1
:100ff800144278000482fb009e0290000482720072
:10100800140798001e0290000402e80014079800d4
:101018005e02900063024200144278000482fb00e2
:101028004822dd00240798005e0290006402420016
:10103800144278000482fb00ae0290000482720021
:10104800240798002e029000e00f5200370032006b
:10105800ae029000c4072000848f520033003e0087
:101068005e029000340798006e0290008002eb0048
:10107800050a7800be02900044c0b300844a780094
:101088003e0290000402e800340798006e029000c7
:10109800140278008402e8006e029000050a7800c5
:1010a8002e0290000442780004424200be029000e2
:1010b800844a78003e0290000402e8003407980051
:1010c8006e029000140278008402e8006e0290001c
:1010d800050a78002e0190009e0090003e009000c6
:1010e8008dbd070000027800440798004e0290006a
:1010f800e00f5200050032004e009000abfe0700e2
:1011080000027800040f78000d0037006e0290008e
:10111800940278002e029000040242008482420069
:101128006e029000050a78000500370034002000a0
:10113800040f78000200370034002000040f780004
:101148001e027800040078000080fa000000060003
:101158000000fa0040a7a9002535800004fc2f00f4
:10116800048262006401b30024358800a53680003b
:1011780004fc2f00048262003400b300a436880007
:101188003535800004fc2f00048262007401b3002e
:1011980034358800c5368000f40f2c008482620044
:1011a8000450200004827200c4368800153580007f
:1011b800f40f2c00848262000480210004827200f3
:1011c8001435880055368000f40f2c0084826200a4
:1011d80004c021000482720054368800453580001e
:1011e80004fc2f00048262003401b30044358800f7
:1011f800d536800004fc2f00048262007400b3001e
:10120800d4368800d5368000f40f2c008482620022
:101218000480200004827200d4368800153a8000c9
:101228000404200004837200640420007505200073
:1012380027742000844b7800854b7800864b780013
:10124800000000007007a8007067a9007087a80058
:1012580070a7a90070c7a90070e7a8007167a90066
:101268007187a90071a7a90071c7a80071e7a80034
:101278007207a8007227a8007247a8007267a80022
:101288007287a80072a7a80072c7a80072e7a80012
:101298007307a8007327a8007347a8007367a800fe
:1012a8007387a80073a7a80073c7a80073e7a800ee
:1012b8007427a8007447a8007467a9007507a800d8
:1012c8007527a8007547a80074e7a8007627a80026
:1012d8007647a8007667a80076a7a8007427a80014
:1012e8007807a8007907a8007a07a8000080fa0004
:1012f800000006000000fa000080fa000000060066
:101308000400fa00100798001e0290006123b8003c
:1013180004ff2f00f5ff2f000602420087824a00d3
:10132800f600200007002000860f5200878f5a0021
:1013380029003e00046001000f003700120037004a
:10134800130037002400370023003700220037003d
:1013580021003700200037001f0037001e0037002b
:101368001d0037001c0037001b0037001a0037002b
:101378001900370009003700646a8000756a800028
:10138800040278001f003700441020001d003700b9
:10139800d6fc0700000278001a0037009417800076
:1013a8006402620004f0a7000402ea00040fea00e5
:1013b8001e0278004f22de00040f78009417800088
:1013c80068026200e00f5200010032001e10a00007
:1013d8001e0278000b0037001e029000f20f520028
:1013e800070036001e029000fe0f520004003e0067
:1013f8001e0090001efa0700000278000100370066
:101408000002eb00040078000080fa0000000600eb
:101418000400fa00000f7800110798001e027800f7
:10142800f20f5200080036001e027800fe0f52002c
:1014380005003e009e0090001e0078003dfa07005f
:101448000002780001003700140020000400780032
:101458000080fa00000006000a00fa002047980001
:101468002107980032079800430798000002eb0014
:10147800040f78004e0290000482e800ff0f52002b
:1014880024003e000002eb001483880014838000cf
:1014980025042100850242002e439000864a7800e8
:1014a8000402e80014838800158380002e0290004f
:1014b800e00f52000200320000c2eb0001003700ca
:1014c8000042eb002604210006834200044b78000a
:1014d8000502e800148388004e029000e00f5200d5
:1014e8000e0032001583800024042100048242008b
:1014f8004e019000be009000040078004fc707001e
:10150800158380004e0290000482420014838800f4
:101518000200370044002000040f78001e02780003
:10152800040078000080fa00000006000400fa00b9
:10153800000f780011079800158380001e02e8004c
:101548000501780021042100040078003bc707004a
:10155800148380008402e8001e029000050a7800c7
:101568000002eb00040078000080fa00000006008a
:101578000800fa00200798003107980000c2eb0025
:10158800044f780000c2eb0014479800130037009e
:101598002e029000944278001e42900004c26a0015
:1015a8000482fb00140798002e0290000402e80051
:1015b80024079800653d2d001e0290000482420019
:1015c800144278001e426a0014479800654d2d00a9
:1015d8001e02900004824200144f78003e029000e0
:1015e80004f0a7000402ea000402ea004f22de0029
:1015f80004427800be0290008502e9003507980091
:10160800e04f5200e2ff3a009e4278000582fb005c
:10161800c822dd001e4290000482fb000482720092
:0c162800040078000080fa0000000600ba
:020000040000fa
:020000040001f9
:101634000200fa00000f78009460a8008460a900fa
:1016440004ca2000140888000002eb002408880063
:1016540014002000040078000080fa000000060056
:101664000000fa000002eb000408880005e1a8006d
:101674000080fa00000006000000fa0017c207000c
:1016840005e1a9008460a90021c207000080fa00d6
:10169400000006003600f800809fbe00829fbe0056
:1016a400849fbe00869fbe000000fa008460a900eb
:1016b400b4838000040001000080fa004f03be00e0
:1016c4004f02be004f01be004f00be003600f900bd
:1016d400004006000000fa000002eb00b487880016
:1016e40014002000040078000080fa0000000600c6
:1016f4000200fa00000f780014002000b48788006c
:101704001e027800a48788001400200004007800da
:101714000080fa00000006000400fa001007980098
:101724000002eb00040f7800b4878000e00f520041
:1017340007003200a58780001e029000050a780089
:101744000002eb00b487880014002000040f780026
:101754001e027800040078000080fa0000000600f1
:020000040000fa
:020000040005f5
:0457f400023e000071
:020000040000fa
:020000040005f5
:0457f800bdfa0000f6
:020000040000fa
:020000040005f5
:0457fc007f3f0000eb
:00000001FF
